:020000040806ec
:1000000000000608b89016080000b6141c00040191
:100010000200360800000000005000102100060811
:100020000d490e4a0e4b9b1a03dd043bc858d050b5
:10003000fbdc0b490b4a0020521a02dd043a8850bf
:10004000fcdc0949094a0a4b9b1a03dd043bc858ea
:10005000d050fbdc07488047281a160820510010b2
:1000600040c6001078200210800006080000000240
:10007000a819100281000002780afa790100000034
:10008000f83d0e02e0b20d023cb30d0284430e02b5
:1000900058420e02a8410e02ac440e02e8400e0285
:1000a00050440e020c450e0274b40d0224b40d022d
:1000b00050400e0254450e0238440e02a43f0e0278
:1000c00098410e02e0e00d02d4b40d023c430e0252
:1000d0006c430e02b8420e021c440e02d0450e02c2
:1000e000703e0e02ac430e02fc440e02ac3f0e0208
:1000f000b4450e02683e0e02ffffffffffffffff49
:100100005bf074fb1ff058fb28f00eff1ff0e0fbc4
:1001100081f0004102e000bf83f0004330b54feab8
:1001200041044fea430594ea050f08bf90ea020f25
:100130001fbf54ea000c55ea020c7fea645c7feab8
:10014000655c00f0e2804fea5454d4eb5555b8bfdb
:100150006d420cdd2c4480ea020281ea030382ea4c
:10016000000083ea010180ea020281ea0303362dde
:1001700088bf30bd11f0004f4fea01314ff4801cb1
:100180004cea113102d0404261eb410113f0004fc3
:100190004fea03334cea133302d0524263eb43037a
:1001a00094ea050f00f0a780a4f10104d5f1200e18
:1001b0000ddb02fa0efc22fa05f2801841f1000173
:1001c00003fa0ef2801843fa05f359410ee0a5f147
:1001d00020050ef1200e012a03fa0efc28bf4cf078
:1001e000020c43fa05f3c01851ebe37101f000452e
:1001f00007d54ff0000edcf1000c7eeb00006eeb3b
:100200000101b1f5801f1bd3b1f5001f0cd34908c4
:100210005fea30004fea3c0c04f101044fea44521b
:1002200012f5800f80f09a80bcf1004f08bf5feaa2
:10023000500c50f1000041eb045141ea050130bd82
:100240005fea4c0c404141eb0101013c28bfb1f594
:10025000801fe9d291f0000f04bf01460020b1fadf
:1002600081f308bf2033a3f10b03b3f120020cdab2
:100270000c3208dd02f1140cc2f10c0201fa0cf090
:1002800021fa02f10ce002f11402d8bfc2f1200cf5
:1002900001fa02f120fa0cfcdcbf41ea0c019040ab
:1002a000e41aa2bf01eb0451294330bd6fea0404f4
:1002b0001f3c1cda0c340edc04f11404c4f12002df
:1002c00020fa04f001fa02f340ea030021fa04f3f1
:1002d00045ea030130bdc4f10c04c4f1200220fa48
:1002e00002f001fa04f340ea0300294630bd21fa86
:1002f00004f0294630bd94f0000f83f4801306bf4c
:1003000081f480110134013d4ee77fea645c18bf3f
:100310007fea655c29d094ea050f08bf90ea020fd6
:1003200005d054ea000c04bf1946104630bd91eace
:10033000030f1ebf0021002030bd5fea545c05d1d1
:100340004000494128bf41f0004130bd14f5800410
:100350003cbf01f5801130bd01f0004545f0fe4184
:1003600041f470014ff0000030bd7fea645c1abfb9
:10037000194610467fea655c1cbf0b46024650eaf0
:10038000013406bf52ea033591ea030f41f400211c
:1003900030bd00bf90f0000f04bf0021704730b5a2
:1003a0004ff4806404f132044ff000054ff0000177
:1003b00050e700bf90f0000f04bf0021704730b538
:1003c0004ff4806404f1320410f0004548bf40420d
:1003d0004ff000013ee700bf42004feae2014fea62
:1003e00031014fea02701fbf12f07f4393f07f4f3d
:1003f00081f06051704732f07f4208bf704793f040
:100400007f4f04bf41f40021704730b54ff4607452
:1004100001f0004521f000411ce700bf50ea010255
:1004200008bf704730b54ff000050ae050ea0102fe
:1004300008bf704730b511f0004502d5404261eb6e
:1004400041014ff4806404f132045fea915c3ff4af
:10045000d8ae4ff003025feadc0c18bf03325fea4c
:10046000dc0c18bf033202ebdc02c2f1200300fafd
:1004700003fc20fa02f001fa03fe40ea0e0021fa22
:1004800002f11444bde600bf70b54ff0ff0c4cf410
:10049000e06c1cea11541dbf1cea135594ea0c0fc2
:1004a00095ea0c0f00f0def82c4481ea030621eafd
:1004b0004c5123ea4c5350ea013518bf52ea033538
:1004c00041f4801143f4801338d0a0fb02ce4ff0ea
:1004d0000005e1fb02e506f00042e0fb03e54ff01a
:1004e0000006e1fb03569cf0000f18bf4ef0010e12
:1004f000a4f1ff04b6f5007f64f5407404d25fea0e
:100500004e0e6d4146eb060642eac62141ea5551c0
:100510004feac52040ea5e504feace2eb4f1fd0c02
:1005200088bfbcf5e06f1ed8bef1004f08bf5fea80
:10053000500e50f1000041eb045170bd06f0004632
:1005400046ea010140ea020081ea0301b4eb5c04df
:10055000c2bfd4eb0c0541ea045170bd41f48011d7
:100560004ff0000e013c00f3ab8014f1360fdebffc
:10057000002001f0004170bdc4f10004203c35dad8
:100580000c341bdc04f11404c4f1200500fa05f35b
:1005900020fa04f001fa05f240ea020001f00042fc
:1005a00021f0004110ebd37021fa04f642eb060172
:1005b0005eea430e08bf20ead37070bdc4f10c049c
:1005c000c4f1200500fa04f320fa05f001fa04f260
:1005d00040ea020001f0004110ebd37041f100014c
:1005e0005eea430e08bf20ead37070bdc4f1200557
:1005f00000fa05f24eea020e20fa04f301fa05f2bf
:1006000043ea020321fa04f001f0004121fa04f266
:1006100020ea020000ebd3705eea430e08bf20ea36
:10062000d37070bd94f0000f0fd101f00046400070
:1006300041eb010111f4801f08bf013cf7d041eaf2
:10064000060195f0000f18bf704703f000465200f6
:1006500043eb030313f4801f08bf013df7d043eac7
:100660000603704794ea0c0f0cea135518bf95ea7d
:100670000c0f0cd050ea410618bf52ea4306d1d104
:1006800081ea030101f000414ff0000070bd50ea23
:10069000410606bf1046194652ea430619d094eaad
:1006a0000c0f02d150ea013613d195ea0c0f05d197
:1006b00052ea03361cbf104619460ad181ea0301eb
:1006c00001f0004141f0fe4141f470014ff00000a3
:1006d00070bd41f0fe4141f4780170bd70b54ff03e
:1006e000ff0c4cf4e06c1cea11541dbf1cea1355be
:1006f00094ea0c0f95ea0c0f00f0a7f8a4eb0504a0
:1007000081ea030e52ea03354fea013100f0888096
:100710004fea03334ff0805545ea131343ea12635f
:100720004fea022245ea111545ea10654fea002614
:100730000ef000419d4208bf964244f1fd0404f5cd
:10074000407402d25b084fea3202b61a65eb030529
:100750005b084fea32024ff480104ff4002cb6ebe6
:10076000020e75eb030e22bfb61a754640ea0c0066
:100770005b084fea3202b6eb020e75eb030e22bfa6
:10078000b61a754640ea5c005b084fea3202b6ebe7
:10079000020e75eb030e22bfb61a754640ea9c00a6
:1007a0005b084fea3202b6eb020e75eb030e22bf76
:1007b000b61a754640eadc0055ea060e18d04fea34
:1007c000051545ea16754fea06164feac30343ead4
:1007d00052734feac2025fea1c1cc0d111f4801fa1
:1007e0000bd141ea00014ff000004ff0004cb6e79a
:1007f00011f4801f04bf01430020b4f1fd0c88bf39
:10080000bcf5e06f3ff6afaeb5eb030c04bfb6eb43
:10081000020c5fea500c50f1000041eb045170bd36
:100820000ef0004e4eea113114eb5c04c2bfd4eb63
:100830000c0541ea045170bd41f480114ff0000ee7
:10084000013c90e645ea060e8de60cea135594ea63
:100850000c0f08bf95ea0c0f3ff43baf94ea0c0f66
:100860000ad150ea01347ff434af95ea0c0f7ff4db
:1008700025af104619462ce795ea0c0f06d152ea2f
:1008800003353ff4fdae1046194622e750ea410613
:1008900018bf52ea43067ff4c5ae50ea41047ff424
:1008a0000daf52ea43057ff4ebae12e74ff0ff3c89
:1008b00006e000bf4ff0010c02e000bf4ff0010c5a
:1008c0004df804cd4fea410c7fea6c5c4fea430cd3
:1008d00018bf7fea6c5c1bd001b050ea410c0cbf22
:1008e00052ea430c91ea030f02bf90ea020f002084
:1008f000704710f1000f91ea030f58bf994208bfeb
:1009000090422cbfd8176feae37040f001007047a7
:100910004fea410c7fea6c5c02d150ea013c07d1fe
:100920004fea430c7fea6c5cd6d152ea033cd3d049
:100930005df8040b704700bf8446104662468c4643
:100940001946634600e000bf01b5fff7b7ff002876
:1009500048bf10f1000f01bd4df808edfff7f4ff9f
:100960000cbf012000205df808fb00bf4df808ed2a
:10097000fff7eaff34bf012000205df808fb00bf4d
:100980004df808edfff7e0ff94bf012000205df86f
:1009900008fb00bf4df808edfff7ceff94bf012024
:1009a00000205df808fb00bf4df808edfff7c4ff1d
:1009b00034bf012000205df808fb00bf4fea410c66
:1009c0007fea6c5c02d150ea013c0ad14fea430c49
:1009d0007fea6c5c02d152ea033c02d14ff0000086
:1009e00070474ff0010070474fea410212f50012c4
:1009f00015d211d56ff47873b3eb625212d94fea66
:100a0000c12343f0004343ea505311f0004f23fa4f
:100a100002f018bf404270474ff00000704750eaa4
:100a2000013005d111f0004008bf6ff00040704761
:100a30004ff00000704700bf4a0011d212f50012bb
:100a400011d20dd56ff47873b3eb62520ed44fea26
:100a5000c12343f0004343ea505323fa02f07047a6
:100a60004ff00000704750ea013002d14ff0ff30e4
:100a700070474ff0000070477bb972b90029bebfc4
:100a800000204ff0004106e008bf00281cbf6ff0b7
:100a900000414ff0ff3000f0e1b9adf1080c6de915
:100aa00004ce002909db002b1adb00f061f8ddf829
:100ab00004e0dde9022304b07047404261eb4101ec
:100ac000002b1bdb00f054f8ddf804e0dde9022325
:100ad00004b0404261eb4101524263eb4303704773
:100ae000524263eb430300f043f8ddf804e0dde934
:100af000022304b0404261eb41017047524263eb74
:100b0000430300f035f8ddf804e0dde9022304b02a
:100b1000524263eb4303704753b94ab9002908bff7
:100b200000281cbf4ff0ff314ff0ff3000f096b9a6
:100b3000adf1080c6de904ce00f01af8ddf804e020
:100b4000dde9022304b07047430803f05533c01aaf
:100b5000830800f0333003f03333184400eb1010f7
:100b600000f00f3000eb002000eb0040000e70475b
:100b70002de9f04f099d04460f46002b48d18a42cb
:100b8000944661d9b2fa82f343b1c3f120019f4088
:100b900002fa03fc9c4020fa01f10f434fea1c418a
:100ba0001ffa8cfe220cb7fbf1f601fb167706fb51
:100bb0000ef042ea0742904208d91ceb020206f10d
:100bc000ff3702d2904200f237813e46121aa4b299
:100bd000b2fbf1f001fb102200fb0efe44ea0244de
:100be000a64508d91ceb040400f1ff3202d2a64549
:100bf00000f21c81104640ea0640a4eb0e040026d9
:100c00001db1dc400023c5e900433146bde8f08f4b
:100c10008b4209d9002d00f0fd800026c5e90001b6
:100c200030463146bde8f08fb3fa83f6002e4bd143
:100c30008b42c0f0f280824240f2ef803046002dbd
:100c4000e3d0c5e90047e0e702b9ffdeb2fa82f37c
:100c5000002b40f09d80891a4fea124e97b2012670
:100c6000200cb1fbfef20efb121140ea014107fb22
:100c700002f088420fd91ceb010102f1ff382cbfb2
:100c80004ff001094ff00009884203d9b9f1000f74
:100c900000f0cf804246091aa4b2b1fbfef00efb71
:100ca000101100fb07f744ea0144a74208d91cebe6
:100cb000040400f1ff3102d2a74200f2b4800846da
:100cc000e41b40ea02409be7c6f12007b34001fa6b
:100cd00006f422fa07fcf940b2404cea030c20fa71
:100ce00007f34fea1c491c431ffa8cfe00fa06f377
:100cf000200cb1fbf9f809fb181140ea014108fb8f
:100d00000ef088420fd91ceb010108f1ff3a2cbf0d
:100d10004ff0010b4ff0000b884203d9bbf1000fdd
:100d200000f08d80d046091aa4b2b1fbf9f009fb9e
:100d3000101100fb0efe44ea01418e4507d91ceb61
:100d4000010100f1ff3401d28e457fd8204640eaf0
:100d50000840a1eb0e01a0fb029841454c46c64657
:100d600002d306d14b4504d20138b9eb020468eb3b
:100d70000c0e002d70d01a1b61eb0e0122fa06f347
:100d800001fa07f7f14000261f43c5e900713ce76f
:100d900002fa03fcc3f1200001fa03f221fa00f683
:100da0004fea1c4e24fa00f11ffa8cf79c401143c5
:100db000b6fbfef00a0c0efb106642ea064200fb90
:100dc00007f696420ed91ceb020200f1ff382cbf49
:100dd0004ff001094ff00009964202d9b9f1000f16
:100de00031d04046921b89b2b2fbfef60efb1622b2
:100df00041ea024106fb07f28a4207d91ceb0101d6
:100e000006f1ff3801d28a4223d84646891a46eabb
:100e1000004625e72e462846f7e6841a61eb0303d1
:100e200001201f460be76444023849e76444023856
:100e3000e1e6023a61442ee7023e6244c6e6a8f1ca
:100e4000020861446fe702386244cbe7023861442c
:100e50007de7023e6144d9e72e46d6e6704700bfe3
:100e600010f8012b11f8013b012a28bf9a42f7d054
:100e7000d01a7047034613f8012b002afbd1181a29
:100e80000138704709b504480068044b03441b68e7
:100e90001b68029309bd000088cc0010040000000c
:100ea00009b504480068044b03441b685b6802935f
:100eb00009bd000088cc00100400000009b50448fa
:100ec0000068044b03441b689b68029309bd000043
:100ed00088cc00100400000000b1807b704708b18e
:100ee000c07b7047ff20704708b1408970474ff6bc
:100ef000ff70704708b1808970474ff6ff707047e8
:100f000042680068101a704709b504480068044b2d
:100f100003441b681b68029309bd000088cc0010c5
:100f2000000000007047000010b5002101201ef0f5
:100f300083fa04461ef002fb24b9bde810400420e9
:100f40000df0fabf0028f8d1024831f0edfd00287d
:100f5000f3d110bd60cc001008b50ef00bf80438ca
:100f600018bf012008bd000010b5fff7f5ff20b144
:100f7000bde81040014bdb69184710bd60cc001084
:100f800010b5fff7e9ff20b1bde81040014b5b6ae7
:100f9000184710bd60cc001010b5fff7ddff20b181
:100fa000bde81040014b1b6a184710bd60cc001013
:100fb000f8b504460e4617461d4624b92846bde836
:100fc000f84029f06ebce72000f042f9304629f0e5
:100fd00068fce72000f060f9384629f062fc013c2b
:100fe000ebe70000014b1860704700bf8ccc00108d
:100ff0002de9ff410446002003911ef0d1fc234b54
:101000001b6813b12046039998474ff47f0000f006
:101010007ff8602000f09ef800f090f80023009325
:1010200001231b4a18461b4901f042fce72000f04f
:1010300033f94ff47f0000f06bf80226164ddff80d
:101040006880164f2b4641460320134afff7b0ff36
:101050002b4639460320104afff7aaff2a4641468d
:1010600003200f4bfff7a4ff3a4620460d4b0b49d8
:10107000fff79eff012e07d100222146822004b0f7
:10108000bde8f0411ef02cba0126dbe78ccc001045
:1010900029360e02ccb40d02a0860100e0930400b4
:1010a000a0bb0d0000350c00f049020037b500254b
:1010b0000195069d079c009500f074fa04b120602c
:1010c0007f28a8bf7f2040b203b030bd10b5054bcc
:1010d0001b7800fb03f4044b0020db689847604357
:1010e000000c10bd3a5100102051001038b50546d3
:1010f000c0f307400c46fff7e9ff2080c5f3072047
:10110000fff7e4ff6080e8b2fff7e0ffa08038bda2
:10111000014b1860704700bf94cc0010014b186061
:10112000704700bf98cc001010b9024b1868704788
:10113000014bfbe794cc001098cc0010044b1a78bc
:1011400022b100210120197001f0cebc704700bf10
:1011500090cc0010014b1870704700bf3a5100103e
:10116000014b1878704700bf3a510010024b1860cd
:10117000024b1960704700bf9ccc0010a0cc00103f
:1011800010b5054b0446db68002098472402b4fbe9
:10119000f0f0c0b210bd00bf205100102de9f341a6
:1011a000dff83480044600216846d8f808309847b4
:1011b0006e46671e02340020d8f80c3036f8025b09
:1011c00098472d02b5fbf0f507f8015fa742f2d171
:1011d00002b0bde8f08100bf2051001010b4054bf3
:1011e00082885c684188a446002300885df8044b2f
:1011f000604700bf2051001030b50e4d85b0044649
:10120000fff7ecff2b689bb12088fff7b9ff039035
:101210006088fff7b5ff0290a088fff7b1ffdde916
:10122000022103460020009003482c680068a04774
:1012300005b030bd9ccc0010a0cc001007b56946ad
:10124000fff754ff6846fff7d7ff03b05df804fbd4
:1012500008b510b1e72805d008bd0120bde8084059
:1012600028f0bfbc074b1b7853b1074b1868fff73a
:10127000e5ff6322054b1a70ff22054b1a70ebe75e
:10128000044bf3e790cc001098cc001039510010bb
:101290003851001094cc001008b510b1e72804d0e4
:1012a00008bdbde8084028f09cbc0020fff7c6ff41
:1012b0000022034b1a700122024b1a70f0e700bfa4
:1012c000395100103851001013b518b1e72807d074
:1012d00002b010bd104b5b6902b0bde8104018476a
:1012e0000e4b1b78a3b10e4b1c680b4b00219b6867
:1012f00068469847bdf80220bdf800301343bdf89a
:10130000042013439bb22bb10020fff797ffdfe7c8
:10131000044be9e72046f8e72051001090cc00107c
:1013200098cc001094cc001038b5094b1a7802f014
:10133000ff0462b90125214620461d7001f0d4fb4f
:101340002046fff77bff034b1c70034b1d7038bd1d
:1013500090cc0010395100103851001013b50446dc
:1013600008466946fff7c2fe6322bdf800306343ba
:10137000b3fbf2f3adf80030bdf802306343b3fbca
:10138000f2f3adf80230bdf8043004fb03f0b0fb1b
:10139000f2f0adf804006846fff72eff02b010bd72
:1013a00010b40f4c024623780e4983b9012008700f
:1013b0000878e72a0344d8b220700ed10a4b1b7874
:1013c0004bb10a4b19685df8044bfff7c7bf632b9d
:1013d000eed1ff20ebe7064bf4e75df8044b7047d6
:1013e000395100103851001090cc001098cc0010ea
:1013f00094cc0010024b1878003818bf01207047b9
:1014000090cc001084b030b503ac84e80f00064cdb
:1014100003ad0fcd0fc495e8030084e80300bde8d9
:10142000304004b0704700bf2051001070b5054631
:1014300000200e46144638f0a3fe40b12346324643
:10144000696840305ff092fe231a5842584170bddf
:1014500070b5054600200e46144638f091fe40b1a6
:10146000234632466968403060f03bf8231a584200
:10147000584170bd01211020c3f068bb08b510b100
:10148000c3f05afd012008bd01210c20c3f05ebb52
:1014900008b510b1c3f050fd012008bd30b50446b9
:1014a00085b078b1684640f00fff6a46234604ad28
:1014b000144603ccac4218605960224603f108037d
:1014c000f6d1012005b030bd1fb5044648b101a8d2
:1014d00041f0a0fa01ab03cb206018686160a06006
:1014e000012004b010bd000038b50d46044608b90f
:1014f000002038bd0029fbd0002038f041fe002834
:10150000f6d00023e360044b0120c4e900354ff01e
:10151000ff33a360ede700bfad130002f8b50e4640
:10152000054608b90020f8bd0029fbd0002038f09e
:1015300027fe04460028f5d04034314620465ff0af
:101540001afc0746314620465ff017fc002fe9db06
:101550000028e7db034bc01ba860c5e9003601206b
:10156000e1e700bfd1130002002908bf3221024b7e
:101570001970024b186070473b510010a8cc001046
:1015800070470cb402b07047034b1860034b1960ee
:10159000034b1a60704700bfaccc0010b0cc0010f9
:1015a000a4cc00102de9f04f4ff0010c00244ff0b7
:1015b000ff36d0f804e0964504d211f80e80b8f159
:1015c000000f09d18268511e03eb0213002980f23b
:1015d000a8812046bde8f08fb8f13a0f7dd033d80e
:1015e000b8f1220f00f0a58010d8a8f109085ffa21
:1015f00088f8b8f1170f0dd8ac4d0cfa08f818eab6
:10160000050f07d0456801354560d2e7b8f12c0fca
:1016100000f02981d0f8048042450ed911f8085015
:101620005db13a2d00f25e811f2d00f246810a2d38
:1016300000f25581082d40f24b81002b40f057817c
:1016400008f1ff354560a4e0b8f17b0f1dd00ad842
:10165000b8f15b0f19d0b8f15d0fdbd1002bd1d001
:101660004ff0020906e0b8f17d0fd3d1002bc9d0ad
:101670004ff001098568013d03eb0518002d2fdab5
:101680000135bfd16ff00104a3e70134002bb9d0bd
:101690008568099faf4265d905f1010ec0f808e0e1
:1016a0004fea051a03eb051e0025cee90166cef8c8
:1016b0000c50c5686f1c1fbf03eb0519d9f80c50ff
:1016c0000135c9f80c50b8f17b0f0cbf012502257c
:1016d00003f80a504568cef804508568013d1ce0c7
:1016e000d8f8047001371ad0d8f808a0baf1ff3f33
:1016f00015d198f800b0cb45c4d10ef1010ec0f859
:101700000ca0c8f808e003eb051edef804700137f2
:1017100009d0def80870013705d1c56072e7013dd8
:10172000a8f11008aae7013d6f1caef1100eecd134
:1017300068e70ef10109c0f80490d0f80480424532
:1017400002d911f8085025b9c0f804e06ff002047e
:101750003fe7222d2dd1e3b18568099faf4204d820
:10176000c0f804e04ff0ff3433e700274ff0030ade
:1017700005f1010e4fea051803eb0515c0f808e066
:10178000c5e90166ef60d0f804e003f808a0c5e9f8
:10179000019ec56801346f1c3ff434af002b3ff449
:1017a00031af03eb051edef80c500135cef80c50be
:1017b00028e75c2d11d108f1010595420dd2456055
:1017c0004d5d752d2cd86d2d0bd8662d28d85b2d31
:1017d0001ed8222d01d02f2d22d14568013545601c
:1017e000abe76e3d072d1bd801a757f825f000bfca
:1017f0005b170002a1170002a1170002a117000247
:101800005b170002a11700025b170002a717000276
:1018100040f241475c3dedb20cfa05f53d42dcd1aa
:10182000c0f804e02ee74ff0040a08f10205456015
:10183000d0f80480424512d911f808507db1a5f1c5
:10184000300bbbf1090f04d925f02005413d052dd2
:10185000e6d808f10105baf1010a4560e8d145680a
:10186000013d4560b9e7002b3ff4ccaec5682d01c2
:101870005d5d013d012d7ff6c5ae856805f1ff3840
:1018800003eb051eb8f1000ffff6bcae1ef8105cae
:10189000013d012d0cd85ef80c5c013508d05ef8d6
:1018a000085c013504d1c0f80c80abe61300800061
:1018b00008f1ff38aef1100ee4e7a5f120091f4f43
:1018c0005ffa89f90cfa09f919ea070f7ff4b5ae46
:1018d000203d5e2da4d808f1010545609ae60d2d46
:1018e000f6d1aae605f0df09b9f15d0ff8e78568e2
:1018f000099faf427ff634af002705f101084fea98
:10190000051903eb0515c0f80880c5e90166ef600d
:10191000d0f8048003f80970c5e901e84568013d85
:1019200090e653f80c2c013204d053f8082c013205
:101930003ff40caf0139103b48e600bf0110000432
:101940000023c0e901334ff0ff33c36070476ff0ed
:10195000770070476ff0770070476ff0770070473f
:101960006ff0770070476ff0770070470020704786
:101970000020704738f05ebb38f038bb38b50d46f4
:10198000002104460171816038220c30c3f021fb34
:1019900025b90a20074a0849fff72afb2846c4f060
:1019a00001fc206020b90a20024a0449fff720fb0d
:1019b000204638bd23a80202a8b50d02c9b50d0204
:1019c00010b50446006808b1c3f0b6fa204610bd51
:1019d00010b58368044623b90a20034a0349fff778
:1019e00007fba068403010bd23a80202ebb50d0232
:1019f00038b5044685682846fff7beff237963b1f2
:101a00002046fff7e5ff04f10c015ff0b6f904464c
:101a10002846fff7afff204638bd6ff0d104f7e747
:101a200070b5054686683046fff7a6ff2c794cb1a5
:101a3000002328462b71fff7cbff05f10c0160f066
:101a40005df804463046fff795ff204670bd2de94e
:101a5000f0430c7807460e46c3b0acb30846fff718
:101a600009fa2f2c804601d101282cd02f21701c7f
:101a7000c4f075fb002405464ff02f0925b3ab1bbe
:101a8000434521d804bb2c703846fff7a1ff6a46b6
:101a900031465ff07bf9041e0eda3846fff798fff7
:101aa000314660f0d1f9044628462f2100f8019b09
:101ab000c4f055fb0546e1e79df80030222b18bf26
:101ac0006ff0d104f0e70024204643b0bde8f08376
:101ad00037b50d4604460192fff77aff2a46019b6f
:101ae00004f10c0103b0bde830405ff05ebd37b5d6
:101af0000d4604460192fff76bff2a46019b04f155
:101b00000c0103b0bde830405ff0ebbc38b50446d3
:101b10000d46fff76dff002802db0f2801dc0948a6
:101b200038bda0f1100100222046fff7d1ff0028a8
:101b3000f5db102229462046fff7d9ff1028eed109
:101b40000020ede7e8feffff1fb50446002110224c
:101b50006846c3f03efa69462046fff7d7ff28b92a
:101b6000034a0399034b914218bf184604b010bdb5
:101b7000e5114f71e8feffff2de9ff41054687683b
:101b80003846fff7f9fe95f80480b8f1000f07d04a
:101b900000243846fff7eefe204604b0bde8f08191
:101ba0002e462846fff714ff56f80c2b40f203137d
:101bb000314660f047fa04460028ead10123014685
:101bc000102268462b71c3f004fa2846fff7bcffc9
:101bd0000028ddd0154b284603930194fff7f8fe4b
:101be000224631465ff0fafc041e16db42464146af
:101bf0002846fff76dff041e0fdb2846fff7e8febf
:101c000010236a4631465ff0b1fa041e05db284610
:101c100000f04cf804460028bad02846fff7d8fe5a
:101c200031465ff06bff00232b71b2e7e5114f7176
:101c3000f8b50646002038f0a3fa054620b90a2078
:101c4000174a1849fff7d4f92846fff795fe2846aa
:101c5000b56038f011fa20b10a20114a1249fff795
:101c6000c7f937682f213846c5f049f8044640b90e
:101c70003046fff781ff04462846fff77bfe2046eb
:101c8000f8bd8742f4d00023037031683046fff777
:101c9000defe2f23237004460028e9d0ece700bfc6
:101ca00023a8020200b60d0214b60d0270b5044658
:101cb00086683046fff760fe23799bb12046fff728
:101cc00087fe04f10c015ff0d1fe054628b12046e5
:101cd000fff7a6fe2046fff74fff3046fff74afe0c
:101ce000284670bd6ff0d105f7e737b50d460446bd
:101cf0000192fff76dfe2a46019b04f10c015ff093
:101d000035fa051e09da2046fff7d0ff28b1204634
:101d1000fff786fe2046fff72fff284603b030bdb1
:101d20002de9f0430646856887b028461f46894658
:101d30009046fff721fe3379002b40d0304602a9b0
:101d4000fff7e4fe041e33db039c002c30db21464e
:101d500000223046fff7bcfe041e29db0023adf84d
:101d6000063044f6ad63082269463046adf80030cf
:101d7000adf80290adf80470fff7b7ff041e17db53
:101d80003a4641463046fff7b0ff041e10db0d4bcc
:101d900010220593039b304608331f4402a9039782
:101da000fff7a3ff041e03db3046fff77fff044667
:101db0002846fff7dffd204607b0bde8f0836ff04f
:101dc000d104f5e7e5114f712de9f04f89b001918c
:101dd00004a9814617469846fff798fe0446002856
:101de00043d14ff0ff34054682462646059905f15a
:101df00008028a42ab4617d8002229464846fff718
:101e000067fe002835db082248460deb0201fff78c
:101e10006efe07282fdd44f6ad62bdf80810914232
:101e20000cd00235002de1da002f1ada01361ad073
:101e3000b8f1000f19d0a8f800a016e0bdf80a10fc
:101e4000019bbdf80c20994208d10136b742924659
:101e500006d908322c4602eb0b05e3e72546f8e7e6
:101e60002c46b742e4d06ff0a904204609b0bde883
:101e7000f08f0446f9e7014cf7e700bfe8feffffeb
:101e80002de9ff410546d0f808801c46404616461d
:101e90000191fff771fd2b7923b3019906b924bb9a
:101ea00028460a9a0df10e03fff78eff011e1edb76
:101eb000bdf80e70a74228bf2746c7b100222846aa
:101ec0000831fff705fe041e05db3a463146284679
:101ed000fff70dfe04464046fff74cfd204604b0d8
:101ee000bde8f0816ff0d104f5e7024cf3e76ff045
:101ef000a904f0e7f2feffff2de9f04f0446d0f809
:101f0000089097b048460f461646fff735fd94f8ff
:101f100004a0baf1000f00f08c804ff00008c34617
:101f20003246394620460df10e03adf80eb0fff7ec
:101f30004bff051e0cda002e03dab8f1000f18bfb4
:101f400000254846fff716fd284617b0bde8f08f7c
:101f50002046fff74dfd04a980462046fff7d6fd39
:101f60000246002863d12046fff732fd2268012394
:101f700008a960f067f80246002858d1bdf80e3075
:101f8000294620460193fff7a3fd021e4fdb019b6c
:101f9000204608331d44fff71bfd2a46002308a9ed
:101fa0005ff003fb021e42db0599a94215d9aab3d3
:101fb0002046fff70dfd0df10d02012308a95ff08a
:101fc00090fa021e2adb012220460df10d01fff7d7
:101fd0008cfe021e22db0135e6e7fab16ff0070541
:101fe0001022bdf80e302046eb1a0b440deb020117
:101ff0000593fff77afe021e19db2046fff7e8fc87
:10200000bdf80e2004f10c01aa1a42445ff0e6fa72
:10201000021e0cdb2046fff749fe024620460192d5
:10202000fff7d6fc08a95ff069fd019a22b11546b9
:1020300087e76ff0d10584e7002ef8dad0466fe726
:102040002de9f3410546d0f808801f464046164664
:102050000191fff791fc2b79bbb101992846089ab1
:10206000fff74aff0199044610b110f1aa0f05d1fc
:102070003b4632462846fff753fe04464046fff7ec
:1020800079fc204602b0bde8f0816ff0d104f5e79d
:102090000148fff795bc00bfb8cc001010b504464e
:1020a0000249fff76bfc204610bd00bf3cb60d0295
:1020b00010b50b4cd4e88f3fdb070cd4204629f039
:1020c0001dfe40b10748fff7e9ff204629f050fe0a
:1020d0000548c2f030fd0348fff7aafd014810bdd6
:1020e000b4cc0010b8cc00101120000213b50024ad
:1020f0009bb20094fff7c4fe02b010bdb3f5803f61
:1021000013b506d200249bb20094fff799ff02b0ea
:1021100010bd6ff0bd00fae72de9f34180460c4693
:1021200000262bf0a8fb37460546d8f8003040467d
:102130009b699847002834db18d0d8f8003001227a
:1021400040461b698df807700df10701984700287c
:1021500027dbd8f80030012140465b69984700280a
:102160001fdb0136e1e700241d46dee7c4b1d8f8e5
:102170000030224653f8140c012158f80030404436
:102180009b68984710f1a00f0ad0002809db2bf0bc
:1021900072fb431b9c42e6d92c440346241ae3e716
:1021a000304602b0bde8f0812de9f0418046c2b072
:1021b00000200d46174637f0e3ff044618b34ff4ee
:1021c0008472002168464034c2f003ff6a46294603
:1021d00020465ef0dbfd50b32f212846c4f08ffd72
:1021e000b8b1854215d0411b2846c4f059fd0646ba
:1021f000c8b1014620465ff027fe38b1113005d046
:102200003046c2f099fe6ff0e0000de03046c2f0bb
:1022100093fe47f480773b462a46414620465ff0ce
:1022200011ff08b1efe7044842b0bde8f0819df826
:102230000030112befd0e6e7fcfefffff8b50746b4
:1022400000200d461646fff71ff90446a0b10022f4
:102250003946fff763f928b132462946204641f056
:102260007ef838b96ff0e00500212046fff710f93d
:102270002846f8bd0025f7e7004df9e7fcfeffff13
:10228000f8b5074600200d461646fff7f3f804465a
:10229000a0b100223946fff727f928b13246294676
:1022a000204640f0dafa38b96ff0e0050021204608
:1022b000fff7e4f82846f8bd0025f7e7004df9e7f9
:1022c000fcfeffff0fb413b50a4b586e32f007f84f
:1022d00058b1094c05ab80212046049a0193c5f002
:1022e000d3f80028bcbf0023237002b0bde8104023
:1022f00004b0704778ce0010fccc001008b5044b39
:10230000586e31f0ecff10b10022024b1a7008bd7c
:1023100078ce0010fccc0010021e80f2ab81a74bdf
:102320009a4200f0a98101339a4280f2a88012f506
:10233000c86f6bdc6ff494710b449a4246da12f565
:10234000e16f00f09b8102f5d6620c2a4dd99c48c2
:102350007047c9320b2afad801a353f822f000bf04
:102360000925000205250002cf220002cf2200022b
:10237000cf220002cf220002cf220002cf22000291
:10238000cf220002cf220002012500020126000216
:10239000e6320b2adbd801a353f822f019250002fc
:1023a000cf220002cf220002cf220002cf22000261
:1023b00015250002cf220002cf220002cf22000208
:1023c000112500020d2500020526000202f24562d9
:1023d000052a00f2eb80dfe812f0e700e500e300f9
:1023e000e10057010600774870470c2aafd8dfe8b4
:1023f00012f03f013d013b01390137013501330145
:1024000031012f01e300e100df004d016e4b9a42e4
:1024100000f03e8101339a421cda1e3b9a4200f0e2
:10242000398101339a420ada12f5af6f00f0348134
:102430006649634b66488a4218bf18467047654b29
:102440009a4200f02b815e48634b12f5aa6f08bfd9
:102450001846704761498a4200f0228101318a4260
:1024600006da9a4200f01e81554b5d480a39e2e7d0
:1024700000f01a8152485b4b12f5a56fe7e712f1a5
:10248000da0f40da12f1e60f82da12f5967f00f0e9
:102490000d811bdc544b9a4200f00a8101339a42b1
:1024a0000bda4f3b9a4200f0058112f5966f00f06f
:1024b00003814e49424b4e48bde74e4b9a4200f0d5
:1024c000fd803f484c4b12f57a7fc0e712f5827fc2
:1024d00000f0f6800cdc12f58c7f00f0f38012f532
:1024e000877f00f0f1803648444b12f5917faee7cc
:1024f00012f1fa0f00f0ea80314b414812f1f00f6f
:1025000018bf1846704712f1aa0f00f0e18012f1cf
:10251000a90f14da12f1bd0f0ada12f1c90fbff6d2
:1025200018af274b374812f1d20f18bf1846704723
:10253000234b354812f1b40f18bf1846704712f1fb
:10254000820f00f0c78012f1810f0eda12f1960fa0
:1025500000f0c28012f18c0f00f0c080184b2b48a5
:1025600012f1a00f18bf1846704712f1780f00f053
:10257000b780134b264812f16e0f18bf18467047ec
:1025800024487047244870472448704724487047bf
:1025900024487047244870472448704724487047af
:1025a000244870472448704724487047244870479f
:1025b000244870472448704724487047e2faffffd8
:1025c00067b60d02ecba0d02b9faffff92faffffef
:1025d0006eb80d02a6faffffc7b80d02cdfaffffd5
:1025e000dfb80d027bb90d0294fbffffecfaffff91
:1025f00060b90d02b4fbffffd1b90d02dcb90d02c9
:1026000080ba0d0272ba0d02c1ba0d024bb60d02ac
:10261000f5ba0d0253ba0d0244ba0d0236ba0d02d4
:1026200023ba0d0211ba0d0206ba0d02f8b90d0255
:1026300001b80d02efb70d02ddb70d02cbb70d02e9
:10264000b4b70d0287b70d026cb70d024fb70d027c
:1026500024487047244870472448704724487047ee
:1026600024487047244870472448704724487047de
:1026700024487047244870472448704724487047ce
:1026800024487047244870472448704724487047be
:1026900024487047244870472448704724487047ae
:1026a000244870472448704724487047244870479e
:1026b000244870472448704724487047244870478e
:1026c000244870472448704724487047244870477e
:1026d000244870472448704724487047244870476e
:1026e0002448704740b70d0230b70d0210b70d02f5
:1026f000f8b60d02e5b60d02d8b60d02bfb60d0252
:10270000adb60d0288b60d02c3c30e0275b60d023a
:10271000d0ba0d0263ba0d021dba0d021cb80d022b
:10272000a2b70d025ab80d022fb80d024db80d0216
:1027300084b80d029ab80d02b0b80d02feb80d02b1
:1027400055b90d022fb90d0239b90d021cb90d0290
:1027500071b90d02a5b90d02bdb90d0294b90d02f2
:10276000e9b90d022cba0d02a3ba0d02afba0d02df
:102770008fba0d0259b60d0210b5084b0446586ebb
:1027800031f0adfd10b1064803782bb92046bde805
:1027900010400021fff7c0bd10bd00bf78ce001073
:1027a000fccc0010a0f13003dab2092a01d8184697
:1027b0007047a0f16103052b01d857387047a0f18d
:1027c0004103052b94bf37384ff0ff307047102a74
:1027d000f8b506460c461bd900252078fff7e2ff26
:1027e000071e15db6078fff7ddff031e10db43eaf1
:1027f0000713052d735505d102340135062decd193
:10280000012006e0a278e31c3a2a01d11c46f4e735
:102810000020f8bd034b1860034b1960034b1a608e
:10282000704700bf7ccd001080cd001084cd00101b
:10283000f0b5164b05461e680f461446abb036b9c8
:10284000134b1b6803b3134b1b7883421cdc2379a7
:102850001b0706d42bf00ff82379606143f00803bf
:1028600023718eb1dde93023a02102a8c4f00cfe53
:102870009f28c4bf7e238df8a63000233a460093dc
:102880002946234602a8b0472bb0f0bd7ccd0010ee
:10289000a8cc00103b51001030b585b008ac54f8fe
:1028a000045bcde900540394fff7c2ff05b030bdcf
:1028b00070b404460d46104619464bb1054b1e68d0
:1028c00036b1002322460393b4462b4670bc6047c2
:1028d00070bc704780cd001070b51a46134b04468b
:1028e0001d680e46aab035b9114b1b68bbb1114b20
:1028f0001b78834213dc2e9ba02102a8c4f0c4fde8
:102900009f28c8bf7e230146c4bf8df8a6309f21f3
:102910003db100232246009302a83346a8472ab0bf
:1029200070bd034b02a81b689847f8e780cd0010e4
:10293000a8cc00103b51001008b410b585b007ac0e
:1029400054f8043b00940394fff7c6ff05b0bde8bc
:10295000104001b0704700002de9f04f884629492a
:1029600007460d68adb0002b3ad035b92649096845
:10297000b1b326490978814232dc00211446dff8e0
:102980009090dff884b08df8ac10d61814f8013ba5
:102990002ca84fea131c19f80cc0084403f00f03cd
:1029a0004a1c00f8a4cc19f8033002312ca80244c8
:1029b000a02902f8a43c09d1adb14ff0000a43466a
:1029c0003a46cdf800a003a8a8475146a642ddd15b
:1029d00031b175b100233a46009303a84346a84796
:1029e0002db0bde8f08fdbf8003003a898472946ea
:1029f000ece72cab1944044b01f8a45c1b6803a85a
:102a00009847ede780cd0010a8cc00103b51001096
:102a100038bb0d02074b02461b680bb1002218475a
:102a2000054b186828b1054b1b789a42b4bf0020ab
:102a30000120704784cd0010a8cc00103b5100103d
:102a40004528dabf0a2390fbf3f00620034bd8bfda
:102a500020eae07053f82000704700bf1cbb0d0255
:102a600070b50d46044620b90a201c4a1c49fef7e1
:102a7000bffa1cf0dbfba37bdb070bd563680bb154
:102a8000a2689a60d4e9013282b15360a37b03f05b
:102a9000fe03a37313490b686db1002283b11e7b43
:102aa000257bae420bd91a465b68f7e70d4a1360e7
:102ab000ece70c6007e063b901238b7409e09c60cc
:102ac000002af6d05460c4e90132a37b43f001032d
:102ad000a373bde870401cf0adbb00bf23a8020289
:102ae00049bb0d0288cd001010b504461cf09efbba
:102af000094b1a8a5cb1013a92b21a821a8a92b2ce
:102b00000ab901229a74bde810401cf093bb01324f
:102b100092b21a82f7e700bf88cd001010b51cf002
:102b200085fb044b1c8a1cf085fba4b2b4fa84f02c
:102b3000400910bd88cd00102de9f04f85b04ff051
:102b4000000905461cf072fbca4683464b4601202d
:102b500049464f464e464a46614cd4f8008010b371
:102b6000b8f1000f1fd098f80d300f2b5ffa83fae1
:102b700015d1d8e90531284698470022d8f81060c9
:102b800098f80e10238a94f812909bb2b3fa83f34c
:102b90000020c9b25b095ffa89f9a274dde7b8f8d1
:102ba0001470bfb2eae75846cde902131cf042fbad
:102bb000dde90213a27a524502d1a289ba4261d05c
:102bc000002284f80aa0a781e281002b57d011f0df
:102bd000020067d1434bc6f307481f78424bffb250
:102be000db6898477843f5b2c6f3072700fb08f87f
:102bf00047434543b4f80cc04fea18413a0c280c3f
:102c0000884617460546bcf1000f05d0a67ae38931
:102c1000022e44d0032e49d0b9f1000f08d1a38869
:102c2000434505d1e388bb4202d12389ab4226d07c
:102c3000dff8b4900023d9f804602a4639464046ac
:102c4000b0472a4e3368b3b1d9f80c30002098470a
:102c50004fea08212b023a02b3fbf0f3b2fbf0f289
:102c6000b1fbf0f000210091c1b221483668006844
:102c7000dbb2d2b2b047a4f80480e780258105b06a
:102c8000bde8f08f002fa0d0e0890544adb2bd4271
:102c900024bfb5fbf7f207fb1255e58195e7b3ebcf
:102ca0005c0fb9d300252f46a846b5e74fea5c066e
:102cb000b3eb5c0f34bff31a9b1b9bb203fb01f811
:102cc00003fb02f703fb00f5b8fbf6f8b7fbf6f7da
:102cd000b5fbf6f51ffa88f8bfb2adb29ce700bfae
:102ce00088cd00103a510010205100109ccc0010eb
:102cf000a0cc0010064b0022194641f8042b5a6064
:102d00001a828a805a81da6001229a74704700bf61
:102d100088cd001070b5d0e90043204643f31d0371
:102d2000002b0ddd5a1050f8226000eb8205b688aa
:102d30008e4203d29b1a281d013bf1e71346efe7b1
:102d4000001b801070bd000070b51048d0e88f5f88
:102d500015f001050e4e16d128f0d0ff98b11020c5
:102d600026f0d6fd044650b1c0e9005585600573d4
:102d70008020c2f0d9f810b120232060a36003485e
:102d8000346028f0f5ff306870bd00bf9ccd0010a6
:102d9000a0cd0010f8b50746fff7d6ff037b044629
:102da00073bbb988fff7b6ff0546d4e90006b54204
:102db00004da50f825309b888b4224d0a3689e42c9
:102dc0000ddb0136002e05ddb100c3f083f820b91c
:102dd0000e4814e0c2f0b0f800202060a66026681b
:102de000626806eb85019200a2eb8502081dc2f025
:102df000d6f8002046f82570636801336360f8bd9b
:102e00006ff0d100fbe76ff0b300f8e7fcfeffffc7
:102e10002de9f84307460e469046fff795ff037be2
:102e20000546a3b177b1d0e9004304eb83094c45d3
:102e3000234607d0414618680434b8470028f6d026
:102e4000bde8f88336b16b6800203360f8e76ff0b7
:102e5000d100f5e73046f3e770b506460c46fff7bc
:102e600073ff037b05467bb13146fff753ff6b6869
:102e700098420cda2b6853f820309a88b24206d177
:102e800044b10020236070bd6ff0d100fbe76ff00c
:102e9000a900f8e72046f6e710b50446fff754ff0f
:102ea000022c05bf012303736ff07700002010bdd3
:102eb00038b538220d4600210446c2f08af84ff09a
:102ec000ff3200232046c4e90f23a56338bd00006c
:102ed00030b505468db0002037f052f9044618b3de
:102ee00037f084f82b6c990706d40025204637f07c
:102ef000a1f828460db030bd294604f140005ef02f
:102f0000b5fd0028f1da202200230290cde9042348
:102f1000aa6b32200192064a0649009204aafff7e2
:102f2000bbfc6ff0e005e1e76ff0e005e1e700bf13
:102f300069bb0d0261bb0d02002370b501f14006b3
:102f4000044601461a4630468eb05ef02efb00283d
:102f50004ff0000511da2023cde90635a36b02906e
:102f600001930f4b322000930e492b4606aafff720
:102f700093fc6ff0e0000eb070bd04232146304694
:102f800005aa05955ef0adfa042807d02023cde907
:102f90000635a36b02900193034be3e70598eae73c
:102fa00088bb0d0261bb0d02a7bb0d0210b5044624
:102fb000236c08468cb0abb1214640305ef09efddc
:102fc00000280dda20220023cde90423a26b029011
:102fd0000192054a32200092044904aafff75cfce2
:102fe000002323640cb010bdc6bb0d0261bb0d02f3
:102ff00038b50546002037f0c3f8044650b136f026
:10300000f5ff28462146fff7d1ff2046bde83840ae
:1030100037f010b838bd000030b505468db000203f
:1030200037f0aef8044610b336f0e0ff21462846ec
:10303000fff7bcffa96b04f140005ff00bf800281c
:103040000fda811c0dd020220023cde90423aa6bc6
:1030500002900192074a32200092074904aafff722
:103060001bfc20460db0bde8304036f0e3bf0db08c
:1030700030bd00bfe6bb0d0261bb0d02002a70b57a
:1030800040f6031518bf0125036c044635ea030317
:103090000e468cb01fd0fff789ff2b462146a26b4e
:1030a00006f140005ef0ceff002813da811c14d038
:1030b00020220023cde90423a26b02900192084a4a
:1030c00032200092074904aafff7e6fb6ff0e00008
:1030d0000cb070bd25640020fae76ff0a900f7e797
:1030e00002bc0d0261bb0d022de9f04705468cb014
:1030f00000208946904637f043f80746002863d001
:1031000036f074ff012239462846fff7b7ff041e48
:103110001bdb07f1400a294650465df02efe061ed5
:1031200010da20200023aa6bcde904030192284a7b
:10313000029600923220274904aafff7adfb6ff0f8
:10314000e00402e0032e07dc234c384636f072ff21
:1031500020460cb0bde8f087eb6b002b09da39464e
:103160002846fff7e9fe041eefdb17d1042eebd152
:10317000ec63ea6b00239045a8bf90462946504671
:10318000b21a5ef012fa00280cda20210023aa6b92
:10319000cde9041301920290104acae7f31ea3423c
:1031a000e6dcd1e743464a46294650465ef099f9a7
:1031b00080450446c9d020220023cde90423aa6b10
:1031c00002900192064ab4e76ff0e004c0e700bf46
:1031d00021bc0d0261bb0d02e8feffff88bb0d02a2
:1031e000a7bb0d022de9f04705468eb000208946a9
:1031f000164636f0c5ff804600287fd036f0f6fe32
:10320000002241462846fff739ff041e18db08f16b
:10321000400a294650465df0b0fd071e17da4ff010
:10322000200c0023aa6bcde906c30192354a029710
:1032300000923220344906aafff72efb6ff0e0041b
:10324000404636f0f7fe20460eb0bde8f087032f6b
:103250000fdc0022294650465ef0c0f9002828da2b
:1032600020260023aa6bcde9066301920290274a2b
:10327000dee7eb6b002b06da41462846fff75cfee3
:10328000041edddbec63eb6bb342e2d13744b7f5f0
:10329000805fdedc33464a46294650465df066ffd5
:1032a00086420446ccd0202200230290cde906239a
:1032b0001ee0002329461a4650465ef076f90028a3
:1032c00008da20240023aa6bcde90643019202907c
:1032d0000f4aade704232946504605aa05965df03e
:1032e00045ff042808d020210023cde906130290d1
:1032f000aa6b0192074a9be7ee63cbe76ff0e0040d
:10330000a1e700bf21bc0d0261bb0d0240bc0d0254
:1033100088bb0d0263bc0d0210b401291346c068be
:1033200008d102685968146803f1080223465df861
:10333000044b18476ff077005df8044b704738b5c1
:10334000144619b904220846226038bd1368032bbd
:1033500007d903685b6898470028f6d104232360e7
:10336000f3e76ff0bd00f0e7836900200b60704762
:10337000836900200b60704713b5114b0c461b7e10
:10338000062b1ad0cbb10121684613f08dfc68469c
:1033900013f04dfc684613f007fedfed0a7a20eecd
:1033a000270abceec00a10ee103a9bb268462360b2
:1033b00013f08afc002002b010bd6ff0d100fae7d4
:1033c000bccd0010000080430a4b10b503601423ed
:1033d0004360012304464381074bc0e90320018178
:1033e000436100210430fff7d5fc044b20462360e5
:1033f00010bd00bfa8bc0d0299320002b4bc0d0282
:1034000010b50446fff7e0ff014b2046236010bdd6
:10341000e4bc0d0208b500f085fcbde8084000f0f2
:1034200097bc07b5019000f07dfc019903b05df8f1
:1034300004eb00f0b5be08b500f074fcbde8084030
:1034400000f0bfbc07b5019000f06cfc019903b01f
:103450005df804eb00f05ebd07b5019000f062fc82
:10346000019903b05df804eb00f06abd38b50025a2
:103470000b4c03210b4a0c48fff7c2ff07212046e3
:103480000a4afff7a1ff0a4ba5612360094c1821e6
:103490002046094afff798ff084ba561236038bd15
:1034a000bccd001083bc0d02a4cd00108cbc0d025d
:1034b000c4bc0d02d8cd001097bc0d02d4bc0d02c7
:1034c000074b1a7812b10021064a11705a7812b1ce
:1034d0000121054a11709b780bb10bf0fdbc7047c0
:1034e000f4cd00102ed200102cd20010fff7e8bf50
:1034f00010b5c36804460bb9c0f0c4ff03690430bb
:1035000098470021a0616069bde8104031f03ab8e9
:1035100010b50bf009fd124b124c1b780246b3faa2
:1035200083f35b09a070237080b101200022052184
:103530006070104604f068ff0bf0f0fcbde810402e
:1035400000231a461946184604f0fabf014604f053
:103550000ffe02460028e8d1014604f058fee5e7d8
:103560002ed20010f4cd0010012af8b5064603d182
:103570000b6803600020f8bd022a08d0032af9d1a5
:1035800000680028f6d01c2126f0caf9f2e71c20ba
:103590000c6826f0bdf9074630b105460fcc0fc5c3
:1035a00094e8070085e807003760e3e7012a70b573
:1035b000054603d10b680360002070bd022a08d0c5
:1035c000032af9d100680028f6d0102126f0a8f9c6
:1035d000f2e710200e6826f09bf9044618b196e831
:1035e0000f0084e80f002c60e6e721b18b8883424e
:1035f00001d08968f9e7084670470000f8b5037df7
:1036000005460f46164653b10368d9680120fff7f7
:10361000ecff044630b18389bb4201d18673f8bd0b
:103620008168f3e7014610200ef04efc08b92c75b6
:10363000f5e7054b0360012383802b698781836055
:1036400086732861ebe700bf1000030008b5c1686e
:103650000120fff7caff28b183891b2b01d08168a5
:10366000f6e7012008bd000038b5037d04460d468d
:103670003bb103680420d968fff7b7ff014608b1e2
:10368000c56038bd10200ef01ffc08b92075f8e7a2
:10369000044b0360042383802369c0e90235206161
:1036a000efe700bf1000030010b58368044613b1b4
:1036b000032201469847204610bd000010b504467d
:1036c000034b40f8043bfff7efff204610bd00bf5f
:1036d000f4bc0d0210b50446fff7f0ff204614219c
:1036e00026f01ef9204610bd10b5074b04460360b6
:1036f000406918b130f021ff002363612046fff7d5
:10370000ddff204610bd00bf08bd0d0210b5044608
:10371000fff7eaff2046182126f002f9204610bde7
:1037200010b50446024b0360fff7deff204610bdd4
:103730001cbd0d0210b50446fff7f2ff20461c2108
:1037400026f0eef8204610bd38b50446006928b1d1
:10375000856800210ef0e2fb2846f8e7204638bdd8
:10376000002330b587b0cde90233049301238df8ef
:1037700014301023adf80430032301ac00280d46ab
:103780000094adf806308df8083005dd4ff47a71fd
:1037900041436846fff768ffab0704d401220a21c2
:1037a0006846fff72bff2046fff750ff80f001002f
:1037b000c0b2fff736fe00222046114625f08ffcee
:1037c00004466846fff7c0ff204607b030bd000042
:1037d0002de9f0470e4698461021002388b0cde928
:1037e00004330693adf80c10012303211746109af9
:1037f0000df10c09002a0546cdf808908df81c3013
:10380000adf80e108df8103005dd4ff47a7102a876
:103810005143fff729ffb5b1beb1002f41d0b8f138
:10382000000f3ed0002407eb080ab4420dd04445f7
:1038300035f8141034bf3a5d1af8012c02a8fff7ce
:10384000ddfe0134f1e72c46ede74846fff7fefeca
:10385000002780f00100c0b2fff7e3fd3a4648467a
:1038600001a9019725f03bfc041e11dbfff7e3fde6
:103870000198c0b183883c46012b07d1b4420ed0d9
:1038800035f81430828901349a42f7d1c1f054fbe3
:1038900002a8fff759ff204608b0bde8f0870024d2
:1038a000f4e7024cf4e70446f2e700bff2feffff44
:1038b00073b506461c200d4626f02af8044628b3a8
:1038c000144b03600023c360ab683bb1022229465e
:1038d00004309847eb682361ab68e3600022204620
:1038e0000d4b0121236040f8142f30f01bfe0b4bd1
:1038f00030462360336801945b6801a99847054608
:1039000020b9236820469b6898472c46204602b081
:1039100070bd00bff4bc0d0208bd0d021cbd0d0240
:10392000f0b51f463c4b164693f86c2005460c46f6
:1039300089b0f2b1586e30f0d2fcd0b906901020a8
:1039400025f0e6ff18b1c0e901460570c760334baa
:1039500004900793324b304804a90693fff7a8ff61
:103960000546b8b9044604a8fff79efe204609b0f4
:10397000f0bd02f0f1fdc8b9f34313f0010300d12b
:1039800095bbfff7c5fd012d3ed0022d3cd0bdb14a
:103990000024ebe700224ff0ff31406930f0d2fd08
:1039a0002b6828469b68ac699847dce716f004034f
:1039b000e2d11a460621012000940ef011f8dbe74f
:1039c000002cd3d0e317cde9044301212b46154a3f
:1039d000009504a8cde906552af09af80446002877
:1039e000c4d0fff76dfdc1e7012d0dd0022dcfd161
:1039f0001a4618460521039304f006fd039b1a4658
:103a00001946184604f09cfd3146204609b0bde831
:103a1000f040fff7a5be00bf78ce0010a939000224
:103a20002d3500026d34000200684168d0e90223a0
:103a30000078fff775bf2de9f0411f4600230446cb
:103a40000d46164601211a46184604f0fefb3b4679
:103a5000324629462046bde8f041fff761bf00002d
:103a60002de9f04f9846554b174693f86c2087b0d8
:103a70000546dde910940e4622b3586e30f02ffc57
:103a800000bb04901c2025f043ff38b1129bc0e915
:103a90000056c0e90278c0e904948361484b029063
:103aa0000593484b454802a90493fff701ff0446dc
:103ab000002855d1054602a8fff7f6fd284607b0b5
:103ac000bde8f08f02f048fd8246002854d1e4435f
:103ad00014f001046dd0fff71bfd4ff0000a002128
:103ae0000846fff701f8e720fdf7d6fb43463a46c4
:103af00031462846cdf80090fff76afe00210546c2
:103b00000120fef7f1ffe720fdf7a2fb002c4dd1cd
:103b100020461ef0c6f80bf02dfa044600200bf0ec
:103b200035fa0646b8bb013ce4b2012c33d80bf0a1
:103b3000fbf980b3304629f091fe4ef6602604462c
:103b4000002029f08bfe001b61f10001b04271f1f1
:103b500000031ed202f000fdd8b902f00dfdefe720
:103b600000224ff0ff31406930f0ecfc2368204622
:103b70009b68a56998479ee714f0040ba7d15b46a4
:103b80005a4606210120cdf800900df029ffda46b3
:103b90009de702f0e1fcbaf1000f8fd007f0eefdd7
:103ba000002304211a4614f062fd87e7fff788fc22
:103bb000b1e720461ef072f891e700bf78ce001002
:103bc000493b0002e93400021fb500688369029393
:103bd0004369019303690093d0e90223d0e900010e
:103be000fff73eff05b05df804fb2de9f0471f46e7
:103bf000dde90889002304460d461646ddf828a0b5
:103c00001a460121184604f020fb3b46324629465d
:103c10002046cde9099acdf82080bde8f047fff7ae
:103c20001fbf70b51d46002388b00e461446adf880
:103c300016001a460121184604f007fb0c9b00945d
:103c4000cde9015301230df11f0219460df11600b4
:103c50008df81f60fff7c9ff08b070bd40f62873ec
:103c600084b0adf80c3040f6277341f2d832984258
:103c700088bf0df10603adf8060098bf03ab1988a5
:103c8000adf80e2091424ff0500288bf0df10e03a7
:103c90001b88a3f628739bb2adf80a30bdf80a3032
:103ca0009bb2b3fbf2f3adf80a30bdf80a309bb219
:103cb00003eb83031b019bb2adf80a30bdf80a3059
:103cc00003f628739bb2adf80a30bdf80a0080b243
:103cd00004b0704770b5002501260446202229460d
:103ce000c0e90055c0e90555c0e90755c0e90955c7
:103cf0000672c560067485853030c1f06af904210a
:103d00002b463246601830f057fb636823b90a200f
:103d1000024a0349fdf76cf9204670bd23a8020250
:103d200028bd0d0210b5084cd4e88f3fdb0709d43d
:103d3000204627f0e3ff28b10448fff7cbff2046d9
:103d400028f016f8014810bdf8cd0010fccd001089
:103d50001fb500234ff4c0620393cde90032084938
:103d6000084b092203a830f0a3fa039b23b90a20c9
:103d7000054a0649fdf73cf905b05df804fb00bfb4
:103d80004bbd0d02cd46000223a802024fbd0d021d
:103d900007b50122054b01a91a70002340681a4695
:103da000019330f014fb03b05df804fb3c510010ac
:103db00008b5fff7b7ffbde80840fff7e9bffff719
:103dc000f7bf07b5036843b102234ff0ff320193f9
:103dd0004068002301a930f0fafa03b05df804fb53
:103de000cb0744bf002380f829308a0741bf002356
:103df00080f82b3080f82d30c3614b0744bf00237f
:103e000080f82830002311f0080f1cbf036280f8ef
:103e10002c3080f82a30704737b504460d4601a88b
:103e2000012113f0bcfd236b01a85b0500d4bdb1db
:103e300013f071fe78b1ff212046fff7d1ff01a8f2
:103e400013f0d2ff01a814f0adf829f014fd606260
:103e50004ff47a73a36101a813f0c0fd03b030bd25
:103e600013f059fe0028f6d1ff212046fff7b8ffd6
:103e700001a813f09eff01a814f0abf8e8e707b51e
:103e8000002108462af0fbfe88b9014601902bf07c
:103e90002ff8019a1346114610462bf0f3f8019ab9
:103ea0001146104603b05df804eb2bf0b5b903b032
:103eb0005df804fb0023202210b504468ab0cde94a
:103ec0000223104a10490092282002aafef7e4fcbf
:103ed000236bd9050ad4012102a813f060fd01214a
:103ee00002a814f043f802a813f078fd1b2012f08a
:103ef00057fd0023054a9361054a936123600ab088
:103f000010bd00bf78bd0d026ebd0d02bccd00100e
:103f1000d8cd001037b50446084600213cf076fbaa
:103f20002368054643b101234ff0ff3201936068d7
:103f3000002301a930f04bfa284603b030bd000041
:103f400070b50c464e79204600213cf04bfb0546ef
:103f500038b92379ff2b04d06379013bdbb2fd2b09
:103f600007d9202e3246204628bf20221b49c1f007
:103f700009f84ff6fd72e3882846013b9bb2934255
:103f800088bf40f628734ff6fd7288bfe38023890f
:103f9000013b9bb2934288bf4ff461734ff6fd72b1
:103fa00088bf23816389013b9bb2934288bf4ff452
:103fb00060734ff6fd7288bf6381a389013b9bb29a
:103fc000934284bf41f21003a381a37b013bdbb288
:103fd000fd2b84bf1223a37370bd00bfb4bd0d02bf
:103fe00001462023303180f83530fff7a9bf0000ab
:103ff000f0b587b00446002101a813f0d0fc01a859
:1040000013f02efd02ad07462a46184bb4f838c00f
:1040100003f1100e2e4618685968083303c673451d
:104020003546f7d108206423194632f8023b9c45f7
:1040300002d30138f8d119468f4202d001a813f0fb
:104040005cfe01a813f03efd0546e08efff706fe7c
:10405000854206d0e08efff701fe014601a813f06d
:10406000c3fd01a813f0bafc07b0f0bdccae0d0241
:1040700013b50c4601a8002113f091fc01a813f020
:1040800021fd40f62871884202d001a813f0acfd52
:1040900014b101a813f0b5ff01a813f09ffc02b002
:1040a00010bd8009431e022b94bf013001207047d0
:1040b000f7b504460e4601a8012113f070fc01a8d3
:1040c00013f075fc01a813f03cffa18f01a813f0b9
:1040d000d5fe642101a813f070fd618f01a813f0d3
:1040e0009bfe4ff4807101a813f0fafe2b4b197e52
:1040f00011b18a1f514251412046fff78dfe01a8a0
:1041000013f01efd10b901a813f091ff01a813f0e0
:10411000cdfc054601a813f0ecfc28b901a813f06a
:1041200033fe002d18bf2e4601a813f0c5fc07462c
:1041300001a813f095fc64281fd93846fff7b1ff9a
:10414000012806d0226b12f4007318d0831e584247
:104150005841ceb105b9b8b929f08dfb054601a883
:1041600013f0a4fc68b129f086fb401bb0f57a7f00
:1041700007d2322026f093fbf1e70020e9e718464a
:10418000e7e701a813f03dffff212046fff728fed7
:1041900001a813f023fc03b0f0bd00bfbccd00109c
:1041a00037b5036804460d46abb10d4b1b7e062b9d
:1041b00002d10021fff77cff7db1237c6bb1002190
:1041c000684612f071fd684612f0a5fe00236846ad
:1041d000237412f079fd03b030bd01232374fae794
:1041e000bccd0010f0b587b0044615460f4629f047
:1041f00042fb42f210730026a361ab1f594260617b
:104200005941204684f82d60e661a662fff704fe5e
:10421000bd422dd1032d12d129f02dfb236ac01ae6
:1042200041f2873398421dd829f025fb94f82c30b1
:1042300020620133dbb2012b03d884f82c3007b0a5
:10424000f0bd314684f82c6004a813f0a8fb80214f
:1042500004a813f045fe4ff47a7304a8a36113f089
:10426000bdfbece729f007fb84f82c602062e6e751
:10427000062f0dd1314604a812f016fd04a812f045
:1042800041fe20460121fff713ff04a812f01cfd98
:10429000022d0ed0032d0fd0104b2a469d61002316
:1042a0004ff480300021cde90133009303f078f919
:1042b000c5e701232372efe729f0ddfa0021206230
:1042c00084f82c1004a813f06afb4ff4807104a842
:1042d00013f006fe04a813f081fbdde7bccd00104f
:1042e000012937b5054614461ad10b21fff778fd91
:1042f0002f4b1a7e012a39d01cb190f82840013486
:10430000e4b24ff47a72012c85f82840aa612dd9c5
:1043100001222846197e03b0bde83040fff762bf96
:10432000022914d10e21fff75bfd214b1a7e022ad0
:104330001cd01cb190f829400134e4b24ff47a72d9
:10434000012c85f82940aa6110d90222e1e703294e
:104350000cd10023038580f82a304ff47a738361ef
:1043600029f089fae8611cb985f82b4003b030bd0b
:1043700095f82b300133dbb2032b85f82b30f5d9c0
:1043800095f82d3013b10622094bc2e7012185f8bb
:104390002b3085f82d1001a813f001fb4ff4967116
:1043a00001a813f00afc01a813f018fbdee700bf18
:1043b000bccd001030b52ded028b002185b0044638
:1043c000fff72afd012102a812f06efc02a812f0ec
:1043d000bffc264db0ee408a297e91b9f7ee007af7
:1043e000b4eee70af1ee10fa4cbf06220122204695
:1043f000fff7f8fe02a812f067fc05b0bdec028bd7
:1044000030bd062912d1f7ee007ab4eee70af1eedc
:1044100010fa1ddd94f82a3013b94ff47a72a261b4
:104420000133dbb2012b84f82a30e3d9012101a842
:1044300013f0b5fa01a813f03ffb43070ad4042296
:10444000297e2046fff7cefe01a813f0c7fad1e778
:104450000a46cce7f7ee007ab4eee78af1ee10fafe
:10446000297e4cbf06220122ebe700bfbccd001025
:104470007fb52d4d0446012101a813f090fa2e7e40
:10448000062e28d101a813f046fb20bb29f0f3f932
:10449000636ac01ab0f5fa5f15d3012102a812f0c1
:1044a00003fc02a812f054fcf7ee007ab4eee70a1f
:1044b000f1ee10fa0cd520463246297efff792fe27
:1044c00002a812f001fc01a813f088fa04b070bd34
:1044d00002a812f0f9fb00212046fff79dfc01a87d
:1044e00013f0eafac0f30111032907d12b7e032b45
:1044f00015d001222046fff7f3fee4e70139012938
:1045000002d801220221f5e7430705d40422204600
:10451000297efff767fed6e701221146eae742f25d
:104520001073a361cfe700bfbccd001073b5294d58
:1045300004462b7e042b04d142f2107382699a4206
:1045400040d0e36993b929f096f96369c01aa36969
:10455000984237d329f08ff9236b60615b052046c1
:1045600032d502b0bde87040fff724bf29f083f9cf
:10457000e369c01ab0f57a7fe5d3012101a813f0f1
:104580000efa236b5a0510d401a813f0c4fa60b1d7
:1045900094f82d6003222046297efff723fe76b192
:1045a000642101a813f009fb09e0ff212046fff771
:1045b00017fc42f210730021a361fff72dfc01a844
:1045c00013f00cfa02b070bd02b0bde87040fff706
:1045d0004fbf00bfbccd00102de9f043584b04463f
:1045e0001a7889b0002a00f081800022012105a8f4
:1045f0001a7013f0d4f9012106a812f055fb05a892
:1046000013f05dfa8df8170005a813f058fa9df81d
:104610001730184302065ffa80f81fd501212046a3
:10462000fff746fd05a813f047fa10f0300f0546d6
:10463000444ec0f38007c0f3011915d005a813f04c
:104640006afa48b1b9f1030f07bf012249460022b7
:1046500002212046fff744fed7b14ee005a813f033
:1046600048fa0028dad0dde718f0080fc8f3c002d6
:1046700006d0354b05222046197efff7b3fdebe748
:10468000002f36d1304b04222046197efff7aafdb9
:104690002d4b1b7e042b0cbf05250025337eab4222
:1046a0000ad000232a464ff400300021cde901331f
:1046b0000093b56102f074ff06a812f098fb78b180
:1046c00006a812f002fc237a53b100234ff40040f5
:1046d0001a460021cde901332372009302f060fff6
:1046e00006a812f0f1fa05a813f078f909b0bde8b0
:1046f000f08301212046fff7f3fd05a8276b13f097
:10470000d5f901460028c3d12846fff7cafc032883
:10471000054610d004280ed0022801d1bb0504d5cf
:104720002046fff765fc0125b8e7b36913f0fd0fdc
:1047300014bf012100212046fff79afcaee700bf1d
:104740003c510010d8cd0010bccd00102de9f04137
:104750008eb0fff7e7fa044600202ff0befd206080
:104760002046fff73dfc256b15f4807514d000251d
:104770002023cde906354e4b4e49009306aa2b4621
:104780002820fef789f82046fff794fb28460eb054
:10479000bde8f0412ff0d7bd2046fff770fb0221a6
:1047a0000a2026f013ff0623cdf811508df81030a3
:1047b0009df8133004af43f004032a463e498df8b8
:1047c00013300a20022300972ef032ff02211b2013
:1047d00026f0fcfe4ff0ff33022238491b200095e3
:1047e00012f0b6f8012103a813f0d9f803a813f0ca
:1047f000def801212046fff75bfc03a813f05ff908
:1048000003a813f05cf9012106a812f04dfa06a8de
:1048100012f0a5fb236b5b0503d4142106a812f04c
:104820002ffb06a812f051fb42f2107306a8a361f9
:1048300012f04afa03a813f0d1f8dff884800023bd
:104840004ff47a72394660682ff0e2fd054658b998
:10485000049e012e0fd12046fff7c2fb29462046b9
:10486000fff726fc88f8006098f80030dbb9204696
:10487000fff75cfee3e7022ef6d101212046fff7a9
:1048800017fc237c7bb9012106a812f00dfa06a8bb
:1048900012f065fb01234ff4fa70237425f0ffff3b
:1048a00006a812f011fa2046fff796fedce700bfdb
:1048b00097bd0d026ebd0d023f3d0002313d00026d
:1048c0003c510010c1684a69506803681b6818476a
:1048d00038b50c461546c8683ab11146c1f0fafa27
:1048e00038b1e0600020256138bdc0f025fbe560ef
:1048f000f8e70148f8e700bffcfeffff10b591f8ac
:1049000043300c46db0748680cd500210df006fb50
:1049100094f8433023f0010384f843300023c4e9c2
:10492000013310bdc0f008fbf8e708b508b10af084
:10493000f5fa002301211a46184603f086fcbde86b
:10494000084000f093bf10b5c468a068c0f0ecfa4e
:1049500060601af06bfc94f842202ab963687bb15e
:10496000022384f8423014461af064fc6cb160688b
:10497000c0f0e2fa2046bde8104000210df0cebaaa
:10498000012284f842201c46eee710bd136810b5e2
:10499000032b17d90b685c1c0c6018700b685c1c2f
:1049a0000c60040a1c700b685c1c0c60040c1c700e
:1049b0000b68000e5c1c0c60187001201368043b2f
:1049c000136010bd0020fce773b58b6804460d46ec
:1049d00000931bb90026304602b070bdcb8800683a
:1049e000694601aa0193fff7d1ff06460028f1d0de
:1049f000019b012beed9009aa389511c00911370e1
:104a0000009a1b0a511c00911370019b2268023b03
:104a1000910701930ed5012bdcd9009ae389511c33
:104a200000911370009a1b0a511c00911370019b96
:104a3000023b019323685a070ed423681b0706d54f
:104a40006946606801aafff7a1ff0028c2d0aa68e2
:104a5000009b9b1aeb80bee76946a06801aafff79e
:104a600095ff0028e9d1b5e738b50c4b41600360ec
:104a70000023c0e90233036104461af0d7fb054660
:104a8000214607482df01aff214606482df022ff47
:104a900028461af0cffb204638bd00bfe4bd0d020a
:104aa0008f4e0002b14e00022de9ff41cb88064631
:104ab0003f2b0f4640f29380886860b1338a032b06
:104ac0000cd9002301220293cde900230323039391
:104ad0006846fff779ff04b0bde8f081002144206b
:104ae0000df0f2f9044638b90123cde90030042372
:104af000029003933946ebe718230380bb884ff0fd
:104b0000000843807b88c0e9038883606ff06303fb
:104b1000c0e90c8846614062c0f83880c363738a7c
:104b200001339bb273828568a0f8403080f84380df
:104b3000002d35d12b4b00f11801c3612a4804f038
:104b400055fa032384f8423063886560462b0ed003
:104b500010d8322b07d004d8283b012b03d90025cd
:104b600008e03c2bfbd10120fff7dffef7e72846ea
:104b7000fff7dbfe0023a362b368e36203b19c622c
:104b8000338ab460013333820023cde90133b4f8b2
:104b90004030adf80c50adf80e3003230093a9e778
:104ba000402d0fd8414628460df08ef9606048b17f
:104bb00094f8433043f0010384f84330022384f82f
:104bc0004230cce7094b0848e36104f1180104f0d6
:104bd0000dfa00230225636084f84230cae7002002
:104be00079e700bf454800024cf60010c7480002b4
:104bf00070b58b8884685cb1b4f840209a4209d0c3
:104c0000e46af8e7d8b9636833448b60012070bd6b
:104c10000020fce794f84230022bf9d1cd88a66b36
:104c2000a36872199a42f3d8402d8868ead8002800
:104c3000edd0636801462a469819c0f0a3f9a26b2b
:104c4000a36815449d42a563e0d1064b0648e36185
:104c500004f1180104f0caf90023a363032384f8c4
:104c60004230d3e7454800024cf60010f8b506463e
:104c70008b8884684cb1b4f840209a4207d0e46a2b
:104c8000f8e7e3683b448b6016e0002019e094f8f5
:104c90004230042bf9d1cd88002df6d0a76b2369c3
:104ca0007a199a42f1d8402debd8886848b1e1686a
:104cb0002a463944c0f066f9a06b2844a06301205d
:104cc000f460f8bdf0b54b780c46502b85b00cd194
:104cd00091f90030002b41dacb8833b1886888b372
:104ce0008a88142a03d01e2a2ed000202ae0102100
:104cf000684624f053fa1028f7d8e3884500b3eb50
:104d0000400ff2d36b46a2685619b24218d01f4624
:104d100019780232090901f13000392888bf01f100
:104d2000370002f8020c3978013301f00f0101f16c
:104d30003000392888bf01f1370002f8010ce4e7a0
:104d4000e580012005b0f0bd042bced90b4b1a68cd
:104d50001b79026003710523cb80f2e78b88282b37
:104d600006d0b3f5977fc0d10120fff7defde8e75d
:104d700000228c2011461af0b3fbe2e7d4bd0d02ed
:104d800010b5cb6a0c460bb18a6a9a62d4e90a2341
:104d900062b1d362038a013b038294f842300bb1c3
:104da000032b05d1042384f8423010bd8360f1e762
:104db000606840b194f84330db070dd500210df059
:104dc000adf800236360e36833b9216b21b9204655
:104dd000bde810400df0a2b8044b04f11801e361e6
:104de0000348bde8104004f001b900bf714f000254
:104df0004cf600101fb5cb880c463f2b38d98b687a
:104e0000002b37d08b88816829b1b1f840209a42b5
:104e100001d0c96af8e700230122cde90233cde9c8
:104e2000002319b391f84230042b0dd8dfe803f0ca
:104e300003070c0312000223adf80c3004e0042336
:104e4000adf80c30fff79cff21466846fff7bcfd2c
:104e500004b010bdcb6b0193092300930b691bb108
:104e600002930d230093efe7c160ede70523e3e72d
:104e70000020ede71846ebe77fb5cb8804463f2bd3
:104e80000d4615d98868a0b18b884bb96ff08b0699
:104e9000a368e3b1de632046a168fff771fff7e77f
:104ea000a16841b1b1f840209a420ad0c96af8e736
:104eb000002004b070bd01230291cde9003105232b
:104ec0000ae06ff08b032046cb63fff759ff002306
:104ed0000122cde900230293294668460393fff798
:104ee00073fde6e74b78013b042b0ed8dfe803f0b7
:104ef000030507090b00fff7d7bdfff77bbffff7df
:104f000077befff7b3befff7b7bf0020704708b505
:104f100003465a780846013a0e2a194605d8fff783
:104f2000e1ff80f00100c0b208bdfff7cbfef8e75b
:104f3000012838b50c460bd0022815d16ff0950525
:104f4000a3689bb1dd632046a168fff719fff7e76f
:104f5000c96849b18a6b0b699a4205d10025204680
:104f6000cd63fff70dffe560002038bde360fbe790
:104f700038b54b6805460c4613b103685b68984723
:104f8000e3682bb12b680022214628461b6898470e
:104f9000236b13b1616be06b98472046bde8384046
:104fa00000210cf0bbbf2de9f0411f464b680546c0
:104fb0000c461646ddf8188013b103685b68984705
:104fc000c4e90c781af032f994f84230032b01bf8f
:104fd0000423e66384f8423000241af02bf92cb144
:104fe00021462846bde8f041fff7c2bfbde8f08189
:104ff000c1684869fff7bcbf08b56bf0b1f818b1dc
:10500000bde808403cf068bf08bd000070b50e4622
:10501000002486b005ab019304ab009305461c4900
:10502000304603ab02aacde90244cde90444c1f005
:105030005bf8042818d1029eff2e23d8039bff2b78
:1050400020d8049aff2a1dd80599ff291ad81b04d5
:1050500043ea06630b4343ea02232c706870c5f8e9
:105060000230204606b070bd3046fbf703ff3f28f4
:105070000ad801236870c21831462b70a81cbff0f3
:1050800081ffeee70348ede76ff0bd00eae700bf00
:10509000f0bd0d02f2feffff70b5032092b00d4689
:1050a0001af05efb002800f08e80002305a8cde9f1
:1050b00005336af001f95b22444905a86bf0e6fc70
:1050c000044640b13cf008ff044605a86af0f8f831
:1050d000204612b070bdcde90700099006206af0a5
:1050e0007fff064600286bd007a86af085ff22469e
:1050f000314607a86af0d8ff002854d107a86bf002
:1051000013f818b13cf0e8fe041e50dbab68042233
:1051100004a907a80493fff76fff041e47dbd5e936
:10512000011207a8fff768ff041e40db2868fbf7a1
:10513000a1fe04220490064604a907a8fff75cff1d
:10514000041e34db3246296807a8fff755ff041e0a
:105150002ddb41f23462ab890df10e01002b08bf4b
:10516000134607a80222adf80e30fff745ff041ed4
:105170001ddb00211c220ba80a91bff02aff0aa9ff
:1051800007a86bf007f8b0b96b69062101932b698a
:105190000aaa009305a820236af0f6f80c4b041e17
:1051a00018bf1c4603e03cf097fe041ea6da07a8d1
:1051b0006af027ff89e73cf08ffe041ef7dbe3e788
:1051c0006ff07704f3e76ff0770481e7fbbf0d0220
:1051d000e8feffff004870474cce001010b50446b3
:1051e000006808b124f09afb204610bd2de9f04775
:1051f0000024a8b01d4616469df8c0705b4a5c4b63
:105200004ff0200aa74208bf134681468846019303
:10521000584b1e20584900930deb0a022346cde956
:1052200008a4fdf739fb554b1e20534900930deba5
:105230000a022346cde90198cde908a4fdf72cfb2d
:105240004f4b01204c4900930deb0a022346019578
:10525000cde908a4fdf720fb2b4632460120cde91d
:1052600000444549fdf778fb02230120454a4249a5
:105270000094fdf71dfb214680220deb0a00bff0d4
:10528000a8fe49460deb0a00fff7c0fe041e5edbd8
:10529000002f14bf4ff0c0094ff44079a945adf875
:1052a000628060d348463849bff0eaf80446079068
:1052b000002853d04a46ff21bff08bfe40f6a2588b
:1052c00040f6a213002f08bf984680224146204690
:1052d00025f03ffcb0bb40f6e24140f62203002f30
:1052e00008bf19464a460798059125f032fc48bb8d
:1052f0002a463046059925f02cfc18bb9df8202045
:10530000079b012a27d89df82120402a28d844222b
:1053100018460deb0a01bff035fe9df8202003462c
:1053200022b9d0f8022012bac0f80220b3f8422005
:1053300052baa3f8422080224146079825f009fc82
:10534000044608b16ff0db0407a8fff747ff2046cb
:1053500028b0bde8f087ff221a70ece70b4cf3e7aa
:105360006ff0bd04f0e76ff0bd04f0e700be0d0282
:10537000fcbd0d0204be0d0260c30d0220be0d0275
:1053800038be0d023f030f0213081002fcfeffffa0
:1053900013b50c4603201af0e3f9a18931b941f2a3
:1053a000346141f23363002808bf1946d4e9012370
:1053b00000902068fff71aff00eae07002b010bd0d
:1053c00007b503201af0ccf968b1012341f234612a
:1053d00000935b23084a0948fff708ff00eae070e2
:1053e00003b05df804fb00904ff4937341f2336116
:1053f000034a0448f0e700bfa0bf0d024fbe0d02f4
:105400007abe0d0263be0d022de9f0430320a9b060
:105410001af0a6f9061e14bfc0274ff440774c4976
:105420003846bff02df801460390002800f08e802a
:1054300040f6a21340f6a2508022002e08bf184664
:1054400025f052fb014640b16ff0db0403a8fff7e3
:10545000c5fe204629b0bde8f083802208a8bff031
:10546000b8fd039c23781bb1012b47d0394cede7e5
:105470006278042afad1d4f802301bba591e0331db
:10548000f4d88df82120cdf82230b4f842305bba40
:10549000adf862309df82030ff2be7d040f6e240b7
:1054a00040f622033a462146002e08bf184625f052
:1054b0001bfb0028c8d103993023cde9041005aaad
:1054c000394404a860f023fb0028cfd1dde9032391
:1054d0009a1a059b07901344cde9053006a869f098
:1054e000ebfe059a039906a86bf0d0fa194b041e3f
:1054f00006a818bf1c4669f0e3fea7e76578ab1c59
:10550000802bb3d83f2db1d86fea0409a11c04f158
:10551000010809eb0803ab4208d218f8010f01910a
:10552000bff0e4fb01990028f3d19fe701232a464d
:105530000df122008df820308df82150bff022fdb2
:1055400028ab1d44002305f87e3c9ee7024c7de716
:1055500013081002f8f8fffffcfefffff8b5044641
:1055600005462f4615f8016b3046bff0b7fb002803
:10557000f7d15f2ef5d0381bf8bd2de9f8430c4666
:105580001746994678b119b38e18a64205d9054633
:1055900015f8013b4bb904f8013b0023781e341b7e
:1055a00006f8013c001bbde8f883242b0dd12846ea
:1055b000fff7d4ff804630b122460146331b284610
:1055c000c847454404442846dfe704f8013bfae7ae
:1055d0000846e8e70023202200b58bb0cde902237e
:1055e000054a01200092054902aafdf755f94ff03e
:1055f000ff300bb05df804fb56c00d0260c30d0216
:10560000f0b5002420274ff4837605460e4bc5b035
:10561000009302aa23461e200c49cde90274fdf72f
:105620003bf93246214602a8bff0d3fc3a46214658
:105630002846bff0cefc23462246314602a805f09c
:10564000fff945b0f0bd00bfb2c00d0260c30d024e
:105650002de9f041ceb04ff4837204460e460ca8fb
:105660000021bff0b6fc00234ff483711a460ca84a
:1056700005f008fab0f5837f2dd1bdf83030b3f5d1
:10568000837f28d180213046149d19f0d3ff8542b5
:1056900034d00025202780213046ddf85080cde928
:1056a000047519f0c7ff214bcde90180009304aace
:1056b0002b4632201e49fdf7eff89df83530322099
:1056c00001931c4b1a49009304aa2b46cde904759b
:1056d000fdf7e2f80ae020210023174acde9041380
:1056e00000922820124904aafdf7d6f82046fff7b9
:1056f00087ff4ff0ff304eb0bde8f0819df83530a8
:10570000002bc6d00dad0fcd0fc495e807000023c8
:1057100084e807002022cde90423084a1e200092d5
:10572000034904aafdf7b8f8e3e700bffec00d0285
:1057300060c30d0223c10d02cac00d0236c10d02a5
:1057400010b504460846802119f074ffe06100207e
:1057500010bd000030b50020b1b004f09df803206a
:1057600019f0feff0446e0b1364b1d88802200216f
:1057700010a8bff02efc10a828f098ff9df840203c
:1057800020218ab1012a4ff000034cd001922e4a09
:10579000cde90813009228202c4908aafdf77cf8cf
:1057a0001fe041f23365e1e7ddf84230cde9081250
:1057b000bdf882101e200791d9b20691c3f30721cc
:1057c0000591c3f307411b0e03930df14203cde98d
:1057d00001231f4b049100931c49134608aafdf7af
:1057e0005bf84ff6fd71bdf88220531e9bb28b42d1
:1057f00002d81cb1aa4201d0adf8825010a91548b8
:10580000fff726ff002c14bf11200620114a10a913
:1058100003f0c4fd044618b90e4810a9fff790ff25
:10582000204631b030bdcde908130df14201cde97c
:105830000121094a1e200092044908aafdf72cf80c
:10584000cfe700bf48510010d7c10d0260c30d0261
:105850006dc10d0250ce0010afc10d0204f01cb896
:1058600008b5002004f05af8c0b208bd0122014b6f
:105870001a7070474dce001013b50f4b04461b78bd
:1058800023b102b0bde81040fff7a4be0b4b01915d
:105890001b78002bf5d1fff7e3ff0028f1d1084b6f
:1058a0001b7803f0ff02002bebd12046019902b0d8
:1058b000bde8104003f08cbf2dd200102ed2001096
:1058c0004dce0010fff7d8bf13b50f4b04461b7821
:1058d00023b102b0bde81040fff77cbe0b4b019135
:1058e0001b78002bf5d1fff7bbff0028f1d1084b47
:1058f0001b7803f0ff02002bebd12046019902b088
:10590000bde8104003f090bf2dd200102ed2001041
:105910004dce0010fff7d8bf08b5002003f0e8ff18
:1059200010f1780f08bf002008bd002003f0f2bf7f
:10593000f0b5022806460d4614468db005d00a285b
:1059400034d01f4c20460db0f0bd202000231d4f49
:10595000cde904033a68cde901211b4a00920120f8
:105960001a4904aafcf798ff3d6000f0f5fd10b954
:1059700014f00104e6d0164b00245b78b342e1d169
:105980002023cde90434134b04aa009301202346bd
:105990000e49fcf781ff082202232946cde90423a2
:1059a0002046234604aa00f0cdfecbe720210023a9
:1059b000094fcde904133a68cde90125074acde73f
:1059c000f2feffff4051001013c20d0260c30d0232
:1059d00050ce001076c20d024451001044c20d0298
:1059e00019b1022803d00a2806d004487047044b96
:1059f0001b6800200b607047024bf9e7f2feffffc7
:105a0000405100104451001003689b6818470eb4c1
:105a100003b503ab53f8042b0021019311f0a7fd4c
:105a200002b05df804eb03b070472de9f041064683
:105a30000d46904627f01fff074627f01cffc01bae
:105a400040450ed83468236820461b6998470028d3
:105a5000f3d0236820465b69984728700020bde892
:105a6000f0814ff0ff30fae72de9f04f16461a4665
:105a7000002385b00f4633600df10f01019282467d
:105a8000fff7d3ff019a044628b14ff0ff342046b8
:105a900005b0bde8f08f9df80f50182d13d008d831
:105aa000022d20d0042df2d0012deed14ff0800830
:105ab0001be005f0df03412b35d0202d14bf4ff044
:105ac000ff340224e3e750460df10f01fff7adff6d
:105ad00004460028d9d19df80f30182bd5d14ff0ae
:105ae000ff333360d3e74ff48068b94609f8015bb0
:105af000012508f1040b5d450cd84946504601923a
:105b0000fff793ff09f101090028bed10135019a81
:105b1000adb2f0e7bb787a78db43dbb29a42b4d11e
:105b2000c6f80080b3e70124b1e738b50d4600217f
:105b300002f58070033313f8014b2cb1b1f5807f6f
:105b400002d054540131f6e700245454ff32195d59
:105b5000202905d0102c03d0013402f8011ff6e7ec
:105b600000210a220155c1f0f1f94ff48063e86089
:105b70002b8138bdf8b51d46531c04460cd08ab1a4
:105b8000d0f818644f78f3b29f4213d00068152103
:105b9000fff73aff012004e000680621fff734ff19
:105ba0000020f8bd00680621fff72eff0120c4f891
:105bb0001404f6e786bbcb7803b30b46069a294656
:105bc000fff7b3ff32463146284609f0a5fe50b133
:105bd00018212068fff718ff20681821fff714ff2d
:105be0004ff0ff30dde72b6906216b602068fff77f
:105bf0000bff43212068fff707ff04e00123c0f8f3
:105c00001434c0f810340120d4f81834c4f8200437
:105c10000133c4f81834c4e72a812846002203312e
:105c200009f0ecfe50b118212068fff7edfe206866
:105c30001821fff7e9fe6ff00100b2e76b682a89cf
:105c4000062113446b60d5e72de9ff411746044652
:105c500000250e464ff4887200213846bff0b9f98e
:105c600004f10808c4f81054c4f81c54c4f82054b3
:105c7000c4f81854c4f8145441462046636803aa73
:105c8000fff7f2fe012810d0022819d030bbc4f86b
:105c90001c04334641462046039a0097fff76affeb
:105ca000002811dc04b0bde8f08118212068fff75e
:105cb000abfe20681821fff7a7fe6ff00200f1e7a6
:105cc00006212068fff7a0fed4f81434002bd3d0af
:105cd000d4f81034002bcbd0f068e3e7d4f82034ac
:105ce000002b08dbd4f81c34432101332068c4f8ae
:105cf0001c34fff789fed4f81c34052be4dd182191
:105d00002068fff781fe20681821fff77dfe002044
:105d1000c8e70000f0b50446c7b040f224400f4683
:105d200023f0f6fd054618b141f288330460436064
:105d30003946284602aafff787ff061e48dd0022e3
:105d40000121384609f010fe021e31db06212868c9
:105d5000fff75afe20462a4911f009fb204629493f
:105d600011f0f2fa204602a911f0eefa2046264977
:105d700011f0fdfa2046254911f0e6fa0a223146d3
:105d8000204611f0fefa2249204611f0f0fa23686d
:105d90002046db6998474ff47a7024f080fd012497
:105da000284640f2244123f0bbfd204647b0f0bd19
:105db000182128680192fff727fe18212868fff7ad
:105dc00023fe2046019a1349fff721fe0024e7e74e
:105dd00018212868fff718fe18212868fff714fe1d
:105de000721c04d10c49204611f0c1faeee7b31c35
:105df00001d10a49f7e703360cbf09490949f2e71f
:105e00009ac20d02bac20d02c3c30e02c1c20d0274
:105e100091ef0d02c8c20d02e0c20d0217c30d02c0
:105e20002dc30d023ec30d0201200bf0adbf08b51e
:105e30000023c269006f2ef0cafab0fa80f0400960
:105e400008bd70b505460e46806900212ef08afa1d
:105e5000002304461a463146286f2ef0d9fa18b1ad
:105e6000201e18bf012070bd0120fce708b50023eb
:105e70008269006f2ef0ccfab0fa80f0400908bdbc
:105e800038b50546fff7d3ff044620b1686e10b160
:105e900000212ef06bfa204638bd012a02d10160a4
:105ea00000207047022a04bf0b680360f8e703680c
:105eb00018470000014b18682ef0e9ba00cf001017
:105ec00010b5044c236813b920462ef0fcfa206864
:105ed00010bd00bfecce001010b50a4cd4e88f3fc7
:105ee000db070cd4204625f009ff40b106482ef010
:105ef000c4fa204625f03cff0448bef01cfe0248d0
:105f000010bd00bf74ce001000cf0010355e00023f
:105f1000014b1860704700bf70ce001038b50023e9
:105f200083608b6804460d462bb102229847eb68cc
:105f3000e360ab68a360204638bd000030b52a4b53
:105f40009db00093294b69460393294b04a8029303
:105f5000fff7e4ff4ff420526423cde908236ff0ec
:105f600000430a933223adf82c300223214c3f2208
:105f700021490df12f008df82e30c0f07dfe204616
:105f80001e4b04a940f8043bfff7c8ff089b04f12f
:105f900023026361099b0df16f01a3610a9be36119
:105fa000bdf82c3023849df82e3084f822300df17a
:105fb0002f0353f8040b8b4242f8040bf9d1002550
:105fc0000f4865662ef059fa0e4b04a8236084f83a
:105fd0006c502567fdf768fb6846fdf765fb0a4bcb
:105fe0009d601db030bd00bfa95d00022f5e0002a4
:105ff0001b5e000278ce00105ac30d0270c30d0262
:10600000e0ce001080c30d02f0ce001010b5c368c2
:1060100004460bb9bef036fa03690430984723688a
:106020002046bde810409b68184710b5c368044679
:106030000bb9bef027fa0369043098470021a0612c
:106040006069bde810402ef09dba10b5c3680446e3
:106050000bb9bef017fa0369043098470021207687
:106060006069bde810402ef08dba08b505f01afb46
:10607000002008bd07b51346002200920a460146db
:106080000548006812f0c9fa002818bf6ff0ef0049
:1060900003b05df804fb00bf2cd40010012a70b5da
:1060a000054603d10b680360002070bd022a08d0aa
:1060b000032af9d100680028f6d0102123f030fc23
:1060c000f2e710200e6823f023fc044618b196e88e
:1060d0000f0084e80f002c60e6e7012a70b5054642
:1060e00003d10b680360002070bd022a08d0032a88
:1060f000f9d100680028f6d0102123f011fcf2e756
:1061000010200e6823f004fc044618b196e80f0036
:1061100084e80f002c60e6e7012a08bf0160002038
:106120007047012a38b5044602d10b68236003e0aa
:10613000022a03d0032a0dd0002038bd0c200d68a0
:1061400023f0e6fb03460028f0d095e8070083e83b
:106150000700ebe700680028eed00c2123f0e0fbfd
:10616000eae7012a70b5054603d10b6803600020f9
:1061700070bd022a08d0032af9d100680028f6d0a1
:10618000102123f0cdfbf2e710200e6823f0c0fbb6
:10619000044618b196e80f0084e80f002c60e6e78b
:1061a000012af8b5064603d10b6803600020f8bd4c
:1061b000022a08d0032af9d100680028f6d0142159
:1061c00023f0aefbf2e714200c6823f0a1fb074696
:1061d00020b105460fcc0fc523682b603760e5e77b
:1061e000012af8b5064603d10b6803600020f8bd0c
:1061f000022a08d0032af9d100680028f6d0142119
:1062000023f08efbf2e714200c6823f081fb074695
:1062100020b105460fcc0fc523682b603760e5e73a
:10622000012a034602d1016000207047022a04bf00
:10623000d1e90001c3e90001f6e7012a02d10160ba
:1062400000207047022a04bf0b680360f8e7012aa8
:1062500008bf016000207047012a02d101600020c0
:106260007047022a04bf0b680360f8e7012af8b5fb
:10627000064603d10b6803600020f8bd022a08d04f
:10628000032af9d100680028f6d0182123f048fb32
:10629000f2e718200c6823f03bfb074630b10546b7
:1062a0000fcc0fc594e8030085e803003760e3e7ef
:1062b000012a034602d1016000207047022a04bf70
:1062c000d1e90001c3e90001f6e700224ff0ff31f8
:1062d0002ef038b900224ff0ff312ef033b9000014
:1062e00010b50446034b40f8043bfdf7ddf92046aa
:1062f00010bd00bf08c40d0210b50446fff7f0ff43
:106300002046142123f00cfb204610bd10b5044696
:10631000024b0360fff7e4ff204610bd1cc40d02d2
:1063200010b50446fff7f2ff2046142123f0f8fad7
:10633000204610bd10b50446034b40f8043bfdf762
:10634000b3f9204610bd00bf90c30d0210b504463e
:10635000fff7f0ff2046142123f0e2fa204610bd9b
:1063600010b5074b04460360406918b12ef0e5f8fc
:10637000002363612046fff7ddff204610bd00bf0c
:10638000a4c30d0210b50446fff7eaff204618210a
:1063900023f0c6fa204610bd10b50446024b036038
:1063a000fff7deff204610bdb8c30d0210b504464e
:1063b000fff7f2ff20461c2123f0b2fa204610bd61
:1063c00010b50446034b40f8043bfdf76df9204639
:1063d00010bd00bfccc30d0210b50446fff7f0ff9f
:1063e0002046142123f09cfa204610bd10b5074b1f
:1063f00004460360406918b12ef09ff800236361e2
:106400002046fff7ddff204610bd00bfe0c30d02b0
:1064100010b50446fff7eaff2046182123f080fa62
:10642000204610bd10b50446024b0360fff7deffa7
:10643000204610bdf4c30d0210b50446fff7f2ff6d
:1064400020461c2123f06cfa204610bd406e2df032
:1064500046bf000010b404460748134600682ab13e
:10646000214600235df8044b11f0bcbf0a462146cb
:106470005df8044b11f0bdbf2cd40010f0b52e4eca
:10648000044696f86c300d4687b0002b4ad0304653
:10649000fff7dcff0746002844d1284b1c2005935a
:1064a000274bcde90245049323f032fa0446002835
:1064b00031d0244bc7600360049b3bb1022202a988
:1064c00004309847059b2361049be3600025204628
:1064d0001d4b2a462360012140f8145f2ef022f85c
:1064e0001a4b01a92360f2692b46306f01942df0fd
:1064f0006eff014650b9706e08b12df037ff0022d3
:106500004ff0ff3160692ef01df8a5692368204621
:106510009b68984700e0054602a8fdf7c5f82846a5
:1065200007b0f0bd05f02af92a46214607b0bde8bc
:10653000f04012f0a6b800bf78ce0010d16400027f
:10654000a1610002ccc30d02e0c30d02f4c30d0231
:10655000d0e90001fff792bf054b1b7803f0ff0065
:1065600023b1044b1878003818bf0120704700bfd2
:106570005dd400105ad4001008b50948fff766ff33
:1065800058b1002008f002fd20b1bde808400448e1
:1065900002f000bd01200bf0f7fb002008bd00bf9a
:1065a0005cd50010002190b583b0044600af0846ca
:1065b00022f0f4fdc31d23f00703adeb030d0146ec
:1065c0007860684622f0eafd20467a68694605f060
:1065d0005bfe20460c37bd4690bd0000014b1860a5
:1065e0000020704728d400107fb51d4d044695f853
:1065f0006c300e46b3b12846fff728ff90b9194b0f
:1066000069460393184b2846cde900460293fdf7ef
:106610004ff9044688b905466846fdf745f828460f
:1066200004b070bd94b1631c13d021460f4802f032
:106630006ffe0e4802f059fe0be04069fff74afe7c
:10664000236820469b68a5699847e5e7074802f05c
:1066500047fe064804b0bde8704002f09dbe00bf92
:1066600078ce0010f16500023162000204cf001004
:10667000d0e90001fff7b8bf2de9ff41014640b363
:10668000684610f0bffa009e9df80940ddf80480ce
:106690009df80850fff760ff00b305f021fe4ff0b2
:1066a0000103d0e8cf7fc0e8423f002af9d1ffb212
:1066b000002ff6d1c660c0f8108005754475002320
:1066c000c0e88f3f08f02afc0024204604b0bde853
:1066d000f0810546804604460646dbe708f01efcce
:1066e00016f0040625d0002cefd0134c94f86c3033
:1066f00013b904f0d7ffe7e72046fff7a7fe00280d
:10670000f7d10e4b694603930d4b20460293fdf7dc
:10671000cff8054658b14069fff7dcfd2b682846e5
:106720009b68ac6998476846fcf7beffcde7044616
:10673000f9e73446c9e700bf78ce0010eb5f0002ee
:1067400099600002f0b504462c481f4690f86c3062
:106750000e46154687b0dbb1fff778fec0b904904e
:10676000102023f0d5f818b1c0e90046c0e902575f
:10677000234b02900593234b204802a90493fdf775
:1067800097f8044660b9054602a8fcf78dff04e0bf
:10679000012c25d9022c0cd01b4d284607b0f0bd8a
:1067a0004069fff797fd236820469b68a5699847d5
:1067b000eae7294602a810f025fa05f091fd029bb0
:1067c0000025d90744bf9df8102002729a0744bfe4
:1067d000039a42605b0744bf9df811304372dce7c7
:1067e0000a4800972b4632462146006811f0dffe2a
:1067f00007b0bde8f04011f011bd00bf78ce001029
:10680000916700025b600002f2feffff2cd40010d3
:106810000068d0e90223d0e90001fff793bf000030
:1068200030b5044628481d4690f86c3087b00bb34d
:10683000cde90012fff70afedde90012d0b904909d
:10684000102023f065f828b1019a0099c0e90225cb
:10685000046041601d4b029005931d4b1a4802a92c
:106860000493fdf725f8044670b9054602a8fcf725
:106870001bff06e0042c19d0052c1cd0032c0cd0d7
:10688000144d284607b030bd4069fff723fd23684b
:1068900020469b68a5699847e8e70f4b1b787bb1ba
:1068a000082007b0bde83040fff7e4bb0a4b1b7877
:1068b00033b10920f5e7084b1b780bb10a20f0e74c
:1068c0006ff0d105dde700bf78ce00105d680002f3
:1068d0001d600002f2feffff5ad400100068d0e9ec
:1068e0000223d0e90001fff79bbf000073b5064605
:1068f0001c200d4623f00cf8044628b3144b03600b
:106900000023c360ab683bb102222946043098479c
:10691000eb682361ab68e360002220460d4b012148
:10692000236040f8142f2df0fdfd0b4b3046236003
:10693000336801945b6801a99847054620b923682c
:1069400020469b6898472c46204602b070bd00bf89
:1069500090c30d02a4c30d02b8c30d022de9f0438c
:1069600005462e48994690f86c3087b00e46904602
:106970000e9f2bb3fff76afd10bb0490182022f086
:10698000c7ff40b10f9bc0e90056c0f8088080f8ef
:106990000c9007614361224b02900593214b1f48e5
:1069a00002a90493fff7a2ff054670bb044602a8a4
:1069b00004f00104fcf778fe204607b0bde8f08340
:1069c000b9f1000918bf4ff00109cde90078164868
:1069d0004b4632462946006811f012fd0446002855
:1069e000ead0fff7b9fd06460028e5d008f0c2fa64
:1069f000012803d10d4b1b78002bddd03a464946c8
:106a00002846fff727fd3446d6e74069fff75dfccf
:106a10002b6828469b682c7e9847c8e778ce0010e4
:106a2000b1690002ed6100022cd400101cd60010e8
:106a300007b500684269037b019202690092d0e9c0
:106a400001120068fff78aff03b05df804fb000045
:106a500030b5174c054694f86c3085b003b320462a
:106a6000fff7f4fce0b9134b20460393124b694641
:106a700000950293fff73aff044678b14069fff7ab
:106a800024fc236820469b68257e9847684605f0cd
:106a90000105fcf709fe284605b030bd0546f5e7bf
:106aa00004f06cfe002105b0bde8304011f0e6bdf9
:106ab00078ce00103d6a0002bb6100020068fff75b
:106ac000c7bf0000f0b5044622481f4690f86c305e
:106ad0000d46164685b0fbb1fff7b8fce0b9029051
:106ae000102022f015ff18b1c0e900450672c760fa
:106af000194b00900393194b694616480293fff710
:106b0000f5fe054658b90446684604f00104fcf752
:106b1000cbfd204605b0f0bd55b9002415e0406915
:106b2000fff7d3fb2b6828469b682c7e9847ebe742
:106b30005cb12046faf79ef94028eed820463b4645
:106b40003246294604f040fe0446003c18bf0124aa
:106b5000dfe700bf78ce0010e16a0002e3600002c8
:106b60000068c368027ad0e90001fff7abbf0000fc
:106b70007fb5054622480c4690f86c301646f3b1b6
:106b8000fff764fcd8b902900c2022f0c1fe10b1ce
:106b9000c0e9005486601b4b009003931a4b694672
:106ba00017480293fff7a2fe044680b905466846df
:106bb00005f00105fcf778fd284604b070bd7db9ed
:106bc0003146204604b0bde8704004f0b6bf4069cd
:106bd000fff77bfb236820469b68257e9847e6e706
:106be00010230021adf80030084b68460195cde92f
:106bf0000234adf8021004f0a0ff0546dce700bf48
:106c000078ce0010916b0002a360000279b90002f7
:106c100003681868d3e90112fff7aabf73b50646e7
:106c200014200d4622f074fe0446d0b10e4b0360d2
:106c30000023c360ab683bb1022229460430984769
:106c4000eb682361ab68e360084b30462360336830
:106c500001945b6801a9984718b9236820469b688e
:106c6000984702b070bd00bf08c40d021cc40d02dd
:106c700030b5114c054694f86c3085b08bb1204688
:106c8000fff7e4fb68b90d4b694603930c4b2046b4
:106c900002930095fff7c2ff6846fcf705fd05b0bb
:106ca00030bd0022074b1146186811f06efc05b08c
:106cb000bde8304004f042bb78ce0010496c0002c1
:106cc000d96100022cd400100068fff7d1bf00008a
:106cd0001fb50e4c94f86c3083b12046fff7b6fb1d
:106ce00060b90b4b694603930a4b20460293fff7aa
:106cf00095ff6846fcf7d8fc04b010bd0021064b98
:106d0000186804b0bde8104011f014bc78ce001033
:106d1000ab6c0002cf6100022cd4001008b5fff765
:106d2000d7ffbde80840fff717bcfff7d1bf000051
:106d30002de9f04705463d4886b013f0100f1c467c
:106d40000e461746ddf8389090f86c300df10808c3
:106d500022d003f0ff0a002b46d0fff777fb002874
:106d600042d10490142022f0d3fd28b1c0e900568e
:106d7000c0e90274c0f810902d4b029005932d4b82
:106d800041462a480493fff749ff4046fcf78cfc34
:106d9000504606b0bde8f08733b3fff757fb18bb8a
:106da0000490142022f0b4fd28b1c0e90056c0e9d7
:106db0000274c0f81090204b029005931f4b41467f
:106dc0001a480493fff792fd044658b14069fff753
:106dd0007cfa236820469b6894f818a098470af02c
:106de000010ad2e78246fae70023cde903330c23f8
:106df0000293b9f1000f05d0d9f804300393d9f804
:106e00000830049314f0010f14bf4522652224f0ca
:106e1000010313430a480093cdf804803b463246f1
:106e20002946006811f080fa8246b1e778ce00105a
:106e3000c56d000261610002df6d00022161000288
:106e40002cd4001007b5006803690093d0e9022331
:106e5000d0e90001fff76cff03b05df804fb07b554
:106e6000006803690093d0e90223d0e90001fff72d
:106e70005fff03b05df804fb0021014802f0d2b9c6
:106e800004cf001030b5cc1c2a3114f8035c033455
:106e900005f00f0205f0f00342ea021243ea15156d
:106ea000130243ea0543436014f8052c02f0f00591
:106eb00045ea12152b4302f00f024360827214f868
:106ec000043ca14203eb830303eb83034fea430338
:106ed00020f8083fd9d130bd002138b50446084616
:106ee000fbf702fe1c2500232046094c05fb03424c
:106ef000416801331161817a0d2b517330f8081ffd
:106f00009182f3d10021bde838400120fbf7ecbdb0
:106f100014cf00100c2808b50ad81c22054b02fb20
:106f20000030002201730121fbf79afd002008bd0b
:106f30000120fce714cf001011f0040238b50cd08a
:106f400000240b4d0022284611460134fbf788fd32
:106f50000d2c05f11c05f5d138bd0c28fcd81c24de
:106f6000034b114604fb0030bde83840fbf778bd09
:106f700014cf00100c289fbf1c22044b02fb0030d2
:106f8000807b94bf00f001000020704714cf0010f8
:106f9000f0b58a0705460c469db01cd50125682230
:106fa000002102a8bef015f8214901a80195fff7bc
:106fb00069ff01a8fff790ffe30709d5ff232a46e1
:106fc00040f6af618df803300df1030023f0c1fdf1
:106fd00000201db0f0bd0368012b27d1fff77cff17
:106fe00014f00100f5d001a9084632262b46683579
:106ff0005a68c2f30357c2f3033444ea07144c70cf
:107000009c7a02f0f00204f00f0422438a7033f8f5
:10701000082fb2fbf6f29d4201f8032fe8d10123bd
:10702000402240f6af618df80430cfe70120d0e771
:1070300028c40d0270b50268012a18d111f00201ae
:1070400005d00c49fff71eff0021084670bd0b4616
:107050001c26094d06fb0352146901334460547b1e
:107060000d2b8472928a20f8082ff3d1ede70121cd
:10707000ebe700bf28c40d0214cf00100c289dbf01
:107080001c22024b02fb00300020704714cf00107e
:10709000022803d0032807d000207047142909d004
:1070a0000adc4ff4fa707047142907d009dc4ff45a
:1070b000fa507047c8207047642070474ff47a60d8
:1070c00070474ff47a7070470021224a30b50b4662
:1070d00015461c24adb004fb015001310d29c2e955
:1070e00000439360037302f11c02437383730361d3
:1070f0008382f0d16822002112a8bdf06aff01232b
:10710000402240f6af6001a9119323f0edfc18b9bd
:107110009df80430012b1ad00f4b01aa03f1200572
:10712000144618685968083303c4ab422246f7d1a5
:10713000998818689b79a1802060a37101a911a882
:10714000fff7a0fe11a8fff7c7fe2db030bd0df16f
:107150000501f4e714cf0010dcae0d022de9f04f6d
:107160004ff0180a91469b460e46154985b0d1e965
:10717000004103900afb014adde90e780c34a4f1ca
:107180000c018a4511d054e90301039b314018409a
:1071900050ea010307d000945b464a463146039803
:1071a00054f8045ca8471834e9e72fb140463b4641
:1071b00005b0bde8f04f184705b0bde8f08f00bf3f
:1071c00080d0001030b5d1e90054d0e900232a4026
:1071d000234013430cd0836813b18a68934207d1cc
:1071e000c3683bb158680b69c31a5842584130bd57
:1071f0000020fce70120fae7704710b5044628217b
:1072000022f08efb204610bd012af8b5064603d1b8
:107210000b6803600020f8bd022a08d0032af9d1c8
:1072200000680028f6d0182122f07afbf2e7182037
:107230000c6822f06dfb074630b105460fcc0fc538
:1072400094e8030085e803003760e3e72de9f043a5
:10725000dff8d88093b08146d8f800000e46154676
:107260001c462df03ff917f0e1ff00230746cde95a
:107270000096cde90333029505933cb1628821461f
:107280000c2a28bf0c2203a8bdf07cfe6d4606ac7c
:107290000fcd0fc495e803000cae0df1180c84e877
:1072a0000300bce80f001f4d0fc694e80300d5f89b
:1072b0000490ab6886e8030099451adb09f10104e4
:1072c000002c286810dd18216143bef003fe70b960
:1072d000154c384617f0aeffd8f800002df011f924
:1072e000204613b0bde8f083bdf026fe00202860e4
:1072f000ac6018236a6803fb09f95a432c68a2ebb7
:1073000009024c442146e0180caebdf048fe0fcef9
:107310000fc496e803006b6884e80300013300247f
:107320006b60d6e780d00010fcfeffff8cd0001011
:107330002de9f04f8fb00193574b8346186889466b
:1073400016462df0cff817f071ff1822534fcde9f4
:1073500002b9d7e90045019b554304960deb020c99
:1073600005930df108090aae824699e80f008ce8f2
:107370000f0086e80f004a4b04eb0508ed105d4353
:10738000ad10002d1ddd21463046fff71bff30bb41
:10739000a346183421463046fff714fff8b90bf125
:1073a000300421463046fff70dffc0b90bf1480409
:1073b00021463046fff706ff88b90bf16004013d16
:1073c000dfe7a8eb0403302b27d0482b1ed0182b67
:1073d0004cd121463046fff7f5fe002846d0a045a7
:1073e00045d004f11806b04541d031464846fff774
:1073f000e9fe48b92546b446bce80f000fc59ce835
:10740000030085e8030018341836ece721463046bf
:10741000fff7d8fe0028e2d1183421463046fff7a6
:10742000d1fe0028dbd11834d3e71d48e31adb1066
:10743000151b00fb03f304d4ed104543581981429a
:1074400000dacd1a182101fb05412046521abdf081
:10745000a6fd7b685b1b7b60504617f0ebfe0e4b76
:1074600018680fb0bde8f04f2df04bb84446182611
:107470007a683b6806fb02339c42edd02546d7e98b
:10748000003106fb01329542cfd0286910b16b69fb
:1074900003b198471835f2e78cd0001080d0001067
:1074a000abaaaaaa2de9f0471f461e4b164693f831
:1074b0006c2086b00546dde90e890c46eab1586eaf
:1074c0002cf00dffc8b90490182022f021fa28b141
:1074d000c0e90054c0e90267c0e90489124b029078
:1074e0000593124b02a90f480493fff797fb02a8dc
:1074f000fcf7daf806b0bde8f087dff834a0daf878
:1075000000002cf0efff28463b4632462146cde9ed
:107510000089fff723fedaf8000006b0bde8f04767
:107520002cf0efbf5cd50010797500028971000264
:107530008cd000102de9f047dff860c00746dde988
:107540000898dcf804c00e46ccf3080c15461c461f
:10755000bcf1000f16d0002128200af0b5fc01462e
:10756000a0b1002383600a4bc0e904760360c0e940
:107570000654c0e90898074b4360bde8f047064849
:1075800001f034bdbde8f047fff78cbfbde8f087e0
:1075900058c40d02537500024cf6001000ed00e0d7
:1075a00010b4039ce40703d55df8044bfff7d6bd88
:1075b0005df8044bfff7bebf002307b5024600216c
:1075c0004ff48040cde90033fff7b4ff03b05df81e
:1075d00004fb13b50446436a0193036a0093d0e9a0
:1075e0000623d0e90401fff75dff0021204602b029
:1075f000bde810400af092bc07b501684b690193e1
:107600000b690093d1e90223d1e90001fff74aff9a
:1076100003b05df804fb00000023044a0448c2e9fb
:107620000033936003602cf04ebf00bf80d0001089
:107630008cd00010002210b51146044600f098fdd1
:10764000024638b1002320461a46194600f078ff5a
:10765000012010bd0146204600f0d9fd0028f8d0d9
:10766000f0e7002373b506220093032101200af0fe
:10767000b7f90320fff7deff06460420fff7daff25
:1076800005460520fff7d6ff0023044626b11a461b
:107690001946032001f08ef82db1002304201a466c
:1076a000194601f087f844b1002305201a4619460f
:1076b00002b0bde8704001f07db802b070bd8369d2
:1076c00000200b60704738b5144619b904220846eb
:1076d000226038bd1368032b07d903685b6898479d
:1076e0000028f6d104232360f3e76ff0bd00f0e734
:1076f000836900200b6070471830036800200b601e
:1077000070471830036800200b60704738b5054695
:107710000c4617f08bfdab69236017f08bfd002042
:1077200038bd000070b5044626f0a5f8124e034699
:10773000726b06f120001ab19b1ab3f57a7f18d349
:107740001023002133621af09bf9051e0fdb26f08f
:1077500092f87063094e234606f11004324603cabc
:10776000a24218605960164603f10803f6d1284674
:1077700070bd0025eee700bff4d1001014d2001058
:107780001fb568460c46fff7cdff0028a4bf039b3a
:10779000236004b010bd1fb568460c46fff7c2ff5a
:1077a0000028a4bfbdf80a30236004b010bd1fb587
:1077b00068460c46fff7b6ff002807db9df805205a
:1077c000bdf80830d20748bf5b42236004b010bd4b
:1077d0001fb568460c46fff7a5ff0028a4bfbdf8fb
:1077e0000630236004b010bd70b50e4e88b026f090
:1077f00042f8336b1bb1c01ab0f57a7f0ed30a4c36
:1078000068460a4902ad0ff05ff80fcd0fc495e846
:10781000030084e8030026f02ef83063014808b026
:1078200070bd00bff4d10010fcd10010a4f700100f
:1078300038b50d46fff7d8ff044688b103685b6989
:107840009847b5eec00af1ee10fa0cd42368204632
:107850009b699847beeec80a002085ed000a38bd36
:107860006ff07700fbe76ff06300f8e738b50d467f
:10787000fff7baff044688b10368db689847b5eea6
:10788000c00af1ee10fa0cd4236820461b69984711
:10789000beeec80a002085ed000a38bd6ff0770003
:1078a000fbe76ff06300f8e738b50d46fff79cff84
:1078b0000446b8b103685b699847b5eec00af1eebb
:1078c00010fa12d4236820465b699847dfed087ae6
:1078d00020ee270abceec00a10ee103a00209bb240
:1078e0002b6038bd6ff07700fbe76ff06300f8e7bf
:1078f0000000804338b50d46fff776ff0446b8b167
:107900000368db689847b5eec00af1ee10fa12d4ae
:1079100023682046db689847dfed087a20ee270ac7
:10792000bceec00a10ee103a00209bb22b6038bdae
:107930006ff07700fbe76ff06300f8e7000080432b
:1079400010b50c46fff750ff28b103689b689847b5
:107950002060002010bd6ff07700fbe70048704703
:1079600090d000102de9f041504c08212046504a9b
:107970000025fbf729fd1c2114274e4b4e4a23609e
:107980006018a561fbf720fd4c4bdff8cc81e3616b
:107990004b4b4c4ec4e90f734b4b2946636404f1c7
:1079a0003803a3646563c4f83880e66404f13c00de
:1079b000fbf7f0f9454b2946a363454bc4e914583e
:1079c000e365444ba765236604f15403c4e9193603
:1079d00004f15800fbf7def93f4b092163653f4a8c
:1079e000e56604f17000fbf7effc3d4bc4f88850ee
:1079f00023673c4c3c4b182223603033636029469c
:107a000004f10800bdf0e5fa1022294604f1200037
:107a1000bdf0dffac4e90c55344c21212046344a2c
:107a2000fbf7d2fc334b25212360334c334a2046ed
:107a3000fbf7cafc324b22212360324c324a2046eb
:107a4000fbf7c2fc314b23212360314c314a2046e5
:107a5000fbf7bafc304b24212360304c304a2046df
:107a6000fbf7b2fc2f4b282123602f4c2f4a2046d6
:107a7000fbf7aafc2e4b292123602e4c2e4a2046d0
:107a8000fbf7a2fc2d4b2a2123602d4c2d4a2046ca
:107a9000fbf79afc2c4b2b2123602c4c2c4a2046c4
:107aa000fbf792fc2b4b2360bde8f08190d00010d7
:107ab00060c40d0218c50d0269c40d0228c50d026f
:107ac0000c0002009932000276c40d0238c50d0286
:107ad0001b00020080c40d0248c50d028cc40d02bb
:107ae00058c50d02f4d1001020df0d0234d1001072
:107af00094c40d0278c50d0264d100109fc40d021c
:107b000098c50d021cd10010abc40d0268c50d0252
:107b10004cd10010b7c40d0288c50d027cd10010f5
:107b2000c4c40d02a8c50d02c4d10010cbc40d02ff
:107b3000d8c50d02dcd10010dcc40d02e8c50d0271
:107b4000acd10010edc40d02c8c50d0294d10010d7
:107b5000fec40d02b8c50d02a8bc0d0230b5134b12
:107b60008db01d78e5b10024042022460df10f01ef
:107b70001c708df80f4007f0a1fd9df80f3093b1f8
:107b80002023cde904340a4b1e200a49009304aa9d
:107b90002346faf781fe22462146042007f076fdaf
:107ba00028460db030bd1d46fae700bf4a5100100f
:107bb000f0c50d0260c30d02012a38b5044602d19a
:107bc0000b68236003e0022a03d0032a0dd00020b3
:107bd00038bd0c200d6821f09bfe03460028f0d034
:107be00095e8070083e80700ebe700680028eed07f
:107bf0000c2121f095feeae7012a02d10160002064
:107c00007047022a04bf0b680360f8e7012a0346a5
:107c100002d1016000207047022a04bfd1e90001af
:107c2000c3e90001f6e7012a02d101600020704794
:107c3000022a04bf0b680360f8e7012a034602d159
:107c4000016000207047022a04bfd1e90001c3e9a6
:107c50000001f6e7012a02d1016000207047022ae4
:107c600004bf0b680360f8e707b5016811f0010174
:107c7000019107d107f054ff019903b05df804ebbf
:107c800008f004b807f04cff03b05df804eb08f00f
:107c900059b8000007b5006850b101a9c0b234f06e
:107ca00009fd28b904f060ff0122019905f008fee2
:107cb00004f05aff05f0c8fb0122044b1a700022a1
:107cc000034b1a7003b05df804fb00bf2fd2001005
:107cd0002ed2001030b50d46044685b010bb0346c9
:107ce0000a4600900321012009f07afe194b1c700e
:107cf0000122194bc3e88f2f04f036ff07222146db
:107d000005f02aff04f030ff294605f00dfcf0b91c
:107d100004f02aff05f062fa022818d0012022f0b0
:107d2000befdf5e703a9c0b234f0c4fc48b904f0c5
:107d30001bff2a46039905f00fff04f015ff05f01d
:107d400005fa04f011ff05f0bef80028dad005b0fe
:107d500030bd00bf2fd2001030d200100179006872
:107d6000fff7b8bf10b504461c220021bdf031f961
:107d7000204610bd38b50c460546fff7f3ff34b179
:107d8000637823b1214628462278bdf0fbf82846c7
:107d900038bd1fb543780446022b05d14068b0fac0
:107da00080f0400904b010bd0a2b0bd11022002135
:107db0006846bdf00ef91022684604f10801bdf0d6
:107dc000d1f8ece7b3fa83f0ebe784b02de9f041aa
:107dd00005468eb005f11c0715ae86e80e00fff7cc
:107de000c1ff3846fff7beff0fceee46aee80f00ec
:107df00096e807000df11c0c1cae8ee807000fceb4
:107e00000024ace80f0096e80700e8462e468ce810
:107e1000070085f83840b8e80f000fc69ee8070055
:107e200086e807003e4607af0fcf0fc69ce8070065
:107e300086e807006b7f022b12d1286a35f05efcc2
:107e400020b390faa0f3b3fa83f3c3f12003dbb2bb
:107e5000284685f838300eb0bde8f04104b07047d0
:107e60000a2b13d1234605f1240105f1340011f842
:107e7000012b002aecd092faa2f2b2fa82f2c2f1fd
:107e8000080213448142dbb2f1d1e1e70023dfe7ce
:107e900010b50446006fbdf04ff8606ebdf04cf8b1
:107ea000a06dbdf049f8e068bdf046f82068bdf06f
:107eb00043f8204610bd000084b037b506ac84e816
:107ec0000f0000240d9d9df819002c6060b19df8f5
:107ed000182010460192bdf027f8286048b1019a99
:107ee00006a9bdf04ff8204603b0bde8304004b00d
:107ef00070470148f8e700bffcfeffff2de9f0479f
:107f000092b01a9f0546894616469846002f00f003
:107f1000a280142021f0fcfc0446386018b94f48b8
:107f200012b0bde8f0874ff0140a00215246bdf0b0
:107f300050f86b68a4f800a0002b84f804904add88
:107f40004ff03c092d68083409fb03590df1200a54
:107f5000a94540d0142021f0dbfc20600028ded0b1
:107f600014220021bdf035f8ae460df1100cbee82c
:107f70000f00ace80f009ee807008ce807002368bc
:107f800003939ae807008de8070004ab0fcbfff7d7
:107f900093ff0028c4db05f11c0e0df12c0cbee88c
:107fa0000f00ace80f009ee8070023688ce807008c
:107fb0008de80700043303930bab0fcbfff77cff77
:107fc000002805f13c05abdb236815f8042c1a7278
:107fd00024681034bce7d8f80430002b27ddd8f82b
:107fe00000404ff01c0808fb03483d680c35444531
:107ff0001dd0142021f08cfc286000288fd0142282
:108000000021bcf0e6ff2b68039304f1100393e812
:1080100007008de8070094e80f00fff74dff0028e8
:1080200004f11c04fff67caf2d681035dfe7707893
:1080300000283ff475af3b681033039306f110033b
:1080400093e807008de8070096e80f00fff734ff7c
:1080500000eae07064e7024862e700bffcfeffff51
:10806000f2feffff70b50446006918b1bcf064ff72
:1080700000232361a5686db1286808b1bcf05cffde
:10808000686808b1bcf058ff2e692846bcf054ff60
:108090003546f0e7e4686cb1206808b1bcf04cffed
:1080a000606808b1bcf048ff25692046bcf044ff79
:1080b0002c46f0e770bd10b5044688b1c06818b111
:1080c000bcf03aff0023e360606818b1fff7caff15
:1080d00000236360a06818b1fff7c4ff0023a3600a
:1080e00010bd08b504f040fd05f094f904f03cfd26
:1080f000bde808400722002105f02ebd042810b578
:108100001bd005282dd1184c7e2200212046bcf022
:1081100060ff4ff0ff33c4f87e30a4f88230c4f81b
:108120005730a4f85b306ff07b03237000232046a8
:1081300063701ff031fc204610bd0c4c572200210b
:108140002046bcf046ff4ff0ff330021c4f8573003
:10815000a4f85b305d2320462370617019f019fb91
:10816000e9e70020e8e700bf31d20010b5d20010e7
:1081700073b50d46d8b911f0ff0506d104f0f4fc33
:1081800002b0bde8704004f0d9bf012d06d104f063
:10819000ebfc02b0bde8704004f018bd022d34d1f4
:1081a00004f0e2fc02b0bde8704004f016bd01a985
:1081b000c0b234f07ffa30bb04f0d6fc019904f071
:1081c00047fe0446f8b104f0cffc019904f08cfea0
:1081d000064604f0c9fc019904f08efe15f0ff0577
:1081e00006d1022e01d002280dd1204602b070bd6a
:1081f000012d04d1022e14bf00240124f5e7022d25
:1082000001d10228f7e70024efe70446ede713b5b4
:1082100030b904f0a9fc02b0bde8104004f084bffe
:108220006946c0b234f046fa68b9019001a90098d5
:1082300034f002fb002806db019800f04100012821
:1082400001d102b010bd0020fbe70020704713b53c
:10825000044638b904f088fc214602b0bde810405d
:1082600004f0d9bd01a9c0b234f024fa30b904f049
:108270007bfc019904f0cffd02b010bd0020fbe7ac
:1082800013b5044638b904f06ffc214602b0bde8ce
:10829000104004f0cebd01a9c0b234f00bfa30b9e1
:1082a00004f062fc019904f0c4fd02b010bd01208d
:1082b000fbe713b5044638b904f056fc214602b07a
:1082c000bde8104004f0febc01a9c0b234f0f2f9e0
:1082d00030b904f049fc019904f0f4fc02b010bd7f
:1082e0000020fbe713b50c4650b101a9c0b234f031
:1082f000e1f938b904f038fc2246019905f03efb5b
:1083000002b010bd6ff0a900fae770470020704777
:1083100008b507f005fcbde8084007f005bc000003
:1083200007b50c4b5b68cde90012c3f3080343b9f2
:1083300007f0f6fbdde9001203b05df804eb07f08f
:1083400039bd07f0edfbdde9001203b05df804eb89
:1083500007f014bc00ed00e010b5052886b011d17f
:10836000104605921ff07efa059b044638b9cde908
:1083700001000090012210200021fff711f9204692
:1083800006b010bd004cfae7f2feffff13b504463d
:1083900048b904f0e9fb214606f0b4f8b0fa80f0e1
:1083a000400902b010bd01a9c0b234f083f940b950
:1083b00004f0dafb019906f0a5f8003818bf012097
:1083c000efe70020ede74ff0ff3070474ff0ff3050
:1083d000704708b507f0a4fbbde8084007f0a8bb4c
:1083e0007047f8b50e46044660b100251827ae4226
:1083f00005d007fb0540fff75efe0135f7e7204695
:10840000bcf09afd0020f8bd7fb5104e044696f8ea
:108410006c300d4693b1706e2bf061ff70b90c4b50
:10842000694603930b4b30460293cde90045fef7b6
:10843000f5fb6846fbf738f904b070bd2046e9b299
:1084400004b0bde87040fff745bc00bf78ce001017
:10845000dd7c0002bb7b000237b504460068a8b98a
:1084600000220121174b10461a70174b1970032177
:10847000fff7caff04f078fb04f0f4ff6368db0742
:108480001dd503b0bde8304006f048bd00220321f1
:10849000fff7baff207801a934f00cf9054628b996
:1084a00004f062fb2a46019905f00afa2368002bc2
:1084b000d6d004f059fb04f006fd0028d0d003b05c
:1084c00030bd00bf2fd200102ed2001030b5174d96
:1084d000044695f86c3085b08bb1686e2bf0fffeca
:1084e00068b9134b28460393124b694600940293d4
:1084f000fef794fb6846fbf7d7f805b030bd54b1e2
:108500006946e0b234f0d6f828b904f02dfb012218
:10851000009905f0d5f904f027fb04f095ff01223e
:10852000054b1a700022054b1a70e6e778ce001052
:10853000157c0002a77b00022fd200102ed2001063
:108540007fb5234e044696f86c300d4693b1706e9d
:108550002bf0c5fe70b91f4b304603931e4b694686
:10856000cde900450293fef759fb6846fbf79cf8fe
:1085700004b070bda4b900220121184b10461a7036
:10858000174b19700321fff73fff04f0edfa04f0d9
:1085900069ffeb07ecd504b0bde8704006f0bebc47
:1085a000204600220321fff72fffe0b2694634f096
:1085b00081f8044628b904f0d7fa2246009905f05c
:1085c0007ff904f0d1fa04f07efc0028d3d0cfe785
:1085d00078ce0010d98300028d7b00022fd20010cc
:1085e0002ed2001070b52a4b0c465b6886b0c3f3e0
:1085f0000803002b39d1274e96f86c30b3b1706e5a
:108600002bf06dfe054688b9234b30460593234b6e
:1086100002a902940493fbf74bf90446c8b9054636
:1086200002a8fbf741f8284606b070bd14f001011e
:10863000019107d107f074fa019906b0bde87040c6
:1086400007f024bb07f06cfa06b0bde8704007f0f5
:1086500079bb2a464ff0ff3140692bf073ff236846
:1086600020469b68a5699847dae711f0010201925c
:1086700008d107f055fa0121019a06b0bde8704013
:1086800007f07cba07f04cfa00220221f5e700bfa0
:1086900000ed00e078ce0010e97b0002797b00025b
:1086a0007fb5174b04465b680d46c3f308031646b7
:1086b000ebb9144b93f86c20cab1586e2bf00ffe37
:1086c000a8b902900c2021f023f910b1c0e90045af
:1086d00086600d4b694603930c4b0090094802934a
:1086e000fef79cfa6846faf7dfff04b070bd324629
:1086f0002946204604b0bde87040fff773bf00bfb5
:1087000000ed00e078ce0010b9880002397b00024d
:1087100037b50122244b05681a700022234b1a70ca
:10872000234bc3e88f2ffff719fa044638b1002214
:108730001146104603b0bde83040fff7b1bf04f06a
:1087400013fa214604f0befa0028f0d01db301a9a7
:10875000e8b233f0afff40b904f006fa019905f032
:10876000ebf904f001fa04f0f1fc04f0fdf904f077
:10877000d3fc18b904f0f8f904f066fe04f0f4f93b
:10878000002104f09ffa60b104f0eef903b0bde8f7
:10879000304004f079be04f0e7f9294605f0ccf941
:1087a000e3e703b030bd00bf2fd200102ed200107f
:1087b00030d2001030b5304d044695f86c3085b09d
:1087c0008bb1686e2bf08bfd68b92c4b2846039358
:1087d0002b4b694600940293fef720fa6846faf79d
:1087e00063ff05b030bd0122264b1a700022264bd4
:1087f0001a70264bc3e88f2ffff7b0f9054638b142
:1088000000221146104605b0bde83040fff748bfd2
:1088100004f0aaf9294604f055fa0028f0d024b350
:108820006946e0b233f046ff40b904f09df9009983
:1088300005f082f904f098f904f088fc04f094f94a
:1088400004f06afc18b904f08ff904f0fdfd04f09f
:108850008bf9002104f036fa0028c2d004f084f924
:1088600005b0bde8304004f00fbe04f07df92146ac
:1088700005f062f9e2e700bf78ce001091860002b1
:10888000d57b00022fd200102ed2001030d2001063
:1088900070b507f045f907f047f900283cd1224ea2
:1088a0003378ebb9214c2378d3b906f03dfb98b36c
:1088b0001f4bd3e88f3fdbb20bb1237863bb04f0cf
:1088c00053f904f03bfc38bb04f04ef904f02cfce7
:1088d000034608bbbde8704002460146fff76abf89
:1088e00004f042f904f02afcb8b100220f4c104603
:1088f00025782378edb2002b14bf07210621fff75e
:1089000083fd00231a4619461846fff719fe002377
:10891000084a33701360257070bd04f025f904f027
:1089200003fc0028e1d1f7e72dd200102ed2001071
:1089300030d2001080f6001003681868d3e90112e5
:10894000fff7aebe38b50d1e0446006805dd3c21bc
:108950006943bdf0bffa18b938bdbcf0edfa00208c
:108960002060a5600120f7e72de9f8430026c0e963
:1089700000668660884649680746b14220ddfff7f9
:10898000e1ffe8b1d8e900934ff03c0c0cfb039ced
:10899000d7f800e009eb0604a4450ed01eeb06054f
:1089a00009d00fcc0fc50fcc0fc50fcc0fc594e865
:1089b000070085e807003c36ece7d8f804307b6018
:1089c0003846bde8f88382b070b50c4604a981e84a
:1089d0000c00d0e90113994206461dda3c23726867
:1089e00003fb04f15a433468521a0c442146e01840
:1089f00004adbcf0d4fa0fcd0fc40fcd0fc40fcd12
:108a00000fc495e8070084e80700736801337360ba
:108a1000bde8704002b070470131fff793ff0028b6
:108a2000dcd1f5e738b50d1e0446006805dd1c21d4
:108a30006943bdf04ffa18b938bdbcf07dfa00208b
:108a40002060a5600120f7e72de9f8430026c0e982
:108a500000668660884649680746b1421eddfff71a
:108a6000e1ffd8b1d8e900934ff01c0c0cfb039c3c
:108a7000d7f800e009eb0604a4450cd01eeb060570
:108a80001cbf0fcc0fc506f11c061cbf94e80700e5
:108a900085e80700eee7d8f804307b603846bde88b
:108aa000f88300002de9f04f884616461c468fb02b
:108ab00020b9654c20460fb0bde8f08f0029f8d0f2
:108ac000002af6d004a9c0b233f0f4fd0028f0d19a
:108ad000cde90500079004f047f8189b049900932e
:108ae00005aa234605f098ff041ec0f2978032685d
:108af000069b15469a42a8bf1d462db91ab135608e
:108b00006ff0a9048ae01d46002d3560f8dd4ff0b6
:108b1000180909fb05f210460392bcf005fac8f8e3
:108b20000000002800f086800021039abcf051fa72
:108b300000277c2309fb07fad8f800b0059c1beb43
:108b40000a0603fb074465d0636833b9e36d23b9b4
:108b500004f12000fff71df910b9a369002b59d0cb
:108b6000236933b9a36e23b904f13c00fff711f96f
:108b700010b9e369002b4dd02bf80a90606f60b1fb
:108b8000bcf0d2f9f06000285ad0d4f874a0216f5c
:108b90005246bcf0f7f9a6f810a0214608a8fff746
:108ba000e3fed4f818a004f158010ba8fff74cff1e
:108bb000331d514604f12002009308a80babfff7c8
:108bc0009df982460b98bcf0b7f90898bcf0b4f94f
:108bd000baf1000f34db04f10c0108a8fff7c4fe62
:108be000d4f81ca004f164010ba8fff72dff06f1d7
:108bf000080304f13c025146009308a80babfff7b1
:108c00007df904460b98bcf097f90898bcf094f9ec
:108c1000002c15db0137bd428bd10024dde9055363
:108c20007c2606fb0356ae4206d02846fff730f9f5
:108c30007c35f8e7054cf1e70598bcf07df939e79c
:108c40003046fff738fae5e7f2fefffffcfeffffd4
:108c500082b070b50c4604a981e80c00d0e901137c
:108c60009942064619da1c23726803fb04f15a4341
:108c70003468521a0c442146e01804adbcf08ff958
:108c80000fcd0fc495e8070084e80700736801332f
:108c90007360bde8704002b070470131fff7c2fe5b
:108ca0000028e0d1f5e72de9f04f002504460f46f6
:108cb00000f12006c0e90055c0e90255c0e904559d
:108cc000c0e90655bbb0304604f13c08fff74af84e
:108cd0004046fff747f8c4e91655c4e91855c4e9fa
:108ce0001a55c4e91c55a567b7b1d7f80c90b9f16e
:108cf000000f0cd03d8a55b12846bcf015f930b1b3
:108d00002a4649462067a567bcf03cf965677b6841
:108d100033b9bb68002b7fd120463bb0bde8f08f54
:108d2000196951b135462ba82baefff723f80fceaa
:108d30000fc596e8070085e807007b681a79a261ed
:108d4000d3f80890b9f1000f3dd00df1380ad9f8e9
:108d500000105046fff70ef804add9f8041015a81e
:108d600015aefff707f80fce0fc596e8070085e8a8
:108d7000070011ab0fcb8de80f002bad9ae80e006a
:108d80001ca81caefff721f80fce0fc50fce0fc5e4
:108d90000fce0fc596e8070085e807006d462dae9b
:108da0000fce0fc50fce0fc50fce0fc533682046af
:108db0002b606168dde92b23fff705fed9f81090e1
:108dc000b9f1000fc3d17b68d3f80c90b9f1000f53
:108dd0009fd004f1580b0df1ac0ad9f800101ca873
:108de0002bad1caefef7c6ff0fce0fc596e80700f1
:108df00085e807006d462dae0fce0fc53368584687
:108e00002b60e16d9ae80c00fff722ffd9f8109073
:108e1000b9f1000fe1d17ce7196951b12ba82bad55
:108e2000fef7a8ff0fcda8e80f0095e8070088e837
:108e30000700bb681a79e261d3f80880b8f1000f27
:108e40003ed00df13809d8f800104846fef792ffe1
:108e500004add8f8041015a815aefef78bff0fcea1
:108e60000fc596e8070085e8070011ab0fcb8de82a
:108e70000f002bad99e80e001ca81caefef7a5ff55
:108e80000fce0fc50fce0fc50fce0fc596e807004a
:108e900085e807006d462dae0fce0fc50fce0fc56e
:108ea0000fce0fc5336804f10c002b602169dde99a
:108eb0002b23fff788fdd8f81080b8f1000fc2d13e
:108ec000bb68df68002f3ff427af04f164090df1a0
:108ed000ac0839681ca82bad1caefef74bff0fcebb
:108ee0000fc596e8070085e807006d462dae0fce4a
:108ef0000fc5336848462b60a16e98e80c00fff759
:108f0000a7fe3f69002fe4d106e7000070b50d46cb
:108f1000a0b018b90d4c204620b070bd6946c0b253
:108f200033f0c8fb0028f5d103f01efe0446009e76
:108f3000294601a8fff7b7fe3146204601aa05f0f1
:108f400051fa044601a8fef7a3ffe4e7f2feffff93
:108f500013b543690446cde9000300f1230190f8fd
:108f60002220094b64302bf0a3f920b10a20074ad4
:108f70000749f8f73df894f86c3013b92bf0b7f9be
:108f8000f9e702b010bd00bf658f000223a80202fe
:108f9000fdc50d02002313b50193036801a91b68e9
:108fa0009847044620b1019828b103681b68984788
:108fb000204602b010bd0446fae708b5012380f848
:108fc0006c30044620f030ffbcf0f4fe251d204636
:108fd000fff7e0ffe3680bb9bbf054fa28462369ba
:108fe0009847f4e708b5fff7e8ff000070b50546bd
:108ff0000c4616f01bf96b686bb19c600026a660ee
:109000006c6016f017f9054b586e30b13146bde86b
:1090100070402bf0abb92c60f0e770bd78ce00103b
:1090200038b50446006868b116f000f92568ab68e9
:109030002360236803b9636016f0fcf828466b6868
:109040009847012038bd704710b504460c2120f028
:1090500067fc204610bd436913b183690c30184783
:10906000704713b50021044608462bf051fa00233f
:10907000204601a901932bf0bbfa019c0cb10123fe
:109080002371002101202bf043fa2cb123682046e4
:109090009b6898470023237102b010bd08b5fdf707
:1090a0005bfa48b10ff0eefc002204210ff039f911
:1090b000bde808400ff0b2b86ff0d10008bd000065
:1090c00009490c2008b5bbf0d9f9014650b1074b4e
:1090d000036000238360064b4360bde808400548f9
:1090e000fff784bf08bd00bf1308100244c60d027d
:1090f000d99000024cf6001010b403685a689968c1
:10910000541001eb6200d20748bf0a591b685df892
:10911000044b48bfd3581847012a38b5044602d13a
:109120000b68236003e0022a03d0032a0dd000203d
:1091300038bd0c200d6820f0ebfb03460028f0d072
:1091400095e8070083e80700ebe700680028eed009
:109150000c2120f0e5fbeae708b510b103685b6875
:109160009847bde80840fff799bf07b5806830b160
:109170000023cde900131a4602212bf045fa03b073
:109180005df804fb38b5836804469bb16ff000417d
:10919000fff7ebff0021a0682bf031fa237903f0f1
:1091a000ff0513b12bf0a3f8f8e72946a0682bf0d0
:1091b00075faa56038bd000038b505460446054b74
:1091c00045f80c3bfff7deff2846faf76dfa20461c
:1091d00038bd00bf54c60d0210b50446fff7ecffc2
:1091e00020461c2120f09cfb204610bd10b50446f3
:1091f000064b03608068fff7c5ff237b23b1a0689f
:1092000010b103685b689847204610bd68c60d0220
:1092100010b50446fff7eaff2046102120f080fb3e
:10922000204610bd284b2de9f04103604ff0ff337d
:1092300006460d4688b04360002943d11c2020f02b
:1092400067fb0446002834d00c20d6f8048006952d
:1092500020f05efb18b11d4b8660c0e900351c4b49
:109260000490236000230df1080c04af97e803007d
:109270008ce803002371a36004f10c0292e8030060
:1092800087e803009ce8030082e80300114a069384
:109290006261a269414607920f4a04f10800a26187
:1092a000cde900330d4a23462bf090f93846faf702
:1092b000fbf9b5fa85f530466d09b460357308b031
:1092c000bde8f0810c46f4e768c60d02419000024b
:1092d00054c60d029990000279900002e38f0002bb
:1092e0006ff000418068fff740bf13b5846800212c
:1092f0002046fff73affa06840b100236ff000421c
:109300001946cde900231a462bf07ef902b010bdb4
:10931000f0b58368054698680e468bb0f0b1002121
:109320002bf0cbf9041e18bf0124ab689868b8b1c4
:1093300000226ff000474ff47a7303217343cde9a5
:1093400000722bf061f9034650b9a8686e60a4b9a9
:1093500039460bb0bde8f040fff707bf0446e4e72d
:1093600020220023cde90223094a32200092094934
:1093700002aaf9f791fa0bb0f0bd80680028fad084
:109380001a460121cde900732bf03ef9f3e700bf47
:1093900015c60d0260c30d02fff780be2de9f04f28
:1093a0000025b5b081460c4692460995002a78d032
:1093b0005378002b75d029462a221da81c95bbf096
:1093c00008fe08230c20cde90130cde90c550cad89
:1093d00000959af800102e2350461caa31f04cfe3e
:1093e000014600285dd1102218a8bbf0f2fd4c23e5
:1093f00014939af80130b9f1110f15930cbf0223a1
:1094000001232946169314aa09ab1ca8cdf85c9039
:1094100031f0f8fd002844d10125099b4bb92022e9
:10942000cde91c23a44a32200092a4491caaf9f7d2
:1094300033fa202100236ff0e508a14acde91c137f
:10944000009201209d4901951caaf9f725fadff841
:109450006cb2099c002c00f0aa81d4e90212606869
:1094600032f0fcfe00262023071ecde91c3680f2d8
:109470009880d4e90173e26807930692bbf07cfb05
:10948000079b0168069acde901738e4b0491039204
:1094900000935946334632201caaf9f7fdf9e469d6
:1094a000d8e7894b5a6822b19b6813b1022509930a
:1094b000b3e7002c73d025781db1012d35d00025e0
:1094c000abe71022294620a8bbf083fd02264c23df
:1094d000b9f1110fcde91c360cbf33460123d4f886
:1094e00002001e93cde91455cde91655cde90c5572
:1094f000cdf87c900a9534f0fff810230a9014aa56
:1095000030460aa934f0f4f8002886d00821b4f8cf
:1095100042306e4a0ca8bcf093fd09ab1caa0ca902
:1095200014a831f06ffd032577e71c2200210da858
:10953000bbf04ffd4823b9f1110f4ff000060c931b
:109540000cbf022301235c2231461da80aaf0e93f3
:10955000cdf83c901c96bbf03cfd60225c4b1ca9f6
:10956000a01ccde90a66fcf708f80821b4f84230df
:10957000564a3846bcf064fd2023cde914361cabb6
:109580000193544b28464d49009314aa3346029741
:10959000f9f782f9394609ab0caa1ca8c1e72546a0
:1095a0003be7e36859460493a3680120039363688b
:1095b0001caacde90173484b00933346f9f76cf9c7
:1095c0002a2231461da81c96bbf003fd60680228c4
:1095d00046d00a2850d020220023cde914231caa0b
:1095e000cde901723d4a594600921e20039614aa05
:1095f000f9f752f9b9f1110f76d1626800230a2afe
:1096000072d11c2219460ca8bbf0e3fc1c228df879
:1096100030206368022b8df8313032d00a2b30d0e5
:10962000012304220a9340f6ff71384600920aabe8
:1096300032f0dffd60b320230026cde91436bbf005
:109640009bfa03685946cde90173254b32200093fc
:1096500014aa3346f9f720f9384632f0f1fd1ee737
:109660002e2361691caa043134f042f863695888da
:1096700034f048f80646aee761692e231caa08318b
:10968000f2e741f2346034f03bf8adf83200c7e75e
:1096900006901c2238460ca932f06cfd069b18b3cc
:1096a0002022cde914230f4a59460092322014aaf1
:1096b000f9f7f2f8d0e700bf80c60d0260c30d02d3
:1096c000a3c60d02b4c60d024c510010d7f10d0215
:1096d00091bc000270c60d02f3c60d0224c70d0234
:1096e00049c70d027fc70d023846d4e9042132f084
:1096f000a9fd20238046149390b100231593bbf05d
:109700003bfa02681cabcde903622c4acde9017338
:10971000009200235946322014aaf9f7bdf89be7be
:109720001cabcde90173264b1590009325490346e8
:109730000396012014aaf9f7aff8b9f1110f224be3
:109740000ad1023d012d07d85968e26931b19a600a
:109750004ab90991c3f80480012505e0002afbd02d
:109760000999c3e9011245461f60baf1000f04d000
:10977000d4e904215046bbf005fc00260c960ca948
:109780006068fcf72df901220c996068fcf7d0f8ad
:10979000304605f0fbfb012808d130462af09dfd3c
:1097a0000a49149014aa384632f093fd15b109986d
:1097b00031f026fc404635b0bde8f08fa9c70d0258
:1097c000dfc70d0260c30d024c5100100873048006
:1097d00030b50a4601461148002300688db032f0ca
:1097e00039fd041e15dabbf0c7f9036800250c2b00
:1097f00012d02023cde90435bbf0bef90368084937
:10980000cde90143074b3220009304aa2b46f9f718
:1098100043f820460db030bd2c46fae74c510010fd
:1098200060c30d0203c80d0230b50a460146174851
:10983000082300688db032f009fd041e07dabbf082
:109840009bf903680b2b05d1bbf096f90024204649
:109850000db030bdbbf090f903680b2bf4d0bbf01a
:109860008bf903680c2befd020230025cde90435bc
:10987000bbf082f903680649cde90143054b32206c
:10988000009304aa2b46f9f707f8e0e74c510010c3
:1098900060c30d021cc80d0230b5144c89b023689a
:1098a000002b1fdbc20715d50121184632f064fcde
:1098b00080b923f0e0ff0546002220216846fff72b
:1098c000b3ff002806db23f0d6ff41f28732431bab
:1098d0009342f1d9206832f0b3fc4ff0ff3323609c
:1098e00009b030bd6ff0d100fae700bf4c51001055
:1098f00013b501a837f078fe002242f2107311462a
:1099000001a837f005ff044601a837f07efe204687
:1099100002b010bd6ff0770070470000014b18686f
:10992000c01770474c510010014b1868704700bfba
:109930004c51001010b50446503066f062fb04f143
:10994000440066f05efb2046f9f752fb2046bde876
:109950001040b0211ff0e4bf38b50446062066f081
:109960003ffb054668b1204666f046fb00222946cb
:10997000204666f099fb034628b1bde8384038f030
:10998000abba6ff07703184638bd08b566f0ccfb6c
:1099900018b1bde8084038f09fba08bd0022142174
:1099a000c0e90022c0e90222026101804261027620
:1099b0004276c2617047000010b50a4cd4e88f3f70
:1099c000db070cd4204622f099f940b10648fff796
:1099d000e5ff204622f0ccf90448bbf0acf8024881
:1099e00010bd00bf18d300101cd30010c19a000294
:1099f0002de9f047c469a0b0289f002c00f09480a6
:109a0000d4f8a0509d4211d39e18ae420ed9eb1a45
:109a1000761b3246194404f14400fbf7edfa0028a6
:109a200069dbd4f8a0303344c4f8a030d4f8a030b7
:109a3000bb4229d200217c2201a80091bbf0c9fac7
:109a400024f0fafcd4f8a030c61900eb030904f1a5
:109a50004408b14516d2a6eb090abaf1800f28bf17
:109a60004ff0800a69465246484624f017fd002808
:109a700041db524669464046fbf7befa00283adb16
:109a8000d144e6e7c4f8a070d4f8a030ab4229d99d
:109a900004f15006304604f1440166f0dffa30bbb1
:109aa000304604f17c0166f075fb18b138f014fa09
:109ab000002820db4822204604f15c01f9f792fbe4
:109ac000002818dbd4f8ac30ab4203d123f0d3fe2e
:109ad000c4f8a400d4f8a830d4f8a02013445d1b27
:109ae000c4f8a850d4f8a83043b9002003e038f0f7
:109af000f3f90028d4da20b0bde8f08723f0bbfeec
:109b0000d4f8a430c01a47f22f539842edd920461a
:109b1000f9f7def90028eedb23f0adfec4f8a4006f
:109b20000020c4f8a800e6e76ff0d100e3e710b525
:109b30000446006808b1fff7fdfe204610bd000096
:109b400008b50248fff7f3ff08bd00bf38d3001087
:109b50000368016013b11846fff7ecbe70470000c0
:109b600070b5c56906468ab03db3d5e927329a4239
:109b700026d1202205f15c0105f17c00bbf0f2f951
:109b8000044688b1002320220e4ccde90223322066
:109b90000d49009402aaf8f77ffe2046f8f792fbe1
:109ba0000a4c20460ab070bd2846f9f721fa214632
:109bb00006f11c00fff7ccfff3e76ff0d104f0e7ec
:109bc000034ceee740c80d0235c80d02cdfaffff89
:109bd000b9faffff10b50446c06992b040b1f9f779
:109be0001bfa002104f11c00fff7b2ff12b010bdf8
:109bf000054901a8f9f75cf901a8f9f70dfa01a8e0
:109c0000f9f7f6f9f2e700bf6fc80d0270b5037ef1
:109c100005468ab0c3b1c469b4b1d4f8a8309bb1c9
:109c200023f029fed4f8a430c01a47f22f539842eb
:109c30000ad92046f9f74cf900284ff0000605db59
:109c400023f019fec4e929060ab070bd2023cde92e
:109c50000236074b0190009332203346054902aa91
:109c6000f8f71afe28460ab0bde87040fff7b2bf09
:109c700080c80d0235c80d027fb5037e05460e462d
:109c80003bb31c300021fff763ff687e08b90df07d
:109c90009dfa0024104ba6421c7018bf01222b46cf
:109ca00008bf4ff0ff3200214ff48070cde901442e
:109cb0002c760094fdf774fc204605f0b1fe234697
:109cc000024600214ff48010cde901440094fdf7d5
:109cd00067fc04b070bd00bf5ed4001070b511f019
:109ce00008020546047e01f0040301f0010626d1b6
:109cf0008cb3e3b9c4691cb1fff732ff041e10db5b
:109d00007eb9002024f0fefb0446e1432846c90f3b
:109d1000fff7b2ff002c10db462005f069fd0024a0
:109d20000be02846fff756ff002ceedbe9e7422167
:109d3000012024f0b5fb00eae074204670bd002c41
:109d4000fbd0002bebd10eb1fff744ff00212846da
:109d5000fff792ffe3e76ff0d104eee72de9f04162
:109d60001f46037e0446884616468cb0002b56d00c
:109d700024f062fb0023c1193246404624f07efbea
:109d80000546d0b100262023264f04aacde904368b
:109d900025493346019000973220f8f77dfd29468a
:109da0003846f8f78ffa31462046fff765ff6ff027
:109db000da0528460cb0bde8f081e369bbb1129b1f
:109dc0003246009341463b462046fff711fe70b1f4
:109dd0002023cde90435154b0190009332202b460a
:109de000114904aaf8f758fd2046fff7f3fe637ef9
:109df00013b9e720f7f768fa236902223b4463604e
:109e000000234ff480700021cde9013300932681b7
:109e10002346fdf7c5fb23f02efd6061c9e76ff017
:109e2000d105c6e7a4c80d0235c80d0280c80d02d1
:109e30002de9f04fa5b001908846b020664916463e
:109e4000baf01cfb044698b100256449f9f730f8d4
:109e500048222946c4e91155c4e91355c4e91555ea
:109e600004f15c00bbf0b5f8c4e92955c4f8ac5066
:109e70000394002c00f0ad8004f14400fff76cfd6a
:109e8000041ec0f2968003985030fff765fd041e53
:109e9000c0f28f80039d482205f15c0739462846b1
:109ea000f9f722f94828044640f08a80d5f89c301a
:109eb000434552d1d5f8a03043454ed820223146f3
:109ec0003846bbf04ff88246002846d1039844300c
:109ed000fff75bfd041e6cdb51467c2205a8cdf824
:109ee00010a0bbf076f824f0a7fa8346d5f8a0308e
:109ef00000eb030ad34517d2aaeb0b09b9f1800f87
:109f000028bf4ff0800958464a4604a924f0c6faf3
:109f1000041e4edb03984a4604a94430fbf76cf854
:109f2000041e46dbcb44e5e7039800f144015030c2
:109f300066f094f8002838d1039804a9503066f0f0
:109f400029f918b137f0c8ff041e32db202204a91a
:109f500005f17c00bbf006f8d8b10398f9f75cf87e
:109f600006f1200356f8042b9e4247f8042bf9d142
:109f70002022002105f17c00bbf02bf80023039880
:109f8000c5f89c80c5f8a0304430fff7fefc041ee5
:109f90000fdb00240399d5f8a0300198c1f8ac304c
:109fa0001c300394fff7d4fd03e037f095ff041e47
:109fb000c2da03a8fff7bbfd204625b0bde8f08f4d
:109fc0000028cada10f1aa0fc7d010f58c7ff0d1a3
:109fd000c3e7034cede700bf130810026fc80d0282
:109fe000fcfeffff2de9f0478cb0149d04460f46a0
:109ff0001e46904605f0040905f0010abab1b3b156
:10a00000c5f34005227ea2b1002320216b4ccde98f
:10a01000041332206a4904aa0094f8f73dfc204654
:10a02000f8f750f96ff0d1000cb0bde8f0870125ca
:10a03000e8e7012004a98df8102005f03ffb9df80a
:10a04000102012b16fb95f48eee7092004a98df81e
:10a05000102005f033fb9df81030002bf2d15a4848
:10a06000e2e724f0eff9b842edd3baf1000f1bd1cb
:10a07000d5b9424639462046fff7dafe002877da9e
:10a0800020220023cde90423504a0190009232207f
:10a090004b4904aaf8f700fcb9f1000f40f08780a3
:10a0a0002046fff797fd07e0b9f1000f7ad120466f
:10a0b000fff790fd002ddcd024f0bef939460022d8
:10a0c00024f0caf9014600285ed04ff000080022b3
:10a0d0001146104605f0dafaf7f78cf90546607676
:10a0e00058b901200df072f829460b20fcf7c6ff85
:10a0f000002850d000690df08cf801230025344a67
:10a10000237613701423a446cde90455cde90755f1
:10a110000695adf810300df1100ebee80f00ace85a
:10a120000f00ccf80050e76024f086f9206124f09d
:10a130008ff92369208163602a4623460021a57296
:10a140004ff48070cde901550095fdf729fa2846b6
:10a1500005f066fc2b46024600214ff48010cde945
:10a1600001550095fdf71cfa23f085fb606120e0a6
:10a17000e369d3f8a080b9f1000f0fd0002104f1fa
:10a180001c00fff7e5fc14e004f11c00fff7e0fc05
:10a190006ff0da0048e74ff0ff10ace7b8f1000fbe
:10a1a00095d189e71db9baf1000f3ff462af4ff0c6
:10a1b00000080eb1c6f80080002035e7c5c80d02c2
:10a1c00035c80d02b9faffff9cfaffffecc80d027b
:10a1d0005ed4001048b10138222896bf052307231a
:10a1e000b0fbf3f34ff47a709840704708b580b134
:10a1f00003881b2b0dd94ff0ff33037102234371ea
:10a200000323837105231422c37103490830bcf072
:10a2100033fd1c2008bd00bfd4bd0d0210b504469f
:10a22000007c10b1d4e902309847207410bd036857
:10a2300002224068184770470eb4f0b5002692b06d
:10a2400017ad55f8047b3c223146044603a802961c
:10a25000baf0bffe3a462b46402102a80195bdf058
:10a2600013f93f28024605dd267412b0bde8f04020
:10a2700003b07047204602a9fff7d0fff5e710b5fd
:10a28000044614211ff04cfb204610bd13b50446b4
:10a2900008460191f6f7eefd02462046019902b00c
:10a2a000bde810400cf06ab937b56fea41416fea7a
:10a2b0005141adf8041001a904461546fff7b7ff58
:10a2c00030b104222368606801950deb02019847c4
:10a2d00003b030bd7fb50e461546044608b103698c
:10a2e00023b90a20094a0a49f6f782fe0c23cde970
:10a2f00001362b68012103932046236901aa984760
:10a3000008b9039b2b6004b070bd00bf23a80202f4
:10a310001fc90d0237b5c3880446012b0d4604d072
:10a320000a20074a0749f6f763fe04232946204618
:10a330000deb03020193fff7cdff03b030bd00bf6b
:10a3400023a8020245c90d0237b5c3880446022b73
:10a350000d4604d00a20074a0749f6f749fe0423b0
:10a36000294620460deb03020193fff7b3ff03b02c
:10a3700030bd00bf23a8020271c90d0273b5cb889e
:10a380000546012b0c4605d0022b17d06ff0770045
:10a3900002b070bd0023694620460093fff7baff64
:10a3a0000246f0b9a388286801a9009eadf80430e0
:10a3b000fff73dff48b96ff0bd00e9e700236946ac
:10a3c00020460093fff7c0ffeae704222b680196be
:10a3d0001c6858680deb0201a0470028ebd0002054
:10a3e000d6e7a1882868fff75ffff6e70b4601462e
:10a3f0001846fff7c3bf13b5044608460191f6f7a8
:10a4000039fd02462046019902b0bde810400cf02b
:10a41000a5b8000038b5044615460068fff7ebff05
:10a4200020680bf0e9ff06492068fff7e4ff2946a2
:10a430000bf0eeff20680bf0bdff2368187c38bde1
:10a440006ecf0d0273b5054688680c4630b1cb88d7
:10a45000012b05d0022b19d06ff0770002b070bd30
:10a460000023204601a90193fff754ff0246f0b9eb
:10a47000019ea1682868fff7beff31460bf0ecff94
:10a480002b681b7ccbb96ff0bd00e7e700232046ab
:10a4900001a90193fff758ff024640b9019ea16848
:10a4a0002868fff7a8ff31460bf0e8ffe8e72846e9
:10a4b000a168fff7afff0028e5d00020cee70b46ec
:10a4c00001461846fff7bebf2de9f04f9a4b99b0f1
:10a4d0001546039300240123cde90501974903a8fc
:10a4e0008df81c308df81040fff785ff69880bf060
:10a4f0008fff24272b8aa3420dd907fb04f6eb68b4
:10a5000003a89959fff777ffe96801343144043112
:10a51000fff7bcfeeee78a4903a8fff76cff03a82c
:10a520000bf05eff4ff00008dff848922b8943459f
:10a5300040f2f980782606fb08f6d5f804b00beb5c
:10a54000060494f82230052b00f2d280002b00f094
:10a55000d380a37b012b04d1b4f870309b0740f16a
:10a56000cb8004f114073846f6f7b6fc824603a800
:10a570000bf042ff734903a8fff73dff5bf806109d
:10a580000bf07cff704903a8fff735ffa37b032b7b
:10a5900096bf6e4a6e4952f82310fff777fe6d4959
:10a5a00003a8fff728ffb4f86e100bf031ff6a49db
:10a5b00003a8fff720ffb4f870100bf029ffbaf1e1
:10a5c000050f2ed100213c2209a80891baf001fd07
:10a5d000624903a8fff70fff04f16c0604f14c0376
:10a5e00008aa13f8011b0232090901f1300cbcf171
:10a5f000390f88bf01f1370c02f802cc13f8011ca7
:10a6000001f00f0101f1300cbcf1390f88bf01f1ed
:10a61000370c9e4202f801cce3d1402208a90bf08e
:10a62000adff4f4903a8fff7e6fe06463846f6f7aa
:10a6300053fc082898bf59f8201030464ff0000608
:10a6400088bf4349fff722fe38460896f6f747fcd5
:10a65000444a0346042108a8bbf0f2fc424903a87f
:10a66000fff7c9fe08a9fff711fe404903a8fff74d
:10a67000c2fe82463846f6f737fc014650460bf0dc
:10a68000c7fe3b4903a8fff7b6fe03a80bf0a8fee0
:10a69000dff8ccb094f8247094f82530b4f826a0f4
:10a6a000052f34d8002f35d003a801930bf0a4fe5a
:10a6b000594603a8fff79ffe59f82710fff7e6fd5c
:10a6c000019b284a042108a8bbf0bafc264903a82c
:10a6d000fff791fe08a9fff7d9fd244903a8fff76a
:10a6e0008afe51460bf094fe03a80bf063fe11e0c6
:10a6f000073b012b7ff62daf08f1010816e7012675
:10a7000094f8287094f82930b4f82aa0c8e7f91f03
:10a710000129c9d9002ef2d003a80bf042fe03a8ec
:10a720000bf048fee8e703a80bf03bfe9df81c0089
:10a7300019b0bde8f08f00bf00ca0d02490f10022a
:10a7400042ba0d0243ce0d029a1b0e02e8c90d0259
:10a75000e4530e0261750e029ec90d02d8f10d027e
:10a76000480d1002d7f10d025c101002276e0e0288
:10a77000e4cc0d02c4c90d0218b10022012123f05e
:10a780006bbd0148704700bff2feffff18b1002209
:10a79000114623f061bd0148704700bff2feffff84
:10a7a00030b587b004460d461222002101a8baf048
:10a7b00010fc14230022adf804300123114601a837
:10a7c000adf81630fff7d8ff294601aa2046fff75b
:10a7d0007bfe0446002101a8fff7d8ff204607b002
:10a7e00030bd000003681f221b680149184700bfe5
:10a7f000a1c90d02f0b512f0010489b00e4605465c
:10a800000e9933d0cde9033103ab0193022302a9a2
:10a8100003a8adf80830fff70afd10b96ff0bd00ce
:10a8200022e00423019802a9adf80830fff7fffced
:10a830000028f3d095b100242746a64233d0002249
:10a8400035f8140002a90297f8f706fb60b90299df
:10a8500001a8fff793fd38b90134eee72b462946ee
:10a860001f4801aaf8f7d4fa09b0f0bdcde90531c7
:10a870001c4b8df81040039301238df81c3003ab63
:10a88000184601930bf0b8fd019b1b7c002bc5d033
:10a89000e5b12746a64208d101980bf08bfd019b3c
:10a8a0001b7c002bbad00020dee7002235f8140014
:10a8b00002a90297f8f7d0fa0028d5d1029901a889
:10a8c000fff7c0fd0028cfd10134e3e72b4629462e
:10a8d000054801aaf8f79cfa0028ddd0c4e700bfbc
:10a8e0006da3000200ca0d023fa4000213b50024ac
:10a8f0000346cde9001420462146fff77bffb0fa5e
:10a9000080f0400902b010bd70b5264b88b000241d
:10a9100003930123cde90501234903a88df81c30d9
:10a920008df81040fff767fd0bf05afd00f00cffab
:10a9300026460546ac420ed0204602a9029600f0fb
:10a9400009ff10b1002008b070bd029903a8fff7fd
:10a950009dfc0134eee703a80bf023fd134903a887
:10a96000fff749fd0bf048fd002400f0cdfe264620
:10a970000546ac4211d0204602aa01a9cde90166e4
:10a9800000f0c8fe0028ddd1019903a8fff733fdd0
:10a9900002990bf03dfd0134ebe703a80bf00afd33
:10a9a0000120d0e700ca0d02480d1002276e0e02ea
:10a9b00070470368c1f8d030d1f8e03043f00403a9
:10a9c000c1f8e03070470368c1f8dc30d1f8e030fe
:10a9d00043f00803c1f8e03070470368a1f8e8309d
:10a9e000d1f8e03043f01003c1f8e030704703685d
:10a9f000a1f8ea30d1f8e03043f02003c1f8e030ac
:10aa000070470368c1f8e430d1f8e03043f0400308
:10aa1000c1f8e03070470368a1f8ec30d1f8e030bd
:10aa200043f08003c1f8e0307047002381f8e03044
:10aa300081f8e13081f8e23081f8e33070470000be
:10aa4000f0b404460f46bab90388b3f5837f0cd13e
:10aa50000b4e051d06f12002334603cb93422860be
:10aa600069601e4605f10805f6d100233a462146e5
:10aa7000f0bc184614f098bf4ff0ff30f0bc7047a0
:10aa800050ce00101fb500240a460094014603abc7
:10aa90002046039414f098ff00b10394039804b087
:10aaa00010bd10b5002488b02146cde9040404a8e7
:10aab000cde9064423f02af8234601224ff48040d2
:10aac0000021cde901440094fcf76afd08b010bdf7
:10aad000f7b50d4616461f460446fef76dff334692
:10aae0002a4621460097fff739f903b0f0bd07b5b4
:10aaf0000190fef761ff019903b05df804ebfff7e9
:10ab0000edb8f7b50d4616461f460446fef754ff4e
:10ab100033462a4621460097fff764fa03b0f0bd9a
:10ab20001830036800200b6070471830036800205d
:10ab30000b60704700b50b4a8bb0137873b10121dd
:10ab4000094b1e201970002313702022cde9022327
:10ab5000064a0749009202aaf7f79efe0bb05df87d
:10ab600004fb00bf5cd400105bd4001010ca0d02bf
:10ab700060c30d0208b510b103685b689847bde873
:10ab80000840fcf76ebd13b504460191f6f772f963
:10ab90000199a0f1180204f11800bcf059f8b0fabc
:10aba00080f0400902b010bdf0b58db005460c46ee
:10abb000f6f760f9172842d9182228466749bcf0f1
:10abc00047f8074600283ad12046f6f753f964497a
:10abd00002462046bcf03cf86249b0fa80f62846ae
:10abe000fff7d1ff7609044638b13a4631460920cd
:10abf0000db0bde8f04004f049bd28465a49fff7c2
:10ac0000c2ffd0b1204604f00bff0122574b05468e
:10ac10001a7031462246204604f038fd204604f0e2
:10ac2000fffe8542024608d023464ff480100021e3
:10ac3000cde901440094fcf7b3fc0db0f0bd132244
:10ac400028464b49bcf004f8064680b92023cde9dc
:10ac50000430484b4849009304aa03460120f7f703
:10ac60001bfe30460db0bde8f04023f0d5bd2846b0
:10ac70004249f6f7f5f8002846d1002cddd02378bc
:10ac8000002bdad021463e48f6f7eaf820b90db09d
:10ac9000bde8f0400cf0f9bd21463a48f6f7e0f87f
:10aca00020b90db0bde8f0400cf0d4bd21463648c7
:10acb000f6f7d6f820b90db0bde8f0400cf0e2bdd3
:10acc00021463248f6f7ccf804460028b5d12023b7
:10acd000cde904302e4b2849009304aa03462820ce
:10ace000f7f7dafd2b490c20b9f0c8fb0146002824
:10acf000a3d0294b84600360284b436028480db0e3
:10ad0000bde8f040fef772b9182228462549bbf08d
:10ad10009fff0446002890d12025234b164904aa02
:10ad2000cde90450009303462820f7f7b5fdfaf764
:10ad300051fafaf745fb00280ada1c4b0190009300
:10ad4000322023460c4904aacde90454f7f7a4fda8
:10ad500096200db0bde8f04004f04abda3d00d022e
:10ad60003bca0d0283d00d02bcd00d025fd400108f
:10ad70006fd00d0240ca0d0260c30d025cd00d02ff
:10ad800076ca0d0280ca0d0284ca0d02abca0d023a
:10ad90008bca0d021308100244c60d02f5aa000268
:10ada0004cf600108ad00d02b3ca0d02ceca0d02b5
:10adb000f7b50646184fd7e88f5f15f0010522d189
:10adc000384620f09bfff0b12a4614210f20fcf7f3
:10add0005ff91e220221114c0346cde900212046d5
:10ade0000f226ff07f410cf073fd0d4b384623604e
:10adf0000c4b84f8225063616423238420f0b8ff55
:10ae00000948b9f098fe00223146084803b0bde871
:10ae1000f040f7f725be00bf3cd3001004d400106b
:10ae2000ccd00d02ee82ee0029b0000208d4001052
:10ae3000012a38b5044602d10b68236003e0022ad8
:10ae400003d0032a0dd0002038bd0c200d681ef061
:10ae50005ffd03460028f0d095e8070083e807006f
:10ae6000ebe700680028eed00c211ef059fdeae760
:10ae7000012af8b5064603d10b6803600020f8bd2f
:10ae8000022a08d0032af9d100680028f6d0182138
:10ae90001ef046fdf2e718200c681ef039fd07464b
:10aea00030b105460fcc0fc594e8030085e80300d8
:10aeb0003760e3e7012a08bf016000207047012adc
:10aec00002d1016000207047022a04bf0b680360b2
:10aed000f8e7012a02d1016000207047022a04bf6e
:10aee0000b680360f8e7012a02d101600020704777
:10aef000022a04bf0b680360f8e7012a02d101604f
:10af000000207047022a04bf0b680360f8e7012a9b
:10af100002d1016000207047022a04bf0b68036061
:10af2000f8e7012a02d1016000207047022a04bf1d
:10af30000b680360f8e7012a08bf01600020704732
:10af4000012a08bf016000207047037b33b9d0e9b4
:10af50000121036809681b68106818477047012ab7
:10af600070b5054603d10b680360002070bd022a4e
:10af700011d0032af9d10468002cf6d004f118008e
:10af80000cf02efb04f108000cf02afb2c212046cb
:10af90001ef0c6fce9e72c200e681ef0b9fc044642
:10afa00088b1338806f1080103807368083040f8df
:10afb000043c0cf0abfb06f1180104f118000cf096
:10afc000a5fbb36aa3622c60cfe770b58568044621
:10afd000681c1668b9f0a8ff306048b100224255dd
:10afe00075602a4620463168bde8704037f0e0bc05
:10aff00070bd134682681ab11b684168c3e900122c
:10b00000002137f0d5bc002307b5009342f00103bf
:10b010003c22fbf78dfe03b05df804fb10b58ab04f
:10b0200003f0a8ff042813d100242023cde9023423
:10b03000084b02aa00931e2023460749f7f72cfc71
:10b040002246064906480ab0bde81040fff7dbbfbc
:10b050000ab010bdfcca0d0260c30d02c3c30e02cc
:10b0600014cb0d02002210b50446044b114640f8e3
:10b07000043bf7f7f5fc204610bd00bfd4cf0d020e
:10b0800010b50446fff7eeff204620211ef048fcd5
:10b09000204610bd10b50446024b0360fff7e2ffe7
:10b0a000204610bdccd00d020148fff7f3bf00bf12
:10b0b00004d4001010b50446fff7ecff204624210d
:10b0c0001ef02efc204610bd038c8b4211d890f848
:10b0d00022300133dbb2072b08bf002380f8223077
:10b0e00090f82220044b53f82230436164230384f8
:10b0f00070475b1afbe700bf40d00d02f0b5a5b06a
:10b10000cde9023205460f46f7f7f8f86ff0630312
:10b110000024049303ab0b9304ab0c93204602abc7
:10b120000d938df83840f6f7aff9064630b9554b18
:10b1300004930ba8fff709ff25b0f0bd23463a465c
:10b140002946f6f7c1f938b96ff0f90304930021e5
:10b150003046f6f79df9ece705ab16934a4b09aa82
:10b16000159307ab1993494b3046cde91a3248493c
:10b1700015aacde90544cde90744cde90944179462
:10b18000189338f0ecf80546a8b92023414ccde9d6
:10b190001c30414903461caa32200094f7f77cfb7f
:10b1a0002046f7f78ff83d4b04930598b9f0c4fe9d
:10b1b000002dbed1cbe721463046f6f769f9059b55
:10b1c0000f93179badf84830079b1093089b119382
:10b1d000099b13930a9b1493f9f7fcff0fa9f9f746
:10b1e0005bff051e12da20232d4f3220cde91c34df
:10b1f0002949234601951caa0097f7f74dfb2946dc
:10b200003846f7f75ff804950125cee7039b204603
:10b21000029998470122234b8df83820d3e8cf4f6d
:10b22000c3e8412f0029f9d1e4b2002cf6d1052260
:10b23000c3e9032440f201129a820022c3e88f2f4f
:10b240000821234622460120009406f0c9fbf9f7a5
:10b25000c1ff0fa9faf79cf800280bda2023cde9eb
:10b260001c34114b01900093322023460a491caa3a
:10b27000f7f712fb962004f0bbfa0598b9f05cfed4
:10b2800057e700bffcfeffff4baf000273af0002a9
:10b2900084680e022acb0d0260c30d02e8feffff98
:10b2a0004ecb0d02d4d3001079cb0d0207b5006848
:10b2b0000369019302238df8033083680bb9b9f059
:10b2c000e1f8c3680df1030201a9984703b05df8e6
:10b2d00004fb000070b500242026144b8ab0144de6
:10b2e0001e201449009302aa2346cde90264f7f711
:10b2f000d3fa2246022128680df013f8044620b143
:10b300000ab0bde870400cf089bf0b4bcde902607c
:10b31000009302aa034607491e20f7f7bdfa2868e2
:10b3200021460df02ff920460ab070bd9ecb0d02cc
:10b330002cd4001060c30d02bbcb0d0230b500242d
:10b340008bb0234622460f49cde900440e48fbf757
:10b3500005fb234605462246cde9004409490b4832
:10b36000fbf7fcfa00b155b920220023cde90223f6
:10b37000074a32200092074902aaf7f78dfa0bb06c
:10b3800030bd00bf29ab0002d1cb0d02dacb0d02dc
:10b39000e0cb0d0260c30d022de9f043adf23c4d50
:10b3a00002aff9f717ff0646faf72ef810f5e16f2e
:10b3b00007f5e67440f0078100254ff02008994b0f
:10b3c00022463220c4e90085974900932b46f7f7bf
:10b3d00063fa964a3046136843f00a031360f9f79c
:10b3e000efff00280ada924bc4e9008500932b4650
:10b3f0000190224632208c49f7f74efa08238d4ef1
:10b400000022394630683b800df0c9f803f0b2fde8
:10b41000042800f0e3807988002026f05efb0120fc
:10b42000b98826f05afb032014f09af94ff03c0833
:10b4300005464246002107f12800b9f0cafd002d5b
:10b4400014bf02230123a7f8288087f82a3000f0d0
:10b45000e380794bfb62794b3b63794b3b65794bde
:10b460007b65794bbb65794b1c227b63784b002154
:10b47000bb63784b07f16800fb63774b07f1a409c6
:10b480003b64764b4ff001087b64754b07f1640514
:10b49000bb64744bfb64744bfb65744b3b66b9f047
:10b4a00098fd40237b66724b4ff493723b67714b60
:10b4b000ff21c7f89c30704b4846c7f884306f4b6b
:10b4c000c7f888306e4bc7f88c306e4bc7f8a03089
:10b4d0006d4bc7f898306d4bc7f890306c4bc7f880
:10b4e0009430b9f076fd4ff41972ff212046b9f07f
:10b4f00070fd10233b8308232046f918bb60c7e981
:10b50000074987f80c8023f041f9484623f028f9d1
:10b51000002108461df042fe0024c1b2cb1d03f4f9
:10b52000fc73adeb030d0df1080948461df036fe26
:10b53000cde900544946306807f1280307f11802a5
:10b540000cf0d2fe009423462246022130680df012
:10b550002ef829f0dbf8b0f57a7f06d30094234665
:10b560004246032130680df022f80024009423465f
:10b5700041f2b642042130680df019f8356822f026
:10b5800061ff234602460521284600940df00ff87e
:10b59000356822f05dff23460246062128460094c6
:10b5a0000df005f808233b823a4b07f110011b68a8
:10b5b00030687b610cf092fefff7c0fe07f2344763
:10b5c000bd46bde8f0830028bff618af2022002357
:10b5d000c4e90023304a019000920ae7002026f0d7
:10b5e0007ffa7880012026f07bfa4ff6ff73798886
:10b5f000b880994204d0002330681a460cf0cbff83
:10b600004ff6ff73b98899423ff40daf00233068bd
:10b610001a460cf0c2ff06e7204bfb62204b3b634f
:10b6200021e700bffccb0d0260c30d0244d3001024
:10b63000ceca0d022cd400104558000295580002c5
:10b6400050ce0010c1a9000205aa000283aa000280
:10b650006faa000251aa0002b5f5010231ad000245
:10b66000f7d7020223aa0002b5aa00027db00002a9
:10b67000e9c60002f1c40002d9e60202dde60202d8
:10b6800021a7000289a800026da8000269c2000279
:10b690007dbb000228d400102ccc0d02f95700020b
:10b6a0004958000210b500232024144accb01e20b3
:10b6b000134900920aaacde90a43f7f7edf80023ef
:10b6c0004ff4837219460aa8b9f083fc00234ff4a3
:10b6d00083711a460aa8fff7b3f900284ff0000358
:10b6e00009da084a019000923220054902aacde900
:10b6f0000243f7f7d1f84cb010bd00bf53cc0d0298
:10b7000060c30d0269cc0d02014b5868704700bf41
:10b71000ecd3001010b50a4b5c6884420bd950245e
:10b720001b6804fb003009b1431d0b602ab103798b
:10b730000020136010bd0348fce71046fae700bf85
:10b74000ecd30010defeffff014b5868704700bfce
:10b75000f8d30010074b5a68824208d929b14c220d
:10b760001b6802fb00300830086000207047024868
:10b77000704700bff8d30010defeffff10b5044c89
:10b78000236813b90df07ef92060206810bd00bf5a
:10b790002cd40010f8b50b4b0546d3e900465023d6
:10b7a00003fb0646b442274609d0601d40222946c5
:10b7b000bbf04efa50340028f4d13846f8bd0027cb
:10b7c000fbe700bfecd300102de9f0410f46164611
:10b7d0001c46beb005464c22002103a8b9f0f9fb77
:10b7e00002978df80c6034b16368149323880b2b97
:10b7f00084bfa36815932846f5f73cfb4028024612
:10b80000294628bf40220df10d00b9f0bbfb2846a8
:10b81000fff7c0ff044638b1502202a9b9f0b2fbcd
:10b8200020463eb0bde8f081254d6e68632e41d8bc
:10b83000502402a9224616a8b9f0a4fb224616a954
:10b840002aa8b9f09ffbab689e4215db06fb0441ba
:10b850002868baf03ffb771c044658b92023cde98d
:10b860002a30184b00933220234617492aaaf7f7ab
:10b8700013f8d5e72860af604ff050086a6808fbfe
:10b8800006f608fb02f22f68921b3744394607eb95
:10b890000800b9f084fb424638462aa9b9f072fb89
:10b8a0006c6801346c6008fb04f4a4f150002c684f
:10b8b0000444b5e72023cde92a30044bd2e700bf8a
:10b8c000ecd30010a5b90d0260c30d0281cc0d02ae
:10b8d000f8b50b4b0546d3e900464c2303fb06465f
:10b8e000b44227460ad004f1080040222946bbf0a2
:10b8f000aff94c340028f3d13846f8bd0027fbe7f8
:10b90000f8d300102de9f0410d460446bcb04422a6
:10b91000002105a8b9f05dfbab6820460493eb68f5
:10b920000393f5f7a7fa40280246214628bf402294
:10b9300005a8b9f027fb2046fff7caff044638b137
:10b940004c2203a9b9f01efb20463cb0bde8f081b3
:10b95000254d6e68632e41d84c2403a9224616a8b3
:10b96000b9f010fb224616a929a8b9f00bfbab6869
:10b970009e4215db06fb04412868baf0abfa771c3f
:10b98000044658b92023cde92930184b00933220c2
:10b990002346174929aaf6f77fffd5e72860af604d
:10b9a0004ff04c086a6808fb06f608fb02f22f68a5
:10b9b000921b3744394607eb0800b9f0f0fa4246cb
:10b9c000384629a9b9f0defa6c6801346c6008fbce
:10b9d00004f4a4f14c002c680444b5e72023cde91d
:10b9e0002930044bd2e700bff8d30010a5b90d02ef
:10b9f00060c30d029acc0d0210b588b004466846ab
:10ba00000bf039fe694604a80bf080fe04a8a0479d
:10ba1000044604a80bf0e4fd68460bf0e1fd204667
:10ba200008b010bd10b50446f5f724fa01462046cb
:10ba3000bde8104013f0febd70b5094b0025d3e9f9
:10ba400000464c2303fb0646a64206d004f108003c
:10ba5000fff7e8ff4c340544f6e7284670bd00bf09
:10ba6000f8d30010f8b50b4b0026d3e9004750235c
:10ba700003fb0747a7420bd0601dfff7d3ff01214f
:10ba80000546201d13f0d6fd284406445034f1e746
:10ba90003046f8bdecd3001007b5fff7e3ff009088
:10baa000fff7caff08210190684613f0c3fd03b0f9
:10bab0005df804fb10b50c46fff7eeffd4f8e0305c
:10bac000c4f8d40043f00203c4f8e03010bd70b5f0
:10bad000142486b02246002101a8b9f07afa78260b
:10bae000adf8044000240022012101a822f0b4fb9b
:10baf000bdf80650bdf80c30a34209dd02982021a4
:10bb000006fb04004c3013f095fd01340544f1e7c9
:10bb1000002201a8114622f09ffb284606b070bd06
:10bb200010b50c46fff7d3ffd4f8e030c4f8d800c6
:10bb300043f00103c4f8e03010bd38b58468054611
:10bb40005cb144684cb12046f5f794f9402808d818
:10bb500020462946fff7d6fe0446201e18bf0120c6
:10bb600038bd0024f9e710b410461a46d1e9103464
:10bb700024b1014620465df8044b184711465df894
:10bb8000044b18471b681268fff7edbf07b5016843
:10bb90000a468b6a32f8080b009301f118034968d2
:10bba000fff7f0ff03b05df804fb30b5c3b04ff40e
:10bbb0008372002104466846b9f00bfa00234ff463
:10bbc00083711a466846fef75dffb0f5837f12d198
:10bbd000bdf80050b5f5837f0dd1a3680bb9b8f05f
:10bbe00051fc69462046e3689847002329461a46d7
:10bbf0006846fef725ff43b030bd000003291fb59e
:10bc000015d128b101280ed0002005b05df804fb45
:10bc10002d4b03932d4b68460293fff7c6ff6846f2
:10bc2000f7f742fdf0e72a4b03932a4bf3e702298b
:10bc300032d102380628e7d801a353f820f000bf1c
:10bc4000ddbb0002e7bb000289bb0002f1bb0002c2
:10bc5000fbbb000205bc00020fbc00021e4b0092a1
:10bc600003931e4bd7e71e4b009203931d4bd2e765
:10bc70001d4b009203931d4bcde71d4b0092039388
:10bc80001c4bc8e71c4b009203931c4bc3e71c4b97
:10bc9000009203931b4bbee701290cd130b1012860
:10bca000b2d105b05df804ebfff711bf05b05df848
:10bcb00004ebfff7f1be0429a6d10428a4d1124b4e
:10bcc0000393124ba7e700bf35ba0002c1ae0002d2
:10bcd000a1ba0002b7ae000233a90002a3ae00026f
:10bce00047a900028fae00025ba900027bae0002f2
:10bcf0006fa9000267ae000283a9000253ae0002e2
:10bd000097a900023fae0002aba9000235ae0002c7
:10bd10002de9f04302291646984691b03dd10a46d6
:10bd200001461f48b9f01ef90446002835d11c25ec
:10bd300001a8faf737fc2a46214609a8039fb9f063
:10bd400048f9214609a8adf82450fef74ffa9df8ae
:10bd50002b20144905a80bf009fdddf81c9007eb1a
:10bd60000905a84513d93a4601993046b9f00af9b0
:10bd70004a460599f019b9f005f905a80bf030fc11
:10bd800001a80bf02dfc284611b0bde8f08305a8f2
:10bd90000bf026fc01a80bf023fc0025f3e700bf05
:10bda00099d20d02b3cc0d020138c0b208289abf57
:10bdb000014b185c0220704734d00d02042906d0d4
:10bdc000092907d0012914bf04200120704718b1a8
:10bdd000f5f750b8082070477047000010b5184bb1
:10bde0008cb01b7803f0ff001bb1164b1c7814b10c
:10bdf00001200cb010bd21f03efd134b1b78002b31
:10be0000f6d043f69821114a1368c31a8b42efd932
:10be10002023cde9043413680d49cde901030d4b0e
:10be20002820009304aa2346f6f736fd2046234631
:10be300022462146009405f0d3fd2046d9e700bff5
:10be40005dd4001084f600105ad4001040d30010c6
:10be500060c30d02b8cc0d0208b5fff78ffc054b8f
:10be600018680cf055fa18b9bde80840fff794ba05
:10be700008bd00bf2cd4001008b5012003f03efc23
:10be8000092003f03bfc002008bd00002de9f04331
:10be900000244ff02008b24bb1b01c70b14bb24e31
:10bea00020ad2a46b14901900093074623461e2043
:10beb000cde92084f6f7f0fc214630680cf01bfa3f
:10bec0000d28034657d12346032240200021cde907
:10bed00001440094fbf764fba54ba4492a461e20ad
:10bee00000932346cde92084f6f7d6fcfff796f8b9
:10bef000fff7c2ff204621f0effd014628b9faf70f
:10bf0000bdfa0146002800f0e68003f033f801286e
:10bf100040f00381974b1b78002b40f0fe80964b3e
:10bf20001868b0b101230a2229460bf058fc0024fe
:10bf30002023cde91034914b1e208c49009310aa88
:10bf400023460195f6f7a8fc224629468c48fff7c0
:10bf50005af800220823306810a9cde91022adf864
:10bf600040300cf09efb0446002800f0e0800cf00e
:10bf700055f90446d7e020b131b0bde8f0430cf0ec
:10bf80004db902220021cde9010000900df14009d8
:10bf90004020fbf705fb4021484622f06afc04469e
:10bfa000b0b99df84030013bdbb2fd2b10d8754b8a
:10bfb0002a46cde920806d490093cdf804900346d0
:10bfc0001e20f6f769fc224649466f48fff71bf82a
:10bfd000002340224946184600931df005f9044607
:10bfe00090b99df840307bb12023cde92030674bdc
:10bff0002a465e49009303461e20f6f74dfc224672
:10c0000049466348fef7fffffff708f800220620c5
:10c010000df117018df8172003f050fb044600289e
:10c0200053d19df81730002b4fd002460146062011
:10c0300003f02cfb224607a906a8cde9064413f01d
:10c04000edfa002841d1ddf81880b8f1000f3cd09e
:10c050005ffa88f3502b079c7ed048d8282b00f03d
:10c06000b5803cd8142b00f0b3801e2b00f0b280ba
:10c070000a2b00f0b1804346464a40212846b9f0d9
:10c08000dfffb8f1820f01460ed1631edbb20c2b2d
:10c090002844c1f140013dd83f4a52f82330002bdb
:10c0a00038d03e4ab9f0ccff00242023cde9083433
:10c0b0003b4b1e202d49009308aa2346f6f7ecfbc4
:10c0c000224629463748fef79efffff7d5fe0fb1ff
:10c0d000f9f72bfc002130680cf02cfa15e73c2b0b
:10c0e0007cd0462b7cd0322bc5d12f4b35e0782b22
:10c0f00078d007d8642b77d06e2b77d05a2bbad153
:10c100002a4b2ae08c2b73d0962b73d0822bb2d182
:10c11000274b22e02346274ac4e7fff7dbf8044613
:10c1200000283ff4fcae204631b0bde8f083119bff
:10c13000012013f0010f0cd01f4b2a46187020234a
:10c14000cde920341d4b094900932346f6f7a4fba3
:10c15000e9e71b4b1870e6e71a4b1b4a8de700bf57
:10c160004dce001074cd0d022cd4001060c30d0212
:10c170009dcd0d021cd6001044d3001080ce0d02c0
:10c18000a5ce0d02c4cd0d02f3cd0d020bce0d02d6
:10c190002bce0d02e3cc0d0200d00d0240ce0d02dd
:10c1a00045ce0d0268ce0d0208cd0d0265cd0d0203
:10c1b000ccb40d02e1cc0d025cd40010bcce0d025b
:10c1c0005bd4001058cd0d0242ce0d020a4bc4e7dd
:10c1d0000a4bc2e70a4bc0e70a4bbee70a4bbce773
:10c1e0000a4bbae70a4bb8e70a4bb6e70a4bb4e783
:10c1f0000a4bb2e70a4bb0e74dcd0d02e6cc0d027b
:10c2000033cd0d02891f0e0244cd0d0276ee0d02d4
:10c21000ffcc0d0217cd0d02f0cc0d02facc0d02b1
:10c2200025cd0d02024b002118680cf066b800bf46
:10c230002cd4001010b5104b8ab01b78bbb1fff79f
:10c24000f1ff044698b92023cde902300b4b0c498d
:10c25000009302aa03462820f6f71efb2346224637
:10c2600001212046009405f0bbfb0ab010bd21f06f
:10c2700002fb044b1860f8e75dd4001005cf0d02f7
:10c2800060c30d0240d30010f8b50c4616461149a4
:10c2900005460bf0f0f92644a64219d0274623782c
:10c2a00028461b0903f13001392988bf03f15701e2
:10c2b0000bf04efa3b78284603f00f0303f13001f0
:10c2c000392988bf03f1570101340bf041fae3e744
:10c2d0002846f8bdc3c30e020048704748d300107b
:10c2e00000487047d4d30010f0b50c461d46096cc9
:10c2f0003d4ba5b0994206462a9f08d12b462146c0
:10c3000030462a9725b0bde8f040fff72cbc00204e
:10c31000019202f03bfe019a0028efd0114602a8dc
:10c320000bf0a9f9294606a80bf0a5f92f4b93f8b5
:10c330006c203ab906a80bf053f902a80bf050f99b
:10c3400025b0f0bd586e27f0caff05460028f1d190
:10c3500002a910a80f94adf838600bf0d7f906a920
:10c3600014a80bf0d3f9bdf8383010a9adf864303b
:10c370000f9b1ba81a9318970bf0c8f914a91fa8b4
:10c380000bf0c4f9189b2c2023930c951df0c0fad8
:10c39000044680b1bdf864301ba903801a9b0830a5
:10c3a00040f8043c0bf098f91fa904f118000bf0b9
:10c3b00093f9239ba3620e4b1fa80d930d4b0a9478
:10c3c0000c930bf00df91ba80bf00af90aa907480a
:10c3d000faf724fc0aa8f7f767f914a80bf000f99c
:10c3e00010a80bf0fdf8a5e729ab00025cd5001002
:10c3f0000dbb0002dfae00022de9f0431f46194bd2
:10c40000164693f86c2085b00446dde90c890d468c
:10c41000eab1586e27f063ffc8b9029018201df0ea
:10c4200077fa28b1c0e90045c0e90267c0e904898c
:10c430000d4b694603930d4b00900a480293faf79f
:10c44000edfb6846f7f730f905b0bde8f0833b46f1
:10c45000324629462046c446cdf8309005b0bde8a6
:10c46000f043604778ce0010f1c30002f1ad000246
:10c4700007b500684369019303690093d0e902237b
:10c48000d0e90001fff7b8ff03b05df804fb00003e
:10c490002de9f041304b174693f86c2004460e46c8
:10c4a00088b0d2b1586e27f01affb0b906900c20b0
:10c4b0001df02efa10b1c0e900468760274b0490aa
:10c4c0000793274b244804a90693faf7a7fb04a86f
:10c4d000f7f7eaf808b0bde8f0810023cde90333af
:10c4e000e36c25688bb1284603aa04a99847002865
:10c4f00025da00231e201a461946cde90067fff70a
:10c500007bff0498b8f018fde4e7d4f84880b8f150
:10c51000000f04d02a462179601dc04705462846f1
:10c520002179fff74bfc8046039040b1b8f0fcfc4a
:10c5300004900028ddd042462946b8f023fd20793a
:10c54000fff732fcdde903320146cde90067002048
:10c55000fff752ffbee700bf5cd50010e5c4000244
:10c56000b1ad000203681868d3e90112fff790bf6c
:10c5700037b50c461546fff70df9034630b12a468c
:10c58000214603b0bde83040fff782bf02460146b6
:10c5900000951d20a04703b030bd38b5002383604f
:10c5a0008b6804460d462bb102229847eb68e36086
:10c5b000ab68a360204638bd012a70b5054603d19b
:10c5c0000b680360002070bd022a0dd0032af9d148
:10c5d0000468002cf6d004f10800f7f765f818217c
:10c5e00020461df09df9ede718200e681df090f92a
:10c5f000044648b1336806f10801036073680830e7
:10c6000040f8043cfff7c9ff2c60dbe7012a70b556
:10c61000044603d10b680360002070bd022a0cd0d1
:10c62000032af9d10468002cf6d02046f7f73cf82d
:10c63000142120461df074f9eee714200e681df059
:10c6400067f9054620b13146fff7a7ff33692b6133
:10c650002560e1e713b56c460b460246d0e90001c0
:10c6600084e8030093e8030082e8030094e80300f1
:10c6700083e8030002b010bdf0b517461c46002247
:10c6800043688fb000680d469847064627b11db134
:10c69000012128461df044f9264b93f86c20002a0e
:10c6a00039d0586e27f01bfe0546002833d12146ad
:10c6b00004a8fff772ff04a909a80896fff76dff09
:10c6c000089b14200d9302951df022f9044670b1c9
:10c6d0000146856009a8fff7bdff0b9ba268a36018
:10c6e0000c9b0b92e268e3600d9b0c922361124b52
:10c6f00009a80393114b00940293f6f7d5ff6946fe
:10c700000c48faf78bfa6846f6f7ceff04a8f6f75e
:10c71000cbff0fb0f0bd02238df81030a36809964f
:10c720000bb9b7f0affe2046e36804aa09a9984701
:10c73000efe700bf78ce00102db200028dc50002d9
:10c7400030b5016885b0d1e9004568460831fff78a
:10c7500024ff6b46012229462046fff78dff6846dd
:10c76000f6f7a2ff05b030bdf0b591b00d46174603
:10c77000fff7aef80446002855d02846b9f012fd60
:10c780002a4b064693f86c20002a40d0586e27f0ba
:10c79000a6fd054600283ad1394606a8cde904464b
:10c7a000fff7fbfe049b06a90a93059b0ca80b93bd
:10c7b000fff7f3fe182002951df0aaf8044688b191
:10c7c0000a9b056103600b9b00f1080143600ca804
:10c7d000fff740ff0e9b226923610e920f9b626957
:10c7e00063610f92124b0ca80393124b00940293b7
:10c7f000f6f75aff69460d48faf710fa6846f6f759
:10c8000053ff06a8f6f750ff002011b0f0bd3946df
:10c810000aa8fff7c2fe2046012231460aabfff705
:10c820002bff0aa8eee74ff0ff30eee75cd50010d3
:10c83000c1c6000239c500022de9f84300254ff0ba
:10c8400014082c4b2c4cc3e900559d602b4b0a213e
:10c85000c3e900552a4a9d602046f6f7b5fd294bed
:10c86000294a1e2104f11c002360a561f6f7acfde6
:10c87000264bdff8c090e361254b264fc4e90f83b8
:10c88000254b2946636404f13c0004f13803a3649a
:10c890006563c4f83890e764f6f77cfa1f4b204ec6
:10c8a000e365204b2946236604f1580004f1540344
:10c8b000c4e91937c4e91459a663c4f85880f6f7d7
:10c8c00069fa194a0d2104f170006665e566f6f70c
:10c8d0007bfd47f23052154bc4f888502367144b48
:10c8e000c3e903551d705a601d725d729d82bde8db
:10c8f000f88300bfecd3001048d30010f8d3001029
:10c9000034cf0d02e8cf0d023fcf0d02f8cf0d025c
:10c910000e000200993200024ecf0d021d000200ef
:10c9200048c50d025acf0d0268cf0d0258c50d0241
:10c93000d4d30010a8bc0d0209490c2008b5b7f0eb
:10c940009dfd014650b1074b036000238360064bf9
:10c950004360bde808400548fcf748bb08bd00bf80
:10c960001308100244c60d02f1c800024cf6001074
:10c9700010b510b103685b689847f9f7edfd40b159
:10c98000fef7fcfebde81040002304211a460bf020
:10c990006ebe10bdc0e8af1f704700002de9ff411b
:10c9a00013680546d3e900461c230f4603fb0646e1
:10c9b000dff84080b4421ad0002110226846b8f057
:10c9c00008fb6946204608f0a1f960b939462846b7
:10c9d00035f071fd38b16a464146284635f097fd7d
:10c9e0001c340028e6d1002004b0bde8f08101200d
:10c9f000fae700bfa0640e022de9f743136805466d
:10ca0000d3e900461c230f464ff0000903fb0646fe
:10ca1000dff83880b44217d0204601a9cdf8049041
:10ca200008f066f960b93946284635f044fd38b15a
:10ca30004146284601aa35f06afd1c340028e9d198
:10ca4000002003b0bde8f0830120fae778640e020d
:10ca50002de9f0474ff03c08074689461368dff898
:10ca600060a0d3e9006308fb03688eb0464525d07b
:10ca700035461822002101a807acb8f0aafa0fcd5c
:10ca80000fc495e8070084e8070001a907a808f08b
:10ca900051f978b996f8383049463846069335f05a
:10caa0000afd38b15146384601aa35f030fd3c3612
:10cab0000028dbd100200eb0bde8f0870120fae7a6
:10cac00010670e0238b51468054623685bb16368c9
:10cad0004bb135f0f0fc38b1d4e900122846bde87e
:10cae000384035f002bd012038bd38b50025044678
:10caf000c0e90055c0e90255c0e90455c0e9065532
:10cb00002030fbf72ff904f13c00fbf72bf920460e
:10cb1000c4e91655c4e91855c4e91a55c4e91c55a9
:10cb2000a56738bd002108b50346c0e900110162c0
:10cb30000a460830c0e8af1f03f10c00fff72affd8
:10cb400003f11000fff726ff03f11401c1e8af2f36
:10cb500003f11801c1e8af2f012103f11c02c2e863
:10cb6000af1f184608bd000010b50a4cd4e88f3f2f
:10cb7000db070cd420461ff0c1f840b10648fff790
:10cb8000d1ff20461ff0f4f80448b7f0d4ff024864
:10cb900010bd00bf30d4001034d4001041cb0002cf
:10cba00010b50446006818b130f05cfa0023236029
:10cbb000606818b12ef0dcf90023636010bd00003e
:10cbc0000148fff7edbf00bf34d400100c30d0e8af
:10cbd000af0f831e5842584170471030d0e8af0f56
:10cbe000831e58425841704710b50c46002120461c
:10cbf0002ef0eaf92ef08ef9204601212ef0e4f90c
:10cc0000bde810402ef086b91fb51c30d0e8af3f0c
:10cc1000022b0fd193681b78022b0bd10023052226
:10cc2000cde90133009320200021faf7b9fc05b0cb
:10cc30005df804fbd0e8af3f002bf8d19268127882
:10cc4000012af4d10322cde901330093ebe773b558
:10cc50000024054601a801942ef04cf8a04219dbef
:10cc60000198264603465bb15a682ab15278022ad7
:10cc700004d00a2a08bf01241b68f4e70126fbe759
:10cc80002ef030f805f11403c3e8af6f05f1180377
:10cc9000c3e8af4f02b070bd002307b50846694630
:10cca0000093adf804302ff0c5fe02226846044917
:10ccb000b9f0ceff003818bf012003b05df804fbc7
:10ccc000d8d00d02f7b506460c4611bb6846009158
:10ccd0002ff07efc002819db2746009d9db1686877
:10cce00078b101a901972ff0a7fd002809db019b6e
:10ccf0001b0706d430466968fff7ceff002818bf2f
:10cd000004462d68eae700982ff08efc204603b019
:10cd1000f0bd03b0bde8f040fff7bebf006a20b130
:10cd200083688b4201d00068f9e77047f0b50025b1
:10cd300085b016460c468df8075031bb02a802910b
:10cd40002ff046fca8421ddb2746029dbdb1686856
:10cd500098b103a903972ff06ffd00280ddb039b0b
:10cd60001a070ad468680df1070130f09efa20b95d
:10cd70009df80730b34208bf01242d68e6e702980a
:10cd80002ff052fc204605b0f0bd20460df1070102
:10cd900030f08bfa28b99df80740a31b5c425c4138
:10cda000f0e72c46eee77fb500250c46019539bb30
:10cdb00002a802912ff00cfca8421edb2646029d21
:10cdc000c5b16868a0b103a903962ff035fd00280e
:10cdd0000edb039b13f008030ad1686801a90193d5
:10cde0002ff09cfc20b9019b13f4801f18bf012475
:10cdf0002d68e5e702982ff017fc204604b070bdbf
:10ce0000204601a92ff08afc18b9019cc4f30054f4
:10ce1000f3e72c46f1e738b5022204460d46fff74a
:10ce200085ff28b129462046bde83840fff7bbbf43
:10ce300038bd38b5012204460d46fff777ff30b103
:10ce400029462046fff7afff80f00100c0b238bd91
:10ce500008b5fff763ff00b1007908bd2de9f04385
:10ce6000002485b0064602a80f4602942ff0b0fbbe
:10ce7000a04224dba146029df5b16868d0b103a9a8
:10ce8000cdf80c902ff0d8fc002813dbddf80c80d7
:10ce900018f0080f0ed1696830460191fff7fcfecb
:10cea00040b130460199fff7d3ff18b137ea0803c4
:10ceb00008bf01342d68dfe702982ff0b5fb20464c
:10cec00005b0bde8f08370b505460026046a4cb194
:10ced00023792bb12846a168fff7defe00b10136a9
:10cee0002468f4e7304670bd08b5fff717ff10b1ae
:10cef0000c30d0e8af0f08bd08b5fff70fff10b139
:10cf00001030d0e8af0f08bd0a4608b5036a73b108
:10cf100012b19968914208d103f10c000021fff78a
:10cf200039fd03f11000fff735fd1b68efe708bd81
:10cf300008b50448baf01cf8002818bf6ff0f900d3
:10cf400008bd00bf40d20d022de9f04100209ab08b
:10cf50000e462df015f90546002847d02df046f86d
:10cf600028462df089f8041e39db244f3822002191
:10cf70000ca8b8f02ef8012239460ca8f5f714f9e0
:10cf8000041e2cdb1e4b1f4902aa0ca80396029319
:10cf9000f5f754f9002805f140062ada00244ff08d
:10cfa0002008194b32201949009304aa2346cde9e1
:10cfb0000484f5f771fc164b28201449009304aa49
:10cfc00023460197cde90484f5f766fc0ca93046a9
:10cfd00054f094fd3946304655f03cf8002428467c
:10cfe0002df028f820461ab0bde8f0816ff0e0047b
:10cff000f8e730460ca954f081fdefe740d20d026e
:10d00000bde80002185f0e02e5d00d02dbd00d0274
:10d0100006d10d022de9f04100209ab088462df08e
:10d02000aff8064600284fd02cf0e0ff30462df038
:10d0300023f8041e38db382200210ca8b7f0c9ff02
:10d04000022223490ca8f5f7aff8041e2cdb06f1e9
:10d050004007002238460ca954f0c0fa054650bbe0
:10d060001c4b1d4902aa0ca8cdf80c800293f5f7c1
:10d0700007f9041e0edb2023cde90435174b0120f0
:10d080000193174b1749009304aa2b462c46f5f73a
:10d0900003fc012538460ca954f030fd7db138461b
:10d0a0000e4a0b4955f024f830462cf0c3ff2046b9
:10d0b0001ab0bde8f08100256ff0e004eae73846d9
:10d0c000034954f0c7ffefe76ff0e004efe700bf5c
:10d0d00051d20d02c9e10002185f0e0240d20d02ca
:10d0e00018d10d02dbd00d0210b504460068b7f070
:10d0f00023ff204610bd10b504460068b7f01cffa2
:10d10000204610bd10b504460068b7f015ff204654
:10d1100010bdd0e8af0f704708b50830fff7f9ff32
:10d12000013818bf012008bd08b50830fff7f1ff2e
:10d13000043802288cbf0020012008bd08b5083043
:10d14000fff7e7ffc31f5842584108bd2de9f341df
:10d150000546fff7e9ff58b14ff000086846cdf8e3
:10d1600000802ff035fa002808da02b0bde8f0811f
:10d170002846fff7e3ff0028eed1f6e7009c44b312
:10d180006068e8b101a9cdf804802ff055fb0028b4
:10d1900016db019e330713d4676828463946fff72c
:10d1a0007bfd68b139462846fff7b8fd40b10379e9
:10d1b00006f0010633b11eb9012138462ff095fb68
:10d1c0002468dce7002efbd0012138462ff0bafba3
:10d1d000f6e700982ff028fa2046c6e708b5083091
:10d1e000fff797ff08bd0000f0b500f10805044601
:10d1f0008db028460e46fff78cff072813d1072e67
:10d2000000f0e580002104f10c00fff7c3fb04f1fe
:10d210001000fff7bffb04f11402c2e8af1f04f1d6
:10d220001802c2e8af1f731e062b1ed8dfe803f0fa
:10d230000439698793c8cf00002704f11c03c3e8b1
:10d24000af7f2a213b463a463846f9f763fe3b4614
:10d25000022200212020cde901770097faf7a0f9fa
:10d26000faf77cfb00f118031f60202300272846f3
:10d27000cde90437fff74dff634b644953f826208f
:10d2800053f8203002920193614b1e20009304aab0
:10d290003b46f5f701fb04f10803c3e8af6f0db09f
:10d2a000f0bd00232a211a460120f9f733fefaf7d0
:10d2b00055fb022200f118031a602846fff729ffe8
:10d2c00003280ed1072204f11c03c3e8af2f00236b
:10d2d0000b22cde90133009320200021faf760f9f9
:10d2e000c3e72846fff715ff0128bed1022204f14b
:10d2f0001c03c3e8af2f00230422cde901330093c0
:10d30000eae7062204f11c03c3e8af2f2846fff723
:10d3100000ff072803d1faf721fb0023c36600238f
:10d320000a22cde90133009320200021faf738f9d1
:10d33000faf714fb052200f118031a6095e70023a1
:10d340002a211a460220f9f7e5fdfaf707fb032226
:10d3500000f11803f1e7042204f11c03c3e8af2f26
:10d360002846fff7d6fe07280fd1faf7f7fa012271
:10d3700000f134031a60faf7f1fa074611f056ff8c
:10d380003b6d01333b6511f055ff00232a211a46fe
:10d390000220f9f7bffd00230622cde901330093f7
:10d3a00000212020faf7fcf8faf7d8fa032200f15e
:10d3b00018031a60faf7d2fac36e0133c36654e752
:10d3c00000232a211a460320f9f7a4fd4de7052280
:10d3d00004f11c03c3e8af2f00232a211a460420be
:10d3e000f9f798fdfaf7bafa042200f118031a6067
:10d3f0002846fff78efe07283ff437af00230722a9
:10d40000cde90133009367e768d20d02dbd00d024e
:10d4100029d10d0210b50368044623b90146084816
:10d420002ff010fe2060636823b9214605482df0d7
:10d4300089fd60602046bde810400121fff7d4bea1
:10d44000b7ed00022bd7000210b504460830fff7f5
:10d4500060fe012803d102212046fff7c5fe6ff0d0
:10d46000d10010bd10b504460830fff752fe012868
:10d4700008d0022803d101212046fff7b5fe6ff046
:10d48000d10000e0002010bd2de9f7430746083029
:10d49000fff73ffe022844d1002504213846fff75c
:10d4a000a3fe684600952ff093f8041e30db2c464f
:10d4b000a946ddf80080b8f1000f24d0d8f80400a8
:10d4c000f0b101a9cdf804902ff0b6f9002817dbd0
:10d4d000019e320714d4d8f8045038462946fff785
:10d4e000dbfb68b129463846fff7b2fc40b1f307d1
:10d4f00006d4012128462ff0f8f90028a8bf0134ee
:10d50000d8f80080d7e700982ff08ef824b1444671
:10d51000204603b0bde8f08305213846fff764fede
:10d52000f6e76ff0d104f3e7f7b5054608300c468f
:10d53000fff7effd0138012846d92846fff7fefd29
:10d5400088b1faf70bfa06466cb100f134031c609f
:10d55000012c01d0062c06d111f068fe336d013389
:10d56000336511f067fe002703212846fff73cfed4
:10d57000684600972ff02cf8041e1ddb3c46009ee9
:10d58000aeb1706888b101a901972ff055f9002854
:10d590000bdb019b1a0708d4db0706d50121706855
:10d5a0002ff0d0f90028a8bf01343668e8e70098ca
:10d5b0002ff03af81cb13446204603b0f0bd0221ea
:10d5c0002846fff711fef7e76ff0d104f4e738b50e
:10d5d000936804461b7800f108059bb12846fff7c5
:10d5e00098fd04281dd105212046fff7fdfd4021af
:10d5f0002046fff733fca0b106212046bde83840a5
:10d60000fff7f2bdfff7f0fa2846fff782fd032887
:10d6100007d101212046fff721fc012801d8022172
:10d62000ebe738bd2de9f047002788b0002106461a
:10d63000fff76afc684600972ff0a2fcb842c0f2e0
:10d64000ad80b846ddf80090b9f1000f5fd0d9f891
:10d65000083013f008043fd103f04103412b3bd1c4
:10d66000d9f80c30002b37d01968002934d04d7808
:10d67000022d34d11a7c002a46d09968002943d063
:10d6800001a8faf777fb01a8faf783fb00283bd142
:10d690000446a845b8bfa84699f81000a74201a9ba
:10d6a000b8bf27462ff006f8b0b930460199fff70a
:10d6b00035fb034680b10c30d0e8af2f954202dd38
:10d6c0002946fff767f903f11000d0e8af3f9c420d
:10d6d00002dd2146fff75ef9d9f80090b4e70a2d84
:10d6e0000ad1da681c7c8b6943b974b162b11478d1
:10d6f00014f0020409d002240025cae72cb11ab1a3
:10d700001478c4f34004f7e700242546c1e70098e5
:10d710002ff049fa06f10c0adae8af9f06f110047f
:10d72000d4e8af5f3046fff792fa41465046fff724
:10d7300031f939462046fff72df9b8f1020f1ad01a
:10d74000022f1fd0002406f1080a5046fff7e1fc23
:10d75000072800d1f4b15046fff7dbfc062820d0a3
:10d760005046fff7d6fc072818d1bcb1c8451ad1de
:10d77000af4218d112e006f11403d3e8af4f012ce9
:10d78000ded1e0e706f11803d3e8af4f631e5c4239
:10d790005c41d8e706213046fff726fd08b0bde81a
:10d7a000f087002cdcd00721f5e7fff73bbf38b549
:10d7b00000f1080504462846fff7abfc072806d110
:10d7c0002046fff72fffbde83840fff7b5b82846e1
:10d7d000fff79ffc0628f6d1f2e770b50446d0e9c2
:10d7e000005305ebc316ae4204d0281dfaf750fbd8
:10d7f0008035f8e72068b7f09ffb204670bdf0b594
:10d8000000260d460446c0e9006686600b680e607f
:10d8100003604b684e6043608b688e60c0e90366ae
:10d8200046618360cb6800f12007c3600b69ce605e
:10d8300003614b690e6143618b694e618361cb6902
:10d8400001f1200cc361bce80f000fc79ce8070082
:10d8500005f13c0c87e80700bce80f0004f13c0729
:10d860000fc79ce8070087e80700c4e9166626662c
:10d87000ab6dae65a365eb6d2046e3652b6eee6583
:10d880002e66c4e91966e66623666b6e6e6663668d
:10d89000ab6eae66a366eb6eee66c4e91c66a66769
:10d8a000e3662b6f2e6723676b6f6e676367ab6fe3
:10d8b000ae67a367f0bdd0e88f0fc0b2704700001d
:10d8c00070b58cb0fff72afa0e46044670b92023d3
:10d8d000cde90430254b2649009304aa03463220a3
:10d8e000f4f7daff6ff0a9000cb070bd00f1140579
:10d8f0001ab3022328468df80c30fff7dcff02280c
:10d9000007d02846fff7d7ff042802d00422c5e835
:10d910008f2f20210023cde90413164a0092012005
:10d9200004aa1349f4f7b8ff0023009301233046fb
:10d93000194603aa2ff0c8fbd6e7012328468df825
:10d940000c30fff7b8ff012809d02846fff7b3ffd6
:10d95000032804d0032204f11403c3e88f2f2022ec
:10d960000023cde90423044ad8e700bf41d10d02ca
:10d97000dbd00d025cd10d027ed10d0270b51546d3
:10d98000fff7ccf900b300f114042046fff793ff32
:10d99000012801d1002070bd1ff06dff0646204612
:10d9a000fff789ff012807d064201cf078ff1ff0e3
:10d9b00062ff831bab42f2d92046fff77cff0128b0
:10d9c000e8d06ff09f00e6e76ff0a900e3e7000002
:10d9d000f0b58fb00d461646fff7a0f960b92023c9
:10d9e000cde90630164b1749009306aa03463220ac
:10d9f000f4f752ff0fb0f0bd00f114073846fff7ff
:10da00005affb3681b789842f4d0c7e88f3f0df1f6
:10da1000170128462ef0f2fe202200239df8171051
:10da2000cde90623d7e88f2fd2b2cde90112064afd
:10da300001200092034906aaf4f72effdae700bf9f
:10da400041d10d02dbd00d02a1d10d0200232de941
:10da5000f04f93b0054608a8059108932ef0b8fd45
:10da600000285fdb089cdff8c8a0dff8c8b0002cf6
:10da700055d06068002850d0002309a909932ef0e2
:10da8000dbfe002849db099b13f0080845d16668d6
:10da900028463146fff742f9074680b95946182013
:10daa000b6f0ecfc0746002837d02b6ac0e90388a3
:10dab00080f8048080f81480866003602862059beb
:10dac00030463b7100230df11e018df81e302ff002
:10dad000ecfb814608bb07f114084046fff7ebfe5c
:10dae0009df81e10884218d0c8e88f1f0df11f0145
:10daf00030462ef083fe20229df81f10cde90a2922
:10db0000d8e88f2f094bd2b2cde9011200935146cc
:10db10004b4601200aaaf4f7bffe2468a7e708983d
:10db20002ef082fd13b0bde8f08f00bfc6d10d020c
:10db3000dbd00d021308100210b521b90121fff747
:10db400085ff002010bdfff7e9f810b10123037134
:10db5000f7e76ff0a900f5e770b505460c461646e5
:10db6000f9f7fcfe00f134031e60214628461cb97b
:10db7000fff76cff204670bdfff7d0f810b100240e
:10db80000471f7e76ff0a900f5e784b0f0b5064639
:10db900091b017ac84e80e0001ad47680fcc0fc5fb
:10dba0000fcc0fc50fcc0fc594e8070085e8070020
:10dbb000b3689f4220da3c21736801fb07f24b43b4
:10dbc000346801ad144421469a1a04f13c00b7f0c0
:10dbd000e6f90fcd0fc40fcd0fc40fcd0fc495e8dc
:10dbe000070084e80700012073680133736011b0f7
:10dbf000bde8f04004b070473046791cfaf7a2fe49
:10dc00000028d8d1f3e700002de9f0430546b7b06e
:10dc1000002114460ca81822b7f0dbf9012328468e
:10dc20003e490caa35f079fb18b9002037b0bde8a1
:10dc3000f08312a8faf796f812a90ca807f044f896
:10dc400081460028f1d1276819ae12ac0fcc0fc65f
:10dc500094e807000df19c0886e8070040469df80f
:10dc60004450faf77ff82ea8faf77cf820ac0df1b3
:10dc7000640cbce80f000fc496e8070046460df19f
:10dc8000800c84e80700bce80f00c4460fc694e887
:10dc900007002eac86e807008df8d450bce80f00d2
:10dca0000fc496e807009df8b93084e80700022bfe
:10dcb00019d14ff0ff33c5f12000c34003fa00f043
:10dcc0002ff01afd2f906c462aad0fcd0fc40fcd4b
:10dcd0000fc495e80f0084e80f00384698e80e005e
:10dce000fff753ffa2e70a2bedd1ff2430aa002d46
:10dcf000e9d0072d8fbfff23c5f1080144fa01f3d6
:10dd00008b4088bf083d09f1010994bfdbb2edb239
:10dd1000b9f1100f02f8013be9d1d4e710670e0208
:10dd2000f0b54b780746022b0e468db011d16c46ec
:10dd300001f10c050fcd0fc40fcd0fc495e80f00f6
:10dd400084e80f0096e80e003846fff71eff0db07e
:10dd5000f0bd0a2bfbd16c4601f10c050fcd0fc4b1
:10dd60000fcd0fc495e80f0084e80f0096e80e0071
:10dd700007f10c00e9e738b50d1e0446006803dd25
:10dd8000b8f0a8f818b938bdb7f0d6f80020206070
:10dd9000a5600120f7e7002370b5151e04460e4666
:10dda000c0e90033836009dd2946fff7e4ff28b1ad
:10ddb0002a4631462068b7f0e5f86560204670bd18
:10ddc00038b50023c0e9003383600d464968044636
:10ddd000994210ddfff7cfff68b1d5e90031226825
:10dde0001944994205d00ab11878107001330132f4
:10ddf000f7e76b686360204638bdf8b504460d460a
:10de0000faf7b2fd05f10c0104f10c00faf7acfdd4
:10de1000ab6904f12006a361eb6905f12007e3611a
:10de20000fcf0fc697e8070005f13c0786e807000b
:10de30000fcf04f13c060fc697e8070086e80700fd
:10de400005f1580104f15800faf7fefd05f16401ef
:10de500004f16400faf7f8fd05f1700104f17000b7
:10de6000fff7aeff2046f8bdf0b504460d4685b07d
:10de700001a8faf779fd019a23682260029a0193ba
:10de800063686260039a0293a36801a8a260039387
:10de9000fff72af905f10c0101a8faf765fd019acf
:10dea000e368e260029a019323692261039a029374
:10deb000636901a862610393fff716f9ab6904f186
:10dec0002006a361eb6905f12007e3610fcf0fc6c0
:10ded00097e8070086e8070005f13c0704f13c06d7
:10dee0000fcf0fc697e8070086e8070005f1580135
:10def00001a8faf7a9fd019aa36da265029a019300
:10df0000e36de265039a0293236e01a822660393f0
:10df1000fff7f1f805f1640101a8faf795fd019a00
:10df2000636e6266029a0193a36ea266039a0293dd
:10df3000e36e01a8e2660393fff7ddf805f17001d7
:10df400001a8fff73dff019a236f2267029a019310
:10df5000636f6267039a0293a36f01a8a26703939a
:10df6000fff7d0f805b0f0bd84b0f0b5054689b034
:10df70000fac84e80e0001ae47680fcc0fc694e8e2
:10df80000700ab6886e807009f421cda1c216b681b
:10df900001fb07f24b432c6801ae144421469a1a48
:10dfa00004f11c00b6f0fbff0fce0fc496e807008b
:10dfb00084e8070001206b6801336b6009b0bde89d
:10dfc000f04004b070472846791cfaf72bfd002872
:10dfd000dcd1f3e72de9ff410023c0e90033836082
:10dfe00032f0020305460e46174618d1d1e9164312
:10dff0004ff01c0808fb034844450bd004f10c0308
:10e000000fcb8de80f00284694e80e00fff7acff19
:10e010001c34f1e72fb1284604b0bde8f0810a2a8c
:10e02000f9d1d6e919461c2303fb0646b442f2d0c7
:10e0300004f10c030fcb8de80f00284694e80e0086
:10e04000fff792ff1c34f1e72de9f04f0646d2e9c5
:10e050000043894604ebc313bdb005931034059a01
:10e06000a4f110039a4200f0e280782200210deb27
:10e070000200b6f0aeff04f1640108a8fff7a0fead
:10e08000089b0693099b079306ab3b93694b3a9316
:10e0900054f8103c1e93e3688df8ac30637d022b7e
:10e0a00010d117ad04f114070fcf0fc597e8070083
:10e0b00085e8070028a917a806f01afe98bb0123d7
:10e0c0008df89c30a4f10c070df12c0b3946584605
:10e0d000faf74afc4ff01c0800230222394617a821
:10e0e000cde90e331093fff775ffdde9175308fbf9
:10e0f00003580df1380aa8451cd005f10c030fcbcd
:10e100008de80f00504695e80e00fff72dff1c35f7
:10e110000028f0d117a8fef7eeff0ea8fef7ebffe0
:10e120000ba8fef7e1ff08a8fef7ecff00203db0ca
:10e13000bde8f08f17a8fef7deff3f4bcdf894b097
:10e1400024933e4bcdf8a8a0299323698df8c030c5
:10e1500094f831300a2b13d117ad04f1300cbce820
:10e160000f000fc59ce8070085e807000df1c2010c
:10e1700017a806f0cbfd0028cfd101238df8c130c0
:10e180000df1440821464046faf7eefb4ff01c0a19
:10e19000002339460a2217a8cde914331693fff756
:10e1a00019ffdde917530afb035a14afaa4516d02d
:10e1b00005f10c030fcb8de80f00384695e80e00f3
:10e1c000fff7d2fe1c350028f0d117a8fef793ff09
:10e1d00014a8fef790ff11a8fef786ff9de717a889
:10e1e000fef789ff144b49462c93154b3046cdf86a
:10e1f000b4802f972e9334f05ef90028e8d0304693
:10e2000010491eaa34f083f980340028e0d0384643
:10e21000fef771ff4046fef767ff0ea8fef76bffa3
:10e220000ba8fef761ff08a8fef76cff17e70120b7
:10e230007de700bf45ca0002d1c9000279c90002ca
:10e240001dc90002a4670e021268fff7fdbe0000a0
:10e2500030b5054691b00021144605a81022b6f04d
:10e26000b8fe012328460f4905aa35f056f810b923
:10e27000002011b030bd256809ac2046f9f772fdc9
:10e28000214605a806f012fd0028f1d110ab13e9d4
:10e290000f008de80f00284694e80e00fff764fe9b
:10e2a000e7e700bfa0640e02002330b58db014462e
:10e2b00004930f49012304aa35f02ff810b9002068
:10e2c0000db030bd256805ac2046f9f74bfd214661
:10e2d00004a806f0e3fc0028f1d10cab13e90f0011
:10e2e0008de80f00284694e80e00fff73dfee7e7b3
:10e2f00078640e028842f8b506460c46154618d9d1
:10e30000904217d2a2f18005a1f18007691a441842
:10e31000af4220d02e1d34b120462b68314640f844
:10e32000043bfff76cfa3046f9f7b2fd803d803cc4
:10e33000eee710d0ac420ed0271d36b13046236830
:10e34000394640f8043bfff75afa3846f9f7a0fd82
:10e3500080348036eee7f8bd2de9f041044651f8ef
:10e36000043ba0b0466801a80093fff748fad4e93f
:10e3700001739f4214db0137002f31dd4feac718cc
:10e380004046b6f0d1fd054618b32168a8f18002d9
:10e390000a44fff7afff2068b6f0cefd2560a76006
:10e3a000276862684feac61807ebc616314607ebc6
:10e3b000c21206f18000fff79dff36b1009b01a954
:10e3c00047f80830301dfff71afa0125636801335a
:10e3d000636001a8f9f75cfd284620b0bde8f08134
:10e3e0000025d8e72de9f043536806460c4615464c
:10e3f000a9b033b9d36d23b902f12000f9f7c9fcf4
:10e4000010b9ab69002b76d02b6933b9ab6e23b949
:10e4100005f13c00f9f7bdfc10b9eb69002b6ad09f
:10e42000002720460df107018df807702ef0e6f960
:10e43000041e46db304602a9cde902770497fef7b9
:10e4400083fd041e3adbdde9024705f1700804eba9
:10e45000c717bc429df807303cd022689a4237d19a
:10e4600004f1740105a8fff7abfc414608a8fff7cb
:10e47000a7fc0699099b99420bd1059a089b114468
:10e48000013b914221d012f8010b13f801cf8445d2
:10e49000f7d04ff0000908a8fef734fe05a8fef7f4
:10e4a00031feb9f1000f13d02946201dfff7dcfc27
:10e4b000304602a9fef7aefd00eae07402a8fff7bd
:10e4c0008cf9204629b0bde8f0834ff00109e2e75e
:10e4d0008034bee7294609a80893fff78efc08a9f7
:10e4e00002a8fff739ff044609a8f9f7d1fc002c70
:10e4f000ded1024ce2e7024ce3e700bffcfeffff87
:10e50000e8feffff2de9f0478846b0b0002107463e
:10e51000fef7d8fb002800f08e80002306a80693a3
:10e520002ef056f8002804da444c204630b0bde8fe
:10e53000f087069e414cdff80c91002e6cd070687d
:10e54000002867d0002307a907932ef075f900284b
:10e5500060db079b13f008035cd1756808a92846a7
:10e560000893adf824302ef065fa28460df1170116
:10e570002ef044f98df81700b8f1000f01d0454591
:10e5800048d10222494608a8b8f062fb054660bba4
:10e5900011f086fe2c4618f03dfd002338460aa9ee
:10e5a000cde90a33cde90c33cde90e33fef7ccfccf
:10e5b00030bbdde90a5305ebc31a04352b1f9a451e
:10e5c0001ed09df8172055f8043c93420bd02946e5
:10e5d00011a81093fff711fc10a90da8fff7bcfebe
:10e5e00011a8f9f755fc8035e8e70222144908a87c
:10e5f000b8f02efb0028d0d113f032fa0446cce755
:10e600000da93846fef706fd0da8fff7e6f80aa8a3
:10e61000fff7e3f8366890e706982ef005f8002c2f
:10e6200083d12346022210200021cde90144009429
:10e63000f8f7b6ff79e7044677e700bff2feffff81
:10e6400071df0d02d8d00d022de9f04f2ded028bb8
:10e6500000248146adf5017d702208ee101a22a833
:10e660000021b6f0b6fcb04b0df1180841a83e935e
:10e67000c8e90044cdf8fc80fef737faab4b0bae8f
:10e68000cde930362893aa4b08ad2d93a94b0eaf98
:10e690000df1440a329348460123a74922aac5e94d
:10e6a0000044c6e90044c7e90044cae9004429958a
:10e6b0002e97cdf8cca0ac60b460bc60caf808401e
:10e6c00034f02bfed0b900245046fef714fd384636
:10e6d000fef711fd3046fef707fd2846fef704fd64
:10e6e00041a8f9f7d5fbd8f80000b6f025fc204684
:10e6f0000df5017dbdec028bbde8f08fd8e900126d
:10e7000031b12ab908460591f2f7b4fb02460599e2
:10e710004ff03c0960a8fff73efb5d9b609a609359
:10e720005d925e9b619a61935e925f9b629a60a824
:10e7300062935f92fef7e6fc229b4093d5e900438b
:10e7400009fb0349a14505d0214641a8fff7e8fa96
:10e750003c34f7e74ff03c09d6e9004309fb034995
:10e76000a14505d0214641a8fff7dafa3c34f7e786
:10e770001c22d7e9004302fb03430df5c67b05933a
:10e780000df5c079059ba34226d0a6460df5c07ca9
:10e79000bee80f00ace80f009ee807008ce8070019
:10e7a0006378022b0cd18df881319be80f008de846
:10e7b0000f0057a899e80e00fff7d6fb1c34e1e7dd
:10e7c0000a2bfbd18df881319be80f008de80f00fb
:10e7d0005aa899e80e00efe71c22dde9114302fb7d
:10e7e00003430df5c67b05930df5c079059ba34248
:10e7f00026d0a6460df5c07cbee80f00ace80f00a1
:10e800009ee807008ce807006378022b0cd18df896
:10e8100081319be80f008de80f0057a899e80e00a2
:10e82000fff7a2fb1c34e1e70a2bfbd18df8813105
:10e830009be80f008de80f005aa899e80e00efe75b
:10e840009df8bc3014a847939df8d0304893f9f751
:10e8500089fa1ba8f9f786fa9df8ac30002b47d14e
:10e860009df8d130002b4ad160ac0df1500cbce8c2
:10e870000f000fc49ce807009df8513084e80700a2
:10e88000022b44d18df8813149ac0df5c07cbce838
:10e890000f000fc49ce8070084e8070060ac0df18e
:10e8a0006c0cbce80f000fc49ce807009df86d30ad
:10e8b00084e80700022b30d18df8813149ac0df589
:10e8c000c07cbce80f000fc49ce8070084e8070088
:10e8d000409b41a961a86093fff78ffa18ee100ad8
:10e8e00060a9fff739fd044661a8f9f7d1faebe614
:10e8f00014a92ca806f0d2f90028b1d0e3e61ba990
:10e900000df1d20006f0d2f90028add0dbe60a2bdb
:10e91000c4d18df8813150acb7e70a2bd8d18df82e
:10e92000813150accbe700bf4baf000289db000266
:10e9300029e20002d1e10002a4670e021168fff78c
:10e9400083be8842f8b504460d46164614d9904257
:10e9500013d2a2f17c06751aa1f17c072c44b742b0
:10e9600018d01cb131462046fef749ff3046f9f772
:10e970008ffa7c3e7c3cf2e70cd0b5420ad01cb149
:10e9800029462046fef73bff2846f9f781fa7c35f9
:10e990007c34f2e7f8bd2de9f0410446a0b04668aa
:10e9a00001a8fef72cffd4e901739f4216db013763
:10e9b000002f2fdd4ff07c0808fb07f84046b6f02b
:10e9c000b3fa0546f8b12168a8f17c020a44fff7c2
:10e9d000b8ff2068b6f0b0fa2560a7607c222368f3
:10e9e000616802fb063602fb013206f17c0031460b
:10e9f000fff7a7ff1eb1304601a9fef700ff012572
:10ea000063680133636001a8f9f742fa284620b031
:10ea1000bde8f0810025dce72de9f0430025a9b031
:10ea2000814608460df10b0117461e46ddf8c080f1
:10ea30008df80b502df0e2fe041e3bdb484603a987
:10ea4000cde903550595fef77ffa041e2fdbdde9be
:10ea5000034304ebc3190434231f99453dd09df8ab
:10ea60000b3054f8042c9a4201d08034f4e77eb184
:10ea700004f1700106a80191fff7a2f9079b019923
:10ea800098451bd0002506a8fef73cfb002decd0d6
:10ea9000214609a8fff7b1f9384609a9fff77bff1e
:10eaa000054609a8f9f7f4f9002dded10c4c03a8ae
:10eab000fef793fe204629b0bde8f08309a8fff7d2
:10eac0007ff9424631460998b6f04cfab0fa80f523
:10ead00009a86d09fef716fbd5e70024e7e700bf9c
:10eae000fcfeffff70b5002586b016460a9acde9f8
:10eaf0000355009203aa0595fff78eff041e08db5d
:10eb0000dde903138bb1012b12dc3046fff7acf9c2
:10eb10002c46dde903537c2606fb0356ae420ad0a1
:10eb20002846f9f7b5f97c35f8e76ff0a904f0e766
:10eb30006ff0bd04ede70398b6f0fef9204606b08d
:10eb400070bd2de9f047936807461b780e461446c2
:10eb5000d6b000f10808002b00f0328137a8fdf78d
:10eb6000c4ffa36831469a68384600925b6837aaaa
:10eb7000fff7b8ff3d9b012b0cd81422002128a8d9
:10eb8000b6f027fa0023042100933046142328aa64
:10eb90002ef09afaddf8f490b9f1010f40f084807c
:10eba0000df14c0a142200215046b6f012fa02224e
:10ebb00037a928a8fff70efa299c28a8fef79bfa88
:10ebc000002c50dd1c2537a902228af8109028a8b5
:10ebd000fff700fadde92843002105fb0345ac42bd
:10ebe0000bd0304601f101092cf0eef90146204628
:10ebf0002cf0f7f81c344946f1e728a8fef77bfa19
:10ec000001239df8fd90b9f1020f2ed121ac3fad4b
:10ec10000fcd0fc495e8070084e8070021ac94e805
:10ec20000f008ae80f00182200211aa8b6f0d1f9c7
:10ec300028a8f9f797f800211c2228a8b6f0c9f9ee
:10ec400028ab30461aa9cde91a338df8a1901c944f
:10ec50002df0b8ff002352460093042114233046c0
:10ec60002ef032fa03e00023cbe7002bf2d13d9bdc
:10ec7000012b04d84ff4803130462df08ffe4046f2
:10ec8000fef747fa052840f08e8006213846fef749
:10ec9000abfa3846fef7c6fc37a8f9f7f9f856b0d4
:10eca000bde8f047fdf748beb9f1020fdfd137a943
:10ecb00028a8f9f759fe299c28a8fef715fa002c78
:10ecc000d5dd4ff4803130462df064fd182200214f
:10ecd0000deb0200b6f07df937a921a8f9f744fe43
:10ece000ddf884c028ac65460fcd0fc40fcd0fc42e
:10ecf0000fcd0fc495e8070084e8070021a89cf811
:10ed000038a0fef7f1f90df1300c65460df14c0e0f
:10ed100028ac0fcc0fc594e80700744685e80700bf
:10ed20002fad0fcd0fc495e807003fad84e8070075
:10ed30001aaccde906ce8df828a00fcd0fc495e80a
:10ed400007004ff01c0a84e807001aab06a93046fa
:10ed500008932df037ff4a4637a903a8fff73af981
:10ed6000dde903324ff0000c99460afb023aca452e
:10ed700015d04d4621ac0fcd0fc495e8070084e8af
:10ed80000700614630460cf101042cf01df90146e4
:10ed900021a82cf026f809f11c09a446e7e703a8ee
:10eda000fef7a9f963e74046fef7b3f907283ff4f9
:10edb00070af4046fef7adf906287ff46daf68e707
:10edc0004ff4803130462df0e5fc31463846fef7f1
:10edd0009bf831463846fdf707ff4046fef799f9a4
:10ede000072808d141213846fef738f850b1384697
:10edf000fef718fc53e74046fef78bf906287ff430
:10ee00004eafefe705213846fef7eef947e7136806
:10ee1000033b052b0ed8dfe803f00305070d090bb4
:10ee2000fef7d5bbfff78dbefef7c1bcfef7d0bd28
:10ee3000fdf7eabe7047fff7eabff7b5174613f0d4
:10ee4000010205460e461c4605d10b460120052150
:10ee5000009202f0c5fd032d0ad0042d0cd0022d26
:10ee60000dd1c4f3400010f073fb002003b0f0bddf
:10ee7000002010f055fbf8e710f040fbf5e700220a
:10ee80003946304610f02cfbefe700680179d0e9f5
:10ee900002230078fff7d1bf012a70b5054603d1e0
:10eea0000b680360002070bd022a08d0032af9d144
:10eeb00000680028f6d010211af032fdf2e7102089
:10eec0000e681af025fd044618b196e80f0084e894
:10eed0000f002c60e6e7000010b5012400220d4b66
:10eee0001c700d4b1a70fdf7fbf9d0e8cf3fc0e85e
:10eef000424f002af9d1dbb2002bf6d1c268036180
:10ef0000c36003754375c0e88f3fd30758bf037aca
:10ef100010bd00bf585100102ed200100022014b2e
:10ef20001a70704758510010024b1878003818bffb
:10ef300001207047585100100b4b28b91a788ab934
:10ef400001221a70fff7c8bf0328187008d80128db
:10ef5000f8d00022054b1a700122054b1a7001e00f
:10ef60000428efd0704700bf59d40010585100104a
:10ef70002ed20010014b1878704700bf59d40010f2
:10ef8000014b1870704700bf58d40010014b18781f
:10ef9000704700bf58d40010f0b51c46431e032b29
:10efa00006460d46174685b04fd8294ad35c00293e
:10efb00008bf1d46274b5b68c3f308035bb144f0f1
:10efc0000104e9b223463a46f0b2fff736ff0025c6
:10efd000284605b0f0bdf7f7bffa0028efd0fdf7df
:10efe0007ff9037a002bead0e307ead41a4b93f8af
:10eff0006c20002ae5d0586e25f071f90028e0d188
:10f00000029010201af084fc18b1c0e90065c0e934
:10f010000274124b00900393114b69460e48029301
:10f02000f4f746fc044670b100224ff0ff3140690e
:10f0300025f088fa236820469b68a56998476846aa
:10f04000f4f732fbc4e70546f9e7064dc0e700bf19
:10f0500088d20d0200ed00e078ce00100bee000229
:10f0600019ee0002f2feffff03681b68184710b597
:10f0700003681446db689847031b5842584110bd8b
:10f0800008b54068fff7f3ff08bd70b5037a044682
:10f090000d4616462bb9d0e90312fff7f1ff012305
:10f0a0002372324629462046fff7eaff70bd7047bb
:10f0b00070470139012908b505d80021083000f052
:10f0c00055fb012008bd0020fce70022012110466d
:10f0d000f9f7e6ba10b50446fff7e9ff20461c2110
:10f0e0001af01efc204610bd08b50021022002f0d7
:10f0f00035ffbde8084025f0f5b9000008b5074820
:10f10000f9f78eff064b586e25f0e9f820b9bde8f7
:10f1100008400448f9f73ebf08bd00bf4cf6001098
:10f120005cd5001078ce0010002108b5022002f056
:10f1300015ff25f0def9b0fa80f0400908bd08b5ea
:10f140000021022002f00affbde8084025f0d9b9ed
:10f1500038b500f1080504462846fff7e5ffe8b199
:10f16000284607f052fcb0b1284607f03ffc011ecc
:10f1700011db236820465b69c9b2984758b9284615
:10f1800007f043fc38b1284607f028fc2368c1b2d9
:10f190001b69204698472846fff7d1ff38bd00007d
:10f1a00010b50446d0e90512024b0360fff76dff6e
:10f1b000204610bd1cd40d0238b50c46054601464c
:10f1c0002046b5f0dffe28461349f1f749fe28b97d
:10f1d00012492046b6f0cdff002038bd2846104920
:10f1e000f1f73efe08b90f49f3e728460e49f1f75b
:10f1f00037fe08b90d49ece728460d49f1f730fe16
:10f2000008b90c49e5e728460b49f1f729fe002823
:10f21000e2d10a49dde700bf8cd20d0291d20d0286
:10f2200096d20d029cd20d024bcf0d02a2d20d023e
:10f23000b0d20d02b3d20d02c1d20d02c8d20d025e
:10f2400038b504460b4b054644f8083b204607f00a
:10f2500023fcfff749ff2046fff771ff204607f028
:10f260000ffc20b94ff41651204607f005fc284644
:10f2700038bd00bf28d40d0270b50d46002400f142
:10f2800008062846f1f7f6fda04205d9295d30466b
:10f2900007f0c2fb0134f4e770bd000037b5044647
:10f2a0000b4b00f1080528460093002307f0d8ff18
:10f2b00020460849fff7e0ff284607f0a6fb002894
:10f2c00003dd284607f08afbf6e703b030bd00bf38
:10f2d0007df000023f030f022de9f0436929044647
:10f2e000a5b070d1142500212a4607a8b5f071fefb
:10f2f0000022012107a8adf81c5010f06bfe00257c
:10f300002023cde90c35bdf82c30012001938f4b23
:10f310008f4900930caa2b46f3f7befabdf82c30a8
:10f32000002b3fd08b492046fff7a6ff03a8f7f735
:10f3300039f920460399fff79fff20468649fff7da
:10f340009bff2427dff85482dff80c92bdf82c30a5
:10f35000ab421cdd07fb05f60a9b142298590ca949
:10f36000fff72aff88b920460ca9fff785ff414621
:10f370002046fff781ff0a99204631440431fff708
:10f380007bff49462046fff777ff0135dee703a8fc
:10f3900008f026f9002207a8114610f01bfe25b040
:10f3a000bde8f0836d492046fff766ff0ca8f7f72c
:10f3b000f9f820460c99fff75fff20466649fff7f2
:10f3c0005bff0ca8e4e76d293ed16549fff754ffc8
:10f3d0005d2200210ca8b5f0fcfd0022052011469d
:10f3e000f8f78cfe014638b102882ab15d2a28bfa1
:10f3f0005d220ca8b5f0c6fd01220df1870107a81a
:10f40000fcf742ff20460799fff736ff07a808f0f0
:10f41000e7f80525534f0df18d0639462046fff7d5
:10f420002bff0122711b07a8fcf72eff204607992e
:10f43000fff722ff07a808f0d3f8013dedd12046e1
:10f440004549fff719ffaae766290bd10834204682
:10f45000454907f08cff0021204625b0bde8f04368
:10f4600000f084b9782905d10368db6825b0bde8d0
:10f47000f0431847732916d13c4b00220c933c4ba8
:10f4800008340f93012310933a4b0ca911930323d3
:10f4900039480d948df838201293fbf781f90ca8a8
:10f4a000fff77efe7be7762908d1344b0c9300f101
:10f4b00008030ca80d93fbf795f9c0e74c290ad176
:10f4c00000220121042000f0e1f8002025b0bde871
:10f4d000f04308f0dab9632910d100201ff0dbf9fe
:10f4e000054627492046fff7c7fe2649264b002d33
:10f4f00008bf19462046fff7bffea0e7432917d1f2
:10f500002249fff7b9fe3f2220460ca9fff7c6fead
:10f510000ca8f1f7affc3f2808d10ca81ff07cf92c
:10f520001b492046fff7a8fe0ca9e3e71949e1e7cc
:10f5300064297ff434af002200f1080300931146e0
:10f540001046154b0192fbf755f978e7e2d20d0210
:10f5500060c30d0202d30d023f030f020ed30d0252
:10f5600021d30d02e9d40d023ed30d021cd40d02ad
:10f5700013f20d027ed30d02e9ef000210d40d024a
:10f5800082d30d02dbd20d02dfd20d0293d30d0226
:10f59000afd30d02c3d30d02efef000226ed0d0233
:10f5a0004ff0ff30704738b51546d0e9022393423b
:10f5b000044607d2d21a4068aa4228bf2a461844f5
:10f5c000b5f0e0fce26801202a44e26038bd012a7f
:10f5d00002d1016000207047022a04bf0b6803605b
:10f5e000f8e713b5044608460191f1f743fc0246db
:10f5f0002046236801991b6802b0bde810401847f7
:10f6000004281fb5034614460cd14ff6ff7345f688
:10f610001b210920002a08bf194604b0bde810408c
:10f6200010f0ecb901280ed100233c2200931123e5
:10f6300012481349002c18bf014612480068f7f71a
:10f6400077fb04b010bd09280ad100230b480c49f0
:10f650000093002c18bf014611233c220a48ede715
:10f660000028eed1002aecd00246cde9010000903e
:10f6700000214ff40070f7f793ffe2e73bca0d0259
:10f680000a370e025c5100106051001009280a462a
:10f6900008b50dd8084b195c914203d1042801d05c
:10f6a000082803d1195c1a54fff7aaff002001e0d3
:10f6b0004ff0ff3008bd00bf6d510010092838b56c
:10f6c0000c4613d8a9b104280b4d0cd1092010f019
:10f6d0009ff945f61b2380b2c31a58425841207047
:10f6e0002871002038bd2b5c0b70fae74ff0ff301b
:10f6f000f8e70846f6e700bf6d51001037b5002265
:10f700000df107010546fff7d9ff044628b99df81a
:10f71000072028461146fff773ff204603b030bd8f
:10f72000014b1860704700bf60d4001038b50b4b18
:10f7300045681c6864b100f1080100222846a04712
:10f74000044618b10649284607f011fe204638bd88
:10f750000449284607f00bfe0349f4e760d4001083
:10f7600044d40d0272d40d02a8d40d020c4a0d4be4
:10f7700000b51a601c2389b00021adf804301423b1
:10f78000029001a8cde90311cde90511adf80610ed
:10f790000791adf80c30fff7c9ff09b05df804fb25
:10f7a000955c000260d4001010b50f4b04461b6836
:10f7b000834208d1002301211a461846f8f745fd77
:10f7c000002008f047f8002211461046f8f7a0fd87
:10f7d000024640b9054b1b68a34204d1bde8104066
:10f7e0000146f8f75dbf10bd64510010685100106c
:10f7f00030b50d4b05469b7885b003f0ff0483b907
:10f80000224601210220fff741ff084b22461d70ce
:10f810004ff4806023460021cde901440094f7f7be
:10f82000bffe05b030bd00bf6d5100106c5100101f
:10f8300013b50024022022460df107018df8074080
:10f84000fff73cff9df8070060b1224603200df151
:10f8500007018df80740fff731ff9df80700001bf7
:10f8600018bf012002b010bd07b5fff7e1ffa0b13e
:10f870000b4b1a7802f0ff0342b1002302201a4614
:10f88000194603b05df804ebf4f7d5b805490093c9
:10f890001a4601200978fff77ffb03b05df804fbef
:10f8a0001dd600106c510010f0b585b0fff7c0fff9
:10f8b00048b3164d2b7833bb01222a70144a4ff4fb
:10f8c00000600021cde9013300921a46f7f768fe87
:10f8d0001df0d1ff47f22f5704460e4efff7a8ff49
:10f8e00030b90020287005b0bde8f040fff7bcbf7c
:10f8f0001df0c1ff001bb842f3d8f6f73dfe3046bd
:10f90000f9f748fbeae705b0f0bd00bf64d400108a
:10f91000e9f7000278ce001037b5837a04460d4629
:10f92000ebb91ef089fd636818442389206113b97f
:10f930001ef08efd2081e36813b91ef083fde060a8
:10f9400015f0010f0cbf00250425faf735f8002348
:10f95000e1681a460095faf745fb03b030bd01484f
:10f96000fbe700bfe2faffff2de9f0411646ca07a8
:10f9700088b038d511f0020f0cbf00240424faf728
:10f980001bf82146faf7aaf914f00805074626d114
:10f9900006b34ff0ff08294642463046b5f019fb42
:10f9a000124b134904a8cde90436cde90685fff7cb
:10f9b00018fe3b460c210f4a01a8cde901550395dd
:10f9c000b6f03efb01a904a8fff70bfe0a4904a804
:10f9d000fff707fe630702d44620fff709ff38460a
:10f9e00008b0bde8f0810824c9e700bff8d40d02d3
:10f9f000e5d40d02e3cc0d02ebd40d0230b5044684
:10fa0000002585b00391f9f7d7ff62682369039950
:10fa1000d31a00952289faf7a1f905b030bd00008c
:10fa200070b5324e044696f86c3086b0002b49d043
:10fa3000706e24f054fc0546002843d12c4b1c204a
:10fa400005932c4b0294049319f062ff044600289e
:10fa500031d0294bc5600360049b3bb1022202a94f
:10fa600004309847059b2361049be36000252046f2
:10fa7000224b2a462360012140f8145f24f052fdf6
:10fa80001f4b01a92360f2692b46306f019424f0cb
:10fa90009efc014650b9706e08b124f067fc00224c
:10faa0004ff0ff31606924f04dfda56923682046c1
:10fab0009b68984700e0054602a8f3f7f5fd284645
:10fac00006b070bdf9f778ff037e63b90d4b1b7864
:10fad00003f0ff05002bf2d00b4b1b78002b0cbf63
:10fae00001250225ebe70325e9e700bf78ce0010ea
:10faf0008dfa00024ff50002f4bc0d0208bd0d02a4
:10fb00001cbd0d025fd400106d5100100068fff79e
:10fb100087bfd0e88f0fc0b2003818bf01207047f0
:10fb20000048704768d4001008b5fff7f2ff08bd21
:10fb30007fb50546fff7edffe0b1686810b10368d7
:10fb40009b6898471df097feeb68c01ab0f57a7f66
:10fb50000ed31df090fe00240646aa682346821aa2
:10fb600000210420cde901440094f7f719fdee606f
:10fb7000002001e06ff0d10004b070bd38b5142052
:10fb80000d460021144602f09ff9014640b1054b95
:10fb90000573046143600448f9f728fa002038bd72
:10fba0000248fce755fd00024cf60010fcfeffff8a
:10fbb00030b58bb0fff7adff002857d000242023cd
:10fbc000cde902342b4b1e202b49009302aa234679
:10fbd000f2f762fe21460920f7f750fa08b30469ec
:10fbe000002214210120f7f753fa282202210346ac
:10fbf000cde9002102a82146012207f069fe00227a
:10fc0000012103a8f2f72cff1a24013c0bd09df828
:10fc10001a30322083f002038df81a301af03ffeba
:10fc2000f3e7ff24dce7fcf79fff2146fef76afcc1
:10fc30000446a8b14ff47f031a2507939df81a30a4
:10fc400003f0fd038df81a30013d09d09df81a30fc
:10fc5000322083f002038df81a301af020fef3e709
:10fc600002a8fbf7fff920460bb030bd6ff0d104be
:10fc7000f9e700bf49d50d023bd50d0203680160cd
:10fc80001bb11a68184652681047704730b58db0de
:10fc90000546fff76ff9042807d12846fff739ff1b
:10fca000044650b16ff0d10045e009200ff058fd37
:10fcb0000028f2d06ff081003de00123c5e88f3fbe
:10fcc0002023cde904301d4b1d49009304aa0346af
:10fcd0001e20f2f7e1fd2346224604210120009474
:10fce00001f07efefcf740ff0721fdf71dfc2346d7
:10fcf0002246a2210920f7f70df9234622460021ca
:10fd00000220cde901440094f7f74afc1df0b3fd51
:10fd1000c5e9020000f0bef800f0c0fc1c2019f09c
:10fd2000f7fd044610b104a9fff78afa281d214601
:10fd3000fff7a4ff00200db030bd00bf63d50d025a
:10fd40003bd50d0230b58db00546fff7e2fe48b356
:10fd500000242023cde90434144b04aa00931e2070
:10fd600023461349f2f798fd224621460920f7f76a
:10fd7000e3f82146281dfff781ffc5e88f4f1df0ee
:10fd80007afdaa682346821a00210820cde90144a1
:10fd90000094f7f705fc00f07df800f013f9204619
:10fda0000db030bd6ff0d100fae700bf7bd50d027a
:10fdb0003bd50d02022906d0032906d0012906d120
:10fdc0000021fff763bffff7bdbffff7f1be6ff084
:10fdd0007700704713b5047b02690021019202f09d
:10fde0009df82146019a034802b0bde81040fff794
:10fdf000e1bf00bf68d400100022024b1a705a60a5
:10fe0000704700bf68d4001010b50378044613b1e2
:10fe1000002026f005fa204610bd00004ff0fa73ce
:10fe2000194a10b5c0e90023184b00f10d02836098
:10fe300000230373164b03f1100153f8044b8b425c
:10fe400042f8044bf9d102220023426540f262627b
:10fe5000c0e90833c0e90a33c0e90c33c0e90e3306
:10fe6000c0e91733c0e91933c0e91b33036480f8d4
:10fe70004430c0f84630c0f84a30c0f84e30a0f8e0
:10fe80005230a0f8582010bd18002800200064004f
:10fe900003af0d0210b50a4cd4e88f3fdb070cd43a
:10fea00020461bf02bff40b10648fff7b7ff204666
:10feb0001bf05eff0448b4f03efe024810bd00bfd8
:10fec00078d400107cd400104902010290f8570049
:10fed000704780f857107047a0f8581000207047fe
:10fee00073b5374b05461e78002e65d130468df828
:10fef000046026f067f9d5e90801012332468df840
:10ff0000043028f0c7f9041e2bdbd5e90b0132467b
:10ff100028f010fa041e24db314605f1460026f0d5
:10ff20007efa041e1ddb314605f1380028f064f925
:10ff3000041e16db314695f9440026f0befa041e75
:10ff40000fdb314695f8540026f021fb041e08db38
:10ff500095f8521059b13146304628f035fb90b132
:10ff6000002401a8fff750ff204602b070bd95f8ad
:10ff700053306bb1084628f027fb0028f0d195f8e4
:10ff80005430022b14d128f0f5f900eae074e8e7c8
:10ff90001946184628f018fb50b195f85430022b3a
:10ffa000ded10120002185f8540026f0f0faece7bc
:10ffb000002026f00afbe8e76ff0d104d4e700bf89
:10ffc0007751001070b51b4e044635788cb06dbb70
:10ffd00028468df80c5026f0f5f801232a462146d4
:10ffe00015488df80c3026f06ef9284626f042f9b7
:10fff00094f8563083b1204684f85650fff770ffce
:020000040807eb
:1000000050b12023cde904350c4b322000930c492c
:100010002b4604aaf2f740fc01233370002303a807
:10002000636223632366e366fff7eefe00200cb0f5
:1000300070bd00bf77510010b1010102a4d50d02bf
:1000400092d50d02f0b52d4b06461d7889b0002dd6
:1000500050d128468df8045026f0b4f801232846e4
:100060008df8043026f006f9041e38db0c2733889f
:100070002946adf80c30738802a8adf80e30f3882d
:10008000adf80850adf81230b388adf80a70adf88d
:10009000103026f0c4f9041e21db33892946adf85f
:1000a0001830738905a805950795adf81670adf859
:1000b0001a3028f0a1f8041e11db2946022026f090
:1000c00066fa041e0bdb294696f90c0026f0f5f9ba
:1000d000041e04db284626f0c5f8041e08da304664
:1000e000fff770ff01a8fff78ffe204609b0f0bdb3
:1000f0002c46f7e76ff0d104f7e700bf7751001007
:10010000037a2bb903681b7813b94068fff75abf0d
:1001100070470000f0b52a4b05461b7885b0002bd0
:100120003fd190f8523013b990f85330cbb395f8d3
:1001300055607ebb012730468df8006026f042f8fe
:100140000df103033046cde901358df800708df8cf
:1001500003608df80c6026f08df8041e24dbd5e9d1
:100160000801324628f096f8041e1ddbd5e90b0184
:10017000324628f0dff8041e16db304626f072f80f
:10018000041e11db01a88df80370fff7b9ff684664
:10019000fff73afe95f8553083f0010385f85530a6
:1001a0005bb96ff0d10405e001a8fff7a9ff68462d
:1001b000fff72afe204605b0f0bd0024fae700bf95
:1001c0007751001073b5194b06461d7855bb28466c
:1001d0008df8045025f0f6ff012328468df80430f1
:1001e00026f048f8041e12dbd6e917012a4628f04b
:1001f00051f8041e0bdbd6e91a012a4628f09af8ba
:10020000041e04db284626f02df8041e08da3046ca
:10021000fff7d8fe01a8fff7f7fd204602b070bd3a
:100220002c46f7e76ff0d104f7e700bf77510010d5
:1002300030b5144b0c461d788bb0adb90368012b5b
:1002400012d10846fff766ff80b12046fff7baffdc
:1002500060b12023cde902350b4b00932b463220b1
:100260000a4902aaf2f718fb0bb030bd002028f0b3
:1002700081f80028f8d020220023cde90223044a87
:100280000092ece777510010cad50d0292d50d020d
:1002900000d60d0210b504460068b4f04dfe2046ad
:1002a00010bd10b504466830fff7f4ff04f15c00a0
:1002b000fff7f0ff04f12c00fff7ecff04f1200042
:1002c000fff7e8ff204610bd0148fff7eabf00bf77
:1002d0007cd4001003680a6802600b6043684a68b7
:1002e00042604b6083688a6882608b60704700233d
:1002f00010b50446c0e900338360fff7ebff2046ea
:1003000010bd38b50d1e0446006803ddb5f0e2fdf2
:1003100018b938bdb4f010fe00202060a56001209f
:10032000f7e770b500260d1e0446c0e9006686603a
:100330000bddfff7e6ff40b123685a199a4203d05c
:1003400003b11e700133f9e76560204670bdf8b552
:10035000d0e901539d4204460e460cda27686268d4
:100360007919521b481cb4f01afe01207e556368af
:1003700001336360f8bd691cfff7c3ff0028edd1ae
:10038000f8e72de9f041476883688846b918994233
:100390000446154612dc266862683e443146d21b8c
:1003a0007019b4f0fcfd2a4641463046b4f0eafd2f
:1003b000012062682a446260bde8f081fff7a1ff76
:1003c0000028e8d1f8e7000070b5674b06461c78b6
:1003d00098b0002c40f0c580022104a8cde9044467
:1003e000cde90644cde90844fff7b1ff48b95f4db8
:1003f00007a8fff74fff04a8fff74cff284618b0e7
:1004000070bd012104a8fff7a2ff0028efd006214c
:1004100004a8fff79cff0028e9d01122214613a869
:100420001294b4f0d6fd2246152112a825f0b9ff8a
:10043000051edddb12a8f0f71dfd0130c1b204a8d6
:10044000fff785ff0028d2d0092104a8fff77fff1e
:100450000028ccd012a8f0f70dfd12a9024604a87e
:10046000fff78fff0028c2d01c23adf80430b6f888
:100470005830062102a8adf806300294adf80c40c1
:1004800021f078fa051eb3db0b2104a8fff75fff0c
:100490000028acd0ff2104a8fff759ff0028a6d000
:1004a00002220df1060104a8fff76bff00289ed081
:1004b000022201a904a8fff764ff002897d00622b2
:1004c00002a904a8fff75dff002890d001f01afef2
:1004d00000f118010da803f091f89df84430012bac
:1004e0002fd1112107a8fff732ff00283ff47faf7b
:1004f000072107a8fff72bff00283ff478af102251
:100500000da907a8fff73dff00283ff470af04a92d
:100510000aa8fff7ecfe0aa906f15c00fff7dafe75
:100520000aa8fff7b7fe07a90aa8fff7e0fe0aa985
:1005300006f16800fff7cefe0aa8fff7abfe002524
:1005400056e7032107a8fff702ff00283ff44faf4b
:10055000032107a8fff7fbfe00283ff448af022263
:10056000cee76ff0d10549e777510010fcfeffffa1
:1005700038b5436805468b420c4612da83689942c7
:100580000adcd5e900230021134422449a420ad010
:1005900003b119700133f9e7fff7b3fe0028f0d17a
:1005a00038bd0029fcdb6c60fae70000f0b53a4b7f
:1005b00005461e788bb0002e6ad11f2101a8fff7d7
:1005c000b0fe1f2104a8fff7acfe32461f210198a0
:1005d00025f0a9ff041e52db214601a8fff7c8ff42
:1005e00032461f21049825f0b8ff041e47db0c2774
:1005f000214604a8fff7bcff31466f8705f138009c
:1006000025f079ff041e3adb314605f1440025f060
:1006100067ff041e33db3146a5f8487005f146003c
:1006200025f01bff041e2adb314605f1540025f09e
:10063000c1ff041e23db304625f0e4ff314685f878
:100640005200304627f0c0ff01a985f8530007a8e3
:10065000fff74dfe07a905f12000fff73bfe07a8b5
:10066000fff718fe04a907a8fff741fe07a905f147
:100670002c00fff72ffe07a8fff70cfe344604a856
:10068000fff708fe01a8fff705fe20460bb0f0bdfe
:100690006ff0d104f9e700bf7751001037b500249f
:1006a000264b054620461c708df8044025f08afd37
:1006b000012320468df8043027f026ff20b10a20c0
:1006c0001f4a2049f0f794fc002025f0cbfd041ec2
:1006d0002fdb2846fff778fe041e2adb2846fff7ab
:1006e00065ff041e25db0123284685f85630fff7f9
:1006f00069fd041e1ddb2846fff7a4fc041e18db61
:1007000000222946104825f0c3fd041e11db95f890
:10071000523033b1002401a8fff776fb204603b026
:1007200030bd95f853000028f4d127f023fe041eb5
:10073000f0da2846fff746fcede700bf77510010de
:1007400023a8020223d60d02b1010102c06870473e
:10075000c2684068101a704710b500200c461df0a2
:100760007df84ff47a720023f0f7d6f9206000206c
:1007700010bd70b5202488b0224606460d46684656
:100780000021b4f026fc00216846adf800400ff0cf
:10079000c5f8044630b96846b369984728602046d2
:1007a00008b070bd6ff06300fae70000012208b5e1
:1007b000094b1a70fef7defb01280cd1f5f7ccfed1
:1007c00028b9064b1b7813b9054b1b781bb1bde844
:1007d0000840faf77fbd08bd1cd600105cd400109d
:1007e0005bd40010fff7e2bf438c8b422cd890f80b
:1007f0002030012b16d0022b11d03bbb90f82430b7
:10080000013bdbb280f82430c3b1012380f82030f3
:100810004ff4af7343844ff420634361704790f803
:1008200024203ab1002380f82030322343844ff44f
:100830007f43f2e711460430f2f712b9022380f841
:10084000203040f2ee23e5e75b1a43847047012a2b
:1008500008bf01600020704710b50446024b0360da
:10086000faf700fc204610bd18d70d020148fff72b
:10087000f3bf00bfd0d5001010b50446fff7ecff62
:100880002046282119f04cf8204610bd10b504462a
:10089000024b0360faf7e6fb204610bd2cd70d0291
:1008a0000148fff7f3bf00bffcd5001010b50446a8
:1008b000fff7ecff2046202119f032f8204610bd4a
:1008c000028c00230421703023f076bd024610b55f
:1008d00008b1002010bd0146f7f71afd0028f8d135
:1008e000054c23889bb2002bf3d01cf0c4ff238857
:1008f000c01a80b2eee700bff8d4001070b58cb01b
:100900002a4904a805f0e0ff04a806f0f3fbb5eec1
:10091000c00af1ee10fa47db04a806f0ebfbb3eed9
:10092000047ac0ee077af8fe677afdeee77a17eef2
:10093000905a1f4ed6e88f2f12f001021d4c1cd189
:10094000304603921bf0daf9039ab0b114210f205c
:10095000f6f79efb1e2202210346cde90021204628
:100960000f226ff07f4106f0b3ff134b3046236038
:100970001bf0fef91148b4f0def8002210481146d1
:10098000f2f76ef8022384f8203040f2ee236384fd
:100990004ff4206300220121094884f82450636148
:1009a000f2f75ef80cb070bd0025c2e7a4f70010a6
:1009b000f0d40010d0d5001018d70d02ed070102b9
:1009c000d4d5001008b50023a2211a460c20f6f752
:1009d000a1fa0122024b1a70bde8084001f068ba82
:1009e0001dd6001010b5094c2378012bdab204d0c3
:1009f000022a07d00023237010bd0028fcd1fff786
:100a00007dfff7e7fff7defff4e700bffad4001041
:100a10001fb5002310490a780b70104902f0ff043b
:100a20000b60bab101220093cde901324ff40050be
:100a300022460021f6f7b4fd094b1c70094b58689b
:100a4000c0f30800003818bf012004b0bde8104012
:100a5000fff7c8bf04b010bd00d5001004d50010ca
:100a6000fad4001000ed00e030b51d2885b025d97e
:100a7000b0f5fa7f04d305b0bde83040fff7c8bf3a
:100a8000104c23780133dbb223702378042b17d862
:100a90001cf0f1fe4ff47a7200250b4b18600b4be3
:100aa0001a60002301214ff48050cde901312278f2
:100ab00000210093f6f774fd002ddcd105b030bda8
:100ac0000125eee700d50010fcd4001004d500107d
:100ad0007fb506462a4de0b1002211461046f7f7d1
:100ae00017fc284c20701cf0c6fe80b228802278ab
:100af00002f0ff0342b901228020cde9013200213a
:100b00001a460093f6f74cfd00221f4b1a7004b0f2
:100b100070bd2b889bb2002bf9d01cf0acfe2c884a
:100b20003246041b31463046a4b2f7f7f1fb60b9f8
:100b300001230090cde901032246034600218020d5
:100b4000f6f72efd2046fff78fff41f28633002295
:100b5000a4f6b934a4b29c422a80d8d8094b1b7899
:100b6000002bd4d011461046f7f7d2fb0022002804
:100b7000cdd00121104604b0bde87040f7f790bd1c
:100b8000f8d4001008d5001009d50010012802d8ab
:100b90000846fff79dbf704710b5314c2288013ad7
:100ba00092b222802ab911461920f1f7c5ff192304
:100bb00023802c4c2388013b9bb22380b3b9fbf7e5
:100bc0000df94ff47a732380274c1af05bfb2368ee
:100bd000002b43d01cf04ffe244b1a682368801a68
:100be00098423bd9bde81040fff712bf00221146e2
:100bf0001046f7f78dfb80b142f210700ef05dfced
:100c000058b11b4b197801f0ff0231b90121104690
:100c100019700321f7f784fbd6e70022114610462e
:100c2000f7f776fb0028cfd140f6b8300ef045fc40
:100c30000028c9d00f4b1b7803f0ff04002bc3d151
:100c400001f036f92046fff743ff204622462146b1
:100c5000f7f726fd0120fff73bffb5e710bd00bf0a
:100c6000785100107a51001004d50010fcd4001007
:100c700009d5001008d5001013b501200ef082fe32
:100c8000ff281ed0c3071cd50420fef755f900210c
:100c900000240846fef774f9224604200df10701ee
:100ca0008df80740fef70afd9df807304bb122464c
:100cb00021460420fef7eafc224621462046f7f7ab
:100cc000effc02b010bd000010b50446fef752f96b
:100cd000022801d0002010bd002cfbd1fef724f922
:100ce0000028f7d0f5f738fc0028f3d1024b18782c
:100cf000b0fa80f04009eee72ed2001030b50d4d6d
:100d000002462c7885b034b108200b4a0b49f0f725
:100d10006ff9b3f009ff01234ff48020cde90143bf
:100d20002b70002123460094f6f73afc2c7005b096
:100d300030bd00bff8d5001023a8020265d60d0211
:100d400001287fb50c463fd00a2843d1224dd5e873
:100d50008f2f12f001021cd1284603921af0ceff09
:100d6000039ab0b114210220f6f792f902221e2153
:100d70001a4e0346cde9001230466ff07f4106f06f
:100d8000a7fd174b284633601af0f2ff1548b3f061
:100d9000d2fe14f0010212d000210846f6f76ef9d7
:100da00050b10369002201210c484361043004b0b2
:100db000bde87040f1f754be6ff07f43f2e7a30740
:100dc00008d511460848f2e7084604b0bde870406f
:100dd000fff794bf04b070bdf4d40010fcd5001030
:100de0002cd70d022108010200d6001070b5044670
:100df00086b0062018f05cfb002c65d1204600f080
:100e0000c3ff3e4b1b78002b5ad1fef78df800280c
:100e100056d0f5f7a1fb002852d1394b1b78002b97
:100e20004ed1fef7a7f801284ad106b070bdfef7f3
:100e300077fefef779fe0028f7d14ce0072018f086
:100e400037fbfef797f8042801d0f0f799f8012353
:100e50002c4e2b7096f86c303bb9fff7a7fc204660
:100e6000fff732ff0028e0d139e0706e23f037fa47
:100e700005460028f1d1244b14200593234b0493fd
:100e800018f046fd044690b1214b02a940f8043bfe
:100e9000f5f744f81f4b3046236001a90194f4f79d
:100ea000c6ff40b1706e10b1294623f05ffa02a868
:100eb000f2f7fafbb9e7236820469b689847f6e704
:100ec000154b1b78002bb0d12046fff7fdfe002804
:100ed000abd1002cabd00a4d2b78012baed1082022
:100ee00018f0e6fafef746f804289ed0f0f754f81a
:100ef000092006b0bde8704018f0daba2ed2001012
:100f0000f9d5001078ce001065070102cf07010265
:100f100008c40d021cc40d025ed400100120fff7ae
:100f200065bf10b50446006808b118f0f7fc20460c
:100f300010bd000030b593b02bf026fbf0f714f88d
:100f40000ef03cfa002000f08ffa052018f0b0fafd
:100f500000232a211a461846f5f7dcff30f094fded
:100f60006e4bda88012a51d100249c71dc7130f07b
:100f7000a7fd2023cde90a34694b0aaa6949282034
:100f800000932346f1f788fc16f044f810f094fb28
:100f90006549c020b3f074fa634906908020b3f02d
:100fa0006ffa06990a9059b350b3c02240f6224016
:100fb00019f09afda04223db802240f6a2300a9964
:100fc00019f092fda0421bdb19f0f8fda04217dbdf
:100fd000c02240f62241069819f0bbfda0420fdb6b
:100fe000802240f6a2310a9819f0b3fda04207db37
:100ff000f4f7f0f8f4f7e4f9fbf7b6fdfbf798ff28
:101000000aa8fff78eff06a8fff78bfff2f702fa98
:1010100000220024202511460220f1f73dff06a8fa
:10102000f5f7c0fa069b3f490193404b0aaa1e20e0
:1010300000932346cde90a54f1f72efc204629f00f
:101040009ff829f0a1f8224601203649f1f7e2fc89
:10105000b0b1224605a904a8cde904440ef0defa99
:1010600070b9049b63b1059acde90a50cde901320c
:101070002f4b2c4900930aaa03460120f1f70cfce0
:1010800018f01efe01f03ef801f026f8fff7f4fd1f
:1010900021f08afb274821f03dfd0020fdf776ff77
:1010a00060b3fdf767ff041f18bf01240021084645
:1010b0001df0d8fa012807d8642019f0f0fb0022af
:1010c000462011460ef00cfa204600f00bfa1a4d9d
:1010d000b4b11a48fff7f4fb1848f7f739ff284670
:1010e000fff7eefb002023f0f8f868662846f7f7d4
:1010f00064ff06a806f074fa13b030bd0446d5e7c5
:10110000204623f0eaf80d4b5866204623f0e5f818
:1011100068660020fff76afefbe700bfb8000c001e
:1011200071d60d0260c30d02130810029cd60d0289
:10113000aed60d0229f700025cd5001078ce001063
:101140002de9f043474b9db00093474b694603930d
:10115000464b04a80293f4f7e1fe4ff440620023eb
:10116000cde9082341f288330a931423adf82c30db
:1011700002233f4c3f223f490df12f008df82e30c6
:10118000b5f07afd20463c4b04a940f8043bf4f747
:10119000c5fe089b04f123026361099b0df16f01f9
:1011a000a3610a9be361bdf82c3023849df82e30a7
:1011b00084f822300df12f0353f8040b8b4242f8d0
:1011c000040bf9d10025142765662c4823f055f946
:1011d0002b4b84f86c502360256704a8f2f764fa5f
:1011e0006846f2f761fa294626481cf049fb264c6e
:1011f000264bdff8c880c4e90173254e254b2946ec
:10120000c4e90334c4f800806661201df1f7c2fd13
:10121000214b29462360214c214bc4e90087a36060
:10122000204b6661c4e90334201df1f7b3fddff8fc
:1012300090901d4bc4f80090a3611c4c1c4b294698
:10124000a3601c4bc4e90087c4e903346661201d18
:10125000f1f7a0fd184bc4f80090a3611db0bde8e4
:10126000f08300bf9d0e01022f5e00021b5e000294
:101270005cd5001000d70d0270c30d02c4d500105c
:10128000f8d60d02c10c01020cd5001006000200b8
:1012900099320002d3d60d0240d70d0240d500107e
:1012a00019000100ded60d02cd06010224d5001082
:1012b0001a000100e7d60d02d1060102a8bc0d02fa
:1012c00050d70d02f0b50246406890b10831d4689d
:1012d00021f003039168201a091a043399424ff050
:1012e000000107d3c4e90013d1680b4401f10800e1
:1012f000d360f0bd0d460846146974b166689e421d
:1013000005d338b14768be423cbf0d462046214652
:101310002468f2e70d462046f9e70028e9d0036883
:101320004db12b602b465169814208bf53610023a8
:1013300040f8083bdde71361f5e7704710b5044658
:10134000182118f0edfa204610bd0000014b586e30
:1013500022f0c5bf5cd50010012a38b5044602d181
:101360000b68236003e0022a03d0032a0dd000207b
:1013700038bd0c200d6818f0cbfa03460028f0d0d9
:1013800095e8070083e80700ebe700680028eed047
:101390000c2118f0c5faeae730b5002939d051f828
:1013a000044cc268a1f108031d19aa4214d1121bf2
:1013b000c2600024426962b35168c3685518ab42e9
:1013c00027d15b1ac360036913b119688a421cd123
:1013d0004361e3b90361ede7056900222c4624b1be
:1013e0009c4238bf22462468f9e72ab905b943610f
:1013f00041f8085c0361dce7146841f8084c1360ad
:1014000041699142d5d14361d3e70b46dce71c60cb
:10141000d0e730bd438c8b4223d890f8203013b1f5
:10142000012b0ad07047012380f82030fa2343842f
:10143000837c43f002038374704790f82420013ac0
:10144000d2b280f8242042b1002380f82030fa2361
:101450004384837c03f0fd03ede711460430f1f78c
:10146000ffba5b1a4384704738b50c4cd4e88f3f01
:1014700013f0010f0a4d09d120461af03ffc28b1a4
:1014800022f098ff286020461af072fc22f092ffaa
:101490002b681b1a5842584138bd00bf24d6001093
:1014a0007cf6001010b50446024b0360f9f7dafd34
:1014b000204610bdfcd80d020148fff7f3bf00bf66
:1014c00054f6001010b50446fff7ecff2046282123
:1014d00018f026fa204610bd014b586e22f0ffbed0
:1014e00078ce0010002210b5044611461046f6f7db
:1014f000f8fd6cb1fdf73efd042805d100231a4626
:1015000019461846f7f756f9bde81040faf7a4bc9b
:10151000fdf730fd0128edd1f0e7000008b5064bde
:101520001b78032b06d105f0d1fabde80840002155
:10153000fef71cb908bd00bf5ed4001070b52d4a7f
:101540008cb01378002b52d0002315781370202212
:10155000cde90423284aedb20092282027490195bd
:1015600004aaf1f799f9264cd4e88f2f12f0010262
:101570001dd1204603921af0c1fb039ab8b1142181
:101580000f20f5f785fd1e2202211e4e0346cde9f0
:10159000002130460f226ff07f4106f099f91a4b77
:1015a000204633601af0e4fb1848b3f0c4fa012d6a
:1015b0001bd8e5b14ff47f060022124c1146201dc6
:1015c000f1f74efafa230022012166616384a37cbd
:1015d000201d03f0fd0384f8245084f82020a37418
:1015e0000cb0bde87040f1f73bba094ee4e70cb02f
:1015f00070bd00bf1ed6001058d70d0260c30d028b
:1016000020d6001054f60010fcd80d023914010247
:101610000060ff00002270b5314d8cb007200df145
:101620000f018df80f20fef749f82b685a1c2a602d
:101630001bb91cf020f92b4b18609df80f301bb321
:101640001cf019f9274e3368c01a274b98421bd952
:1016500000242023cde9043405230193234b04aa5d
:101660000093282023462249f1f716f90122214b45
:1016700034601a70204b2c601c709df80f300bb931
:101680001e4a13600cb070bdf4f746f91c4cc8b18b
:1016900010f1aa0f14d01b4a1b4b10f1a00f08bf6a
:1016a0001a46002320210192184acde90413009222
:1016b00028200f4904aaf1f7eff802232370dce792
:1016c000134aeee72023cde90430124b084900937a
:1016d00004aa03462820f1f7dff80323eee700bf52
:1016e00080f600102cd60010df93040075d70d0291
:1016f00060c30d022dd2001030d6001014d300109c
:101700001ed60010abca0d02e7b70d02c3d70d02fb
:1017100071d70d02dcd70d0208b5074a1378ff2bed
:101720001cbf013313701cf0a6f8044b1860bde811
:101730000840fff76fbf00bf30d6001028d600105a
:1017400000222de9f04111468cb01046f6f710fd4d
:1017500000287ed0404b1b78002b7ad13f4f3b783e
:1017600003f0ff04002b74d12346224652210520aa
:10177000f5f7d0fb1cf07ff8394b1d68394b451b42
:101780001878f8f727fd854263d34ff02008364bd1
:1017900004aa364900931e202346cde90484f1f7bc
:1017a0007bf8faf799fd0122054600f118031a604b
:1017b000402023460021cde901440094f5f7f0fed6
:1017c000eb6e0133eb66f3f7c5ff061e10db01235a
:1017d0003b70274b1e2000932449234604aacde9e1
:1017e0000484f1f759f80cb0bde8f041fff7a6be4c
:1017f000204b01960093282023461c4904aacde9da
:101800000484f1f749f8e63609d12246214606203c
:10181000f5f792fb224621460520f5f78dfb0023c4
:1018200005f118023b70136040201a46cde90133e0
:1018300000930021f5f7b4fe0f4b1b7803f0ff0275
:101840003bb911461046f6f763fd10b9fff764ff88
:10185000c9e70cb0bde8f0812ed200105dd40010b5
:1018600028d6001030d6001004d80d0260c30d0237
:1018700016d80d022dd80d022dd2001008b5032068
:101880000df06eff034b1870bde8084080f00100ba
:10189000faf7fcba84f6001008b5fef741f9fef736
:1018a00043f948b109200df05bff28b1fef738f984
:1018b000bde80840fef746ba08bd08b5002001f0b3
:1018c00055fa40b109200df04bff014618b9bde8ab
:1018d000084001f0b7ba08bd2de9f74f0d460446a0
:1018e000002854d0dff8b4804ff47a79d8f800306b
:1018f000dff8acb00344c8f800301bf0bcff06466c
:101900001bf0b5ff0746002018f0c9ff1bf0b3ff1e
:10191000a0eb060a544534d3621e924510d34ff40f
:101920007a7000fb04741b4d1bf0a1ff201aa84223
:101930002dd84008012828bf012018f0b2fff3e796
:10194000012018f0acff144b1a78002aded1002dcc
:10195000dcd1ca4504d2d8f80020b2f57a7fd5d3bd
:101960000020fdf713fb02460af57a790192f4f79d
:1019700003fe019a002ac9d19bf80030002bf5d153
:10198000c4e725b903b0bde8f04ff4f7f5bd03b0e7
:10199000bde8f08fa08601002ed2001088f600105e
:1019a0005ed4001013b50c4b0446586e019122f022
:1019b00096fc58b1094b01995b68c3f308032bb936
:1019c000204602b0bde81040fff786bf204602b0b7
:1019d000bde8104018f063bf5cd5001000ed00e0da
:1019e0002de9f04fdff8b0b193b005939bf80030cc
:1019f00080460e469246604f1bb93b78002b00f0a4
:101a0000ad8020230024cde90a345c4b1e205c49c4
:101a100000930aaa2346f0f73ffffaf75dfc3b78f4
:101a20000546b3b1c4663eb100f134031e60012e19
:101a300002bf036d01330365032205f118031a6029
:101a40000023092240200021cde901330093f5f75e
:101a5000a7fdfaf745fc4ff00102d0e8cf3fc0e800
:101a6000412f0029f9d1dbb2002bf6d1c268016900
:101a7000047d90f81590c360036103754375c0e859
:101a80008f3fd3075cbf047ae4b2930758bf416825
:101a900053073b7858bf90f8099018f0010f08bf22
:101aa000002413b3002c5fd01023adf81830059b31
:101ab000adf81a60adf81e301c9badf81ca0cde946
:101ac000083106f0dfff0022022106ab06f0cffd51
:101ad00058b120220023cde90a232a4a019000921e
:101ae000282027490aaaf0f7d7feb9f1000f01d044
:101af000f9f7d8fd18f0020f02d12046f3f7aefe39
:101b00000024214b3c701c70204b224621460720ac
:101b10001c708bf80040f5f70ffa2246214606208c
:101b2000f5f70afa224621460520f5f705fa2023a3
:101b3000cde90a34164b0aaa00931e202346104909
:101b4000f0f7aafe224605f118031c604020234648
:101b50000021cde901440094f5f722fd00220d4b50
:101b60001a7013b0bde8f08f06f08cff23462246b2
:101b7000032106f07cfdb8e75ad4001050d80d02be
:101b800060c30d0265d80d025cd400105bd4001058
:101b900097d80d021ed600105dd40010f0b5634b2f
:101ba00005461b788db0002b00f0bd80604f3b7860
:101bb000002b40f0a1805f4b1b7803f0ff04002b4b
:101bc00040f09a805c4e327802f0ff03002a3dd04c
:101bd000faf728fb002800f097802023cde9043491
:101be000564b04aa564900931e202346f0f754fe94
:101bf00001233b70534b34701c70faf76dfb0222cb
